:020000040800F2
:10000000C05E0124DD03000811AF000869A00008EC
:1000100009AF00086912000841CF00080000000085
:10002000000000000000000000000000D1B2000845
:10003000C11900080000000021AF000809B3000842
:10004000FB030008FB030008FB030008FB03000898
:10005000FB030008FB030008FB030008FB03000888
:10006000FB030008FB030008FB03000871120008F3
:100070008112000891120008A1120008B1120008B4
:10008000C1120008FB030008FB030008211A000846
:10009000411A0008311A0008511A0008FB03000831
:1000A000FB030008FB030008FB030008FB03000838
:1000B000FB030008FB030008FB030008FB03000828
:1000C000FB030008FB030008FB030008FB03000818
:1000D000D9B1000801C9000821C9000831C90008C8
:1000E000C9190008FB03000800000000FB0300081A
:1000F000FB030008FB030008FB030008FB030008E8
:10010000FB030008FB030008FB030008FB030008D7
:10011000FB030008F9B80008FB030008FB03000814
:10012000FB030008FB030008FB030008FB030008B7
:10013000FB030008FB030008FB030008FB030008A7
:1001400000000000000000000000000000000000AF
:10015000FB030008FB030008FB030008FB03000887
:10016000FB030008FB030008FB030008FB03000877
:10017000FB030008FB030008FB030008000000006D
:10018000FB030008FB03000819B90008FB03000883
:10019000FB030008FB030008FB030008FB03000847
:1001A000FB030008FB030008FB030008000000003D
:1001B000FB030008FB030008FB030008FB03000827
:1001C000FB030008FB030008000000000000000023
:1001D0000000000000000000FB0300080000000019
:1001E000000000000000000000000000000000000F
:1001F0000000000000000000FB030008FB030008F3
:10020000FB030008FB03000800000000FB030008DC
:10021000FB030008FB030008FB030008FB030008C6
:10022000FB03000800000000FB03000800000000C2
:10023000FB030008FB030008000000005910000841
:10024000FB03000869110008FB030008FB0300081A
:10025000FB030008FB030008FB030008FB03000886
:10026000FB030008FB030008FB030008FB03000876
:10027000FB030008FB030008FB030008000000006C
:10028000FB030008FB030008FB030008FB03000856
:1002900000000000FB030008FB0300080000000052
:1002A00000000000FB030008FB030008FB0300083C
:1002B000F1C80008FB030008FB030008611A0008EE
:1002C000711A0008E9B40008FB03000800F002F806
:1002D00000F074F80AA090E8000C82448344AAF16C
:1002E0000107DA4501D100F069F8AFF2090EBAE86A
:1002F0000F0013F0010F18BFFB1A43F0010318475A
:10030000B4010100D40101000A4410F8014B14F0BB
:100310000F0508BF10F8015B240908BF10F8014B56
:100320006D1E05D010F8013B6D1E01F8013BF9D19F
:10033000641E03D0641E01F8015BFBD19142E4D33B
:10034000704700000023002400250026103A28BF33
:1003500078C1FBD8520728BF30C148BF0B60704737
:10036000692900F05581642900F05281752900F057
:100370004F816F2900F0E681782900F00D82036833
:10038000DB0928BF41F08001632900F0CA85732989
:1003900000F0CF85E32900F0DA85002070471FB513
:1003A0000FF076FF00F01EFE0400002000210FF089
:1003B00059FF401C60601FBD10B510BD00F017FE56
:1003C0001146FFF7ECFF0CF06BFF00F035FE03B4B5
:1003D000FFF7F2FF03BC00F039FE00000A48804737
:1003E0000A4880470A480047FEE7FEE7FEE7FEE7C7
:1003F000FEE7FEE7FEE7FEE7FEE7FEE70548064903
:10040000064A074B70470000F119000811B40008B4
:10041000CD020008C02E0124C05E0124C03E01248C
:10042000C03E012453EA020C00F069802DE9F04B34
:100430004FF00006002B1FBFB3FA83F503FA05F453
:1004400024FA05F65E4012BF1643B2FA82F502FAAC
:1004500005F4C5F120051EBF22FA05FC44EA0C0490
:10046000203556EA044C4FEA144418BF641C4FF080
:1004700000084FF00009904271EB030C39D30029BA
:1004800019BFB1FA81F701FA07F6B0FA80F700FA5E
:1004900007F6C7F120071EBF20FA07FC46EA0C0644
:1004A0002037B6FBF4FCA7EB0507103F07F01F0B46
:1004B000CBF120062CFA06F60CFA0BFB44BFB34630
:1004C0000026202FA4BF5E464FF0000B5BEA060C0F
:1004D00008BF4FF0010B19EB0B0948EB0608ABFB0B
:1004E000027C06FB02CC0BFB03CCC01B71EB0C01A6
:1004F000C1E70B46024641464846BDE8F08B13B5BE
:10050000084318BF4FF0FF300146AFF30080BDE84D
:100510001C4070470FB47CB50C0009AA009001D0B4
:100520002044401E084B7B4469460190089800F027
:10053000CEFC05461CB10020694600F0DBFC2846D5
:100540007CBC5DF814FB0000D509000070B50446C2
:1005500085690068C10601D5302600E02026C00765
:1005600007D070BDD4E9012130469047206A401C75
:1005700020626D1EF6D570BD70B5044685690078A1
:10058000C00707D170BDD4E9012120209047206A1F
:10059000401C20626D1EF6D570BD09684A0501D564
:1005A00040B27047C905FCD500B2704709684A05DA
:1005B00001D5C0B27047C905FCD580B2704770B58F
:1005C0000C460546012A05D02878800600D5EA6940
:1005D000002302E0012305E05B1C934202D2E05CB1
:1005E0000028F9D1A869E618C01AA861286A184439
:1005F00028622846FFF7AAFF04E0D5E9012114F894
:10060000010B9047B442F8D32846FFF7B5FF70BD01
:100610002DE9F0410646002410687529314616A5DB
:1006200010D0FFF7BAFF002802DA404213A507E016
:1006300031688A0701D512A502E0490704D511A542
:10064000012401E0FFF7B2FF00210A2206F124078E
:1006500009E0B0FBF2FCB0FBF2F302FB1C0030300F
:1006600078541846491C0028F3D123462A463046C0
:10067000BDE8F04100F0CDBB000000002D000000FF
:100680002B000000200000002DE9FF5F15468A4680
:100690000446DFF8AC80F8440027D8E900103E4655
:1006A000CDE9001010E03AF816106A4602A800F0F2
:1006B00068FC411C07D02178890603D5E269391806
:1006C00091420DD80744761C2078800602D5E06957
:1006D000B84205DDAE42E6DB3AF816000028E2D16A
:1006E000A069C01BA0612046FFF730FFD8E90010C9
:1006F000CDE90010002017E03AF818106A4602A869
:1007000000F03FFCB0F1FF3F81460BD000250DF11A
:10071000080B05E0D4E901211BF8050090476D1C8A
:100720004D45F7D308F10100B0428046E4DB206A72
:10073000384420622046FFF71FFFBDE8FF9F0000FE
:1007400012FC000070B5044621461068FFF72EFF2A
:10075000002104F1240505E000F007023032C00852
:100760006A54491C0028F7D12068002308A2050715
:1007700008D500F02000084304D0E069012305A259
:10078000401EE0612046BDE8704000F042BB000022
:10079000000000003000000070B504460D46214600
:1007A0001068FFF703FF2188090502D50F4A7A4434
:1007B00002E00E4A7A440E32002104F1240305E0DF
:1007C00000F00F060009965D5E54491C0028F7D121
:1007D00020780023000704D5702D02D009B1022330
:1007E00011322046BDE8704000F013BB02FB000050
:1007F0002DE9F05F894604464FF0000ADFF874B136
:10080000FB44C0F820A02046E1688847002874D047
:10081000252806D0D4E901219047206A401C206297
:10082000F1E700265F462046E16888472028054614
:1008300007DB312D05D2781910F8200C08B10643DA
:10084000F1E7B00701D526F00406C4F81CA0002784
:10085000C4F818A02A2D09D028460FF0FBFC38B3A5
:1008600004EB8708303DC8F8185019E059F8041B0C
:10087000204604EB87029161E1688847012F054615
:1008800018D1E069002820DA26F020061DE0D8F80B
:10089000180000EB800005EB40003038C8F8180065
:1008A0002046E168884705460FF0D4FC0028EED1C9
:1008B000012F0AD02E2D08D12046E16888477F1CE1
:1008C0000546022F46F02006C4DBA069002803DAA3
:1008D000404246F00106A061F00701D026F0100664
:1008E0006C2D0BD0682D09D04C2D39D06A2D35D008
:1008F000742D35D07A2D33D016E038E0E1682F46DC
:1009000020468847B842054609D16C2F26D04FF4BF
:100910008060E168064320468847054604E06C2F66
:100920001AD04FF4807006430DB3A5F14100192889
:1009300002D8203546F400664A46294620462660FD
:100940004E46FFF70DFD80B101280BD0F61D26F0B5
:10095000070000F1080956E74020E4E78020D8E7C7
:100960000020D6E706F104094DE7284652E7206A41
:10097000BDE8F09FD8FA00002DE9FF5F1D464FF05B
:10098000FF3B91464FF000085F46D5E90146A96953
:1009900001987F1C8847296A824688470028F6D13B
:1009A000BAF1FF3F0CD0002E24F4C06419DD6006BC
:1009B00014D5BAF12B0F09D0BAF12D0F0ED103E0E7
:1009C000584604B0BDE8F09F44F48064A9690198DA
:1009D0007F1C8847761E8246002E02DDBAF1300F5A
:1009E00003D0B9F1000F26D032E0A969761E019834
:1009F0007F1C44F400748847002E824605DDBAF15E
:100A0000780F06D0BAF1580F03D0B9F1000F10D00B
:100A10001EE0B9F1000F02D0B9F1100F18D1A96989
:100A2000761E01987F1C24F40074884782461020AB
:100A300002E0082000E00A20814609E0A96908FBDD
:100A40000908761E01987F1C44F40074884782468A
:100A5000002E05DD4946504600F085FA0028EDDA03
:100A6000E96901988847A00502D46FF00100A8E762
:100A7000E00725D1600613D5600502D5C8F1000056
:100A800000E0404629680A1D2A600968220501D550
:100A9000087015E0220701D5088011E008600FE01A
:100AA0002868011D29600068210502D580F80080B2
:100AB00006E0210702D5A0F8008001E0C0F8008020
:100AC00038467EE72DE9FF5F4FF00008994614464F
:100AD00046469169D2E901A7DDF838B00198884708
:100AE000054659EA0B0005D009E0A1690198761C7A
:100AF00088470546216A284688470028F5D1681CA2
:100B000003D05FEACA7005D015E04FF0FF3004B0A3
:100B1000BDE8F09F2068011D2160D0F800800AE048
:100B20005FEACA7001D108F8015BA169761C0198DF
:100B30007F1E88470546002F1ADD681C18D0B9F1C2
:100B4000000F0DD0E81705EBD060421120F01F0018
:100B500059F822102A1A012090400142E0D107E002
:100B6000BBF1000FDCD12846216A88470028D7D086
:100B7000E16901988847BBF1000F07D1002E05DD20
:100B80005FEACA7002D1002188F80010A068B8425C
:100B900003DDBBF1000F03D017B16FF00100B6E722
:100BA0003046B4E7032A40F2308010F0030C00F026
:100BB000158011F8013BBCF1020F624498BF11F897
:100BC00001CB00F8013B38BF11F8013BA2F1040250
:100BD00098BF00F801CB38BF00F8013B11F00303C8
:100BE00000F02580083AC0F0088051F8043B083A2C
:100BF00051F804CBA0E80810F5E7121D5CBF51F8CE
:100C0000043B40F8043BAFF30080D20724BF11F847
:100C1000013B11F801CB48BF11F8012B24BF00F8AC
:100C2000013B00F801CB48BF00F8012B704710B51D
:100C3000203AC0F00B80B1E81850A0E81850B1E895
:100C40001850A0E81850203ABFF4F5AF5FEA027CD4
:100C500024BFB1E81850A0E8185044BF18C918C004
:100C6000BDE810405FEA827C24BF51F8043B40F8A5
:100C7000043B08BF7047D20728BF31F8023B48BF8A
:100C800011F8012B28BF20F8023B48BF00F8012BC8
:100C9000704702F0FF0343EA032242EA024200F0F7
:100CA00024B84FF000020429C0F0128010F0030CA9
:100CB00000F01B80CCF1040CBCF1020F18BF00F84F
:100CC000012BA8BF20F8022BA1EB0C0100F00DB8FE
:100CD0005FEAC17C24BF00F8012B00F8012B48BF5C
:100CE00000F8012B70474FF0000200B51346944600
:100CF0009646203922BFA0E80C50A0E80C50B1F174
:100D00002001BFF4F7AF090728BFA0E80C5048BF87
:100D10000CC05DF804EB890028BF40F8042B08BF25
:100D2000704748BF20F8022B11F0804F18BF00F821
:100D3000012B704710B5044610F0030F08BF11F0E7
:100D4000030F40F015804FF0013E121FC0F20E80DD
:100D500051F8043BA3EB0E0C2CEA030C1CEACE1C4E
:100D600008BF40F8043BF0D0A1F1040102F10402F5
:100D7000521E08DB11F8013B00F8013B002BF7D1B4
:100D80001146FFF78EFF204610BD00000000000056
:100D900030B44FF0013C50F8042BCCFA52F451F827
:100DA000043BD51A20D1FCB950F8042BCCFA52F4EC
:100DB00051F8043BD51A17D1B4B950F8042BCCFA2A
:100DC00052F451F8043BD51A0ED16CB950F8042BEB
:100DD000CCFA52F451F8043BD51A05D1002CDAD0E4
:100DE00030BC4FF00000704729BAB1FA81F111F020
:100DF0001801D1F120008440F2D1CA40CB4012F05A
:100E0000FF0213F0FF0330BCD01A704770477047E1
:100E100070472DE9F0470D4699469246044600F189
:100E200024080168880604D5E06921F010012160DA
:100E300000E00120A84201DD471B00E00027A16976
:100E40007A1902EB0900081AA0612078C00602D4C2
:100E50002046FFF77BFB002608E0D4E901211AF8C1
:100E600006009047206A401C761C20624E45F4DB49
:100E70002078C0060AD52046FFF768FB06E0D4E9D3
:100E8000012130209047206A401C2062381EA7F1C3
:100E90000107F4DC07E0D4E9012118F805009047C8
:100EA000206A401C2062281EA5F10105F3DC2046C3
:100EB000FFF762FB2078000602D50220BDE8F0872C
:100EC0000120FBE701694A1C02610878704700B500
:100ED0008FB0CDE901310021059105497944CDE973
:100EE000031011466846FFF783FC0FB000BD0000F9
:100EF000E5FFFFFF0A6802F8010B0A607047D1E9BD
:100F000000239A4202D2531C0B601070704710B538
:100F1000436913B1AFF3008001E0FFF750FB0120FC
:100F200010BD127800F124010A7000224A700122DB
:100F3000EDE711684FF0FF32E9E710B5436913B1EF
:100F4000AFF3008001E0FFF79FFB012010BD128886
:100F500000F1240182840022C2840122EDE711689D
:100F60004FF0FF32E9E73A2800D2303820F0200273
:100F7000412A01D3A2F13700884201D34FF0FF305C
:100F800070472DE9F04116460C46054600F022F860
:100F9000036893F80101012807D0FF2C12D8185DCF
:100FA00080B101202C70BDE8F081D3F807013246F2
:100FB000214603F20713C7182846BC46BDE8F04196
:100FC000002360474FF0FF30EDE700000048704716
:100FD000280D002410B500F005F8001D10BD00BF5D
:100FE00085F2000000487047480D002470477546A0
:100FF000FFF7ECFFAE4605006946534620F00700B8
:10100000854618B020B5FFF7F9F9BDE820404FF04C
:1010100000064FF000074FF000084FF0000BAC4601
:10102000ACE8C009ACE8C009ACE8C009ACE8C0094C
:1010300021F007018D46704710B50446AFF30080DC
:101040002046BDE81040FFF7C2B900000149182052
:10105000ABBEFEE72600020041F2B000C2F2004043
:1010600001F0F6B80000000010B50446006842F236
:10107000001140F48070C4F20201884218D142F29B
:101080000830C4F20200006810F4403F18D006F0A7
:101090009FFA6168B1F5803F05D0B1F5403F2BD094
:1010A000B1F5003F29D1090CB0FBF1F025E000BFFC
:1010B00046F20830C5F60200006810F4403FE6D161
:1010C0004FF40020002105F083F96168A1F580222A
:1010D0004FEAB2420A2A10D8DFE802F006060606F6
:1010E00006063C3E404244006FF0010202EA5141D4
:1010F000B0FBF1F001E000BF80084BF62141C0F2E7
:10110000BE01884206D82068816821F44071816060
:1011100010BD00BF47F64101C0F27D11884207D8DB
:1011200020680122816862F30921816010BD00BF3F
:1011300021684FF28102C0F2FA229042886805D8F5
:10114000022262F30920886010BD00BF40F44070A5
:10115000886010BD0009D0E74009CEE78009CCE7E0
:10116000C009CAE7000AC8E741F29810C2F200407D
:1011700001F0CEBF000000002DE9F0410CF020F995
:1011800004460EF0C5FD4EF218074FF47A78CEF201
:101190000007B8FBF4F404FB00F63D680EF0B8FD60
:1011A00060433968864200FB08F008BF294657F8BB
:1011B000042C01FB08F10132B1FBF2F1401A0021CD
:1011C00000F57A70BDE8F08141F6146242F26401E4
:1011D000C2F20042012818BF0022C2F200410028DA
:1011E00018BF1146084670470068C169C90658BF54
:1011F000704745F200010323C4F2000101F54042AB
:10120000904240F6987208BF0123411AC2F2004290
:1012100018BF194601EBC10102EB810110220262E5
:10122000086A08B1004700BF7047000000000000D6
:1012300032B1FF23012898BF082905D958B2704759
:10124000FE2358B2704700BF00EBC00040F6987311
:10125000C2F2004303EB8000002340F8212058B283
:101260007047000000000000FEE7000000000000E2
:1012700041F22010C2F2004001F04ABF000000001D
:1012800041F21020C2F2004001F042BF0000000015
:1012900041F28820C2F2004001F03ABF0000000095
:1012A00041F20030C2F2004001F032BF0000000005
:1012B00041F2F030C2F2004001F02ABF000000000D
:1012C00041F27830C2F2004001F022BF000000007D
:1012D00040F20F42D0F800C0C4F20202944511DC83
:1012E0006F22C4F20202944522DC3F22C4F20202C1
:1012F000944539DC1022C4F2020294455AD02822C7
:1013000054E000BF40F26F42C4F2020294451BDC7D
:1013100040F23F42C4F2020294452DDC40F21042FA
:10132000C4F20202944545D040F228423EE000BF9C
:101330009F22C4F20202944528DC7022C4F2020209
:10134000944537D0882231E040F29F42C4F2020235
:10135000944523DC40F27042C4F20202944529D045
:1013600040F2884222E000BF4022C4F202029445CB
:1013700020D058221AE000BF40F24042C4F20202DC
:10138000944517D040F2584210E000BFA022C4F2AA
:10139000020294450ED0B82208E000BF40F2B842E5
:1013A000C4F20202944505D040F2A042C4F2020207
:1013B000944519D16FF00F024AF6AB2352FA8CF222
:1013C000CAF6AA23A2FB03310AA35F2AC1F30211C2
:1013D0005B5C40F2FF312CEA0101C36588BF043138
:1013E00081650846704700BF2CF0FF018165084603
:1013F000704700BF0006101600061016000000001F
:1014000070B540F26F44D0F800C0C4F20204D0F8C6
:1014100058E0A4451ADC9F25C4F20205AC4533DC34
:101420005725C4F20205AC455ADC1025C4F202056A
:10143000AC4500F098802825C4F20205AC4500F0C8
:1014400092804025C4F202058AE000BF45F22F4594
:10145000C5F60205AC452DDC40F2B745C4F20205E5
:10146000AC454BDC40F27045C4F20205AC457AD085
:1014700040F28845C4F20205AC4574D040F2A04564
:10148000C4F202056CE000BF40F22745C4F2020539
:10149000AC4543DCA025C4F20205AC4563D0B825B9
:1014A000C4F20205AC455ED040F21045C4F202051C
:1014B00056E000BF45F26B45C5F60205AC453FDC82
:1014C00045F23045C5F60205AC454CD045F24445E1
:1014D000C5F60205AC4546D045F258453EE000BF92
:1014E0005825C4F20205AC453DD07025C4F2020572
:1014F000AC4538D08825C4F2020531E040F2B84549
:10150000C4F20205AC452ED045F20845C5F60205E9
:10151000AC4528D045F21C4520E000BF40F22845EC
:10152000C4F20205AC451ED040F24045C4F20205AB
:10153000AC4518D040F25845C4F2020510E000BF97
:1015400045F26C45C5F60205AC450CD045F2944514
:10155000C5F60205AC4506D045F28045C5F6020544
:10156000AC4540F0D580456EC66E002E866E6E602E
:101570001CBFD0E91C566E60A44515DC9F24C4F244
:101580000204A4452CDC5724C4F20204A44551DC17
:101590001024C4F20204A4457AD02824C4F2020420
:1015A000A44575D040246FE045F22F44C5F60204EF
:1015B000A44529DC40F2B744C4F20204A44545DC4A
:1015C00040F27044C4F20204A44561D040F2884461
:1015D000C4F20204A4455BD040F2A04454E000BF32
:1015E00040F22744C4F20204A4453FDCA024C4F224
:1015F0000204A4454CD0B824C4F20204A44547D048
:1016000040F2104440E000BF45F26B44C5F60204CE
:10161000A44555DC45F23044C5F60204A44561D02A
:1016200045F24444C5F60204A4455BD045F2584453
:1016300054E000BF5824C4F20204A44528D070240A
:10164000C4F20204A44523D088241DE040F2B8442B
:10165000C4F20204A4451BD045F20844C5F60204B6
:10166000A4453FD045F21C4438E000BF40F2284476
:10167000C4F20204A4450BD040F24044C4F2020478
:10168000A44505D040F25844C4F20204A4453FD119
:101690008468C06D00F01F003F2505FA00F0CEF809
:1016A0000800DCF80000402C20F48020CCF800007A
:1016B000CCF8043023D0CCF80810CCF80C2070BD46
:1016C00045F26C44C5F60204A4450BD045F28044B3
:1016D000C5F60204A44505D045F29444C5F60204BB
:1016E000A44515D1C46D806804F01F04012540286D
:1016F00005FA04F4CEF80440CCF8043004D1CCF858
:101700000820CCF80C1070BDCCF80810CCF80C20D8
:1017100070BD000000000000B0B5D8B140F6D8643C
:10172000C2F20044207818B1FD2568B2B0BD00BFF8
:101730000CF06AF8606068B141F679120020C0F6DA
:10174000000203210025FFF773FD0120207068B21D
:10175000B0BD00BFFE2568B2B0BD000000000000B3
:1017600010B538B13421002400F8244BFFF7BBFA40
:1017700060B210BDFE2460B210BD00000000000089
:10178000B0B508B30546044655F8100F01466FF38F
:10179000DF21A1F5B671B1F5A56F11D8C0F3CA214B
:1017A000A1F5B671B1F5A56F0AD8A988800D40EAF8
:1017B00081206FF3DF20A0F5B670B0F5A56F07D9D3
:1017C000FF2040B2B0BD00BFFE2040B2B0BD00BFA0
:1017D00011F4405F4FF0FF0000F0C5808AB2B2F50F
:1017E000804FC0F0C080C1F34A01A1F5B671B1F5D8
:1017F000A56F00F2B88001202070FFF7BDFC2A68B9
:1018000094F81CC013466FF3DF23BCF1000F00EE09
:10181000103AA369C4E90201C2F3CA20A988B8EE4C
:10182000401A9FED520AE36331EE001A31EE012AAD
:1018300001EE100A4FEA925040EA81206FF3DF2058
:10184000B8EE413A04EE100A9FED491AC1F34A007E
:1018500082EE012A05EE100A33EE003AB8EE444A51
:1018600084ED0B2A4FEA913284F83920B8EE455ABC
:10187000E28A34EE004A4FF0000033EE033A60652E
:10188000C1F3013135EE005A34EE044A84F83810C1
:1018900083EE013A628735EE052A84ED0C3A84EE38
:1018A000013A627F84ED093A82EE012A84ED0A2A28
:1018B00018BF4FF0010C002A84F840C018BF012265
:1018C000E38B84F852C084F84120DDB203F00101BB
:1018D00084F84210C5F3400184F84310C5F3800139
:1018E00084F84410C5F3C00184F84510C5F3001115
:1018F00084F84610C5F3401184F84710C5F38011F1
:1019000084F84810E90984F84910C3F3002184F8E9
:101910004A10C3F3402184F84B10C3F38025218C77
:1019200084F84C5002EE101A84F85320C3F3C021FF
:1019300084F84D10C3F3003184F84E10C3F34031E6
:10194000B8EE422A84F84F10C3F3803184F8501067
:1019500032EE000AD90B84F8511030EE000A80EE06
:10196000010A84ED0D0A40B2B0BD00BF000080C482
:101970000000A5440000000040F6D8600121C2F23A
:10198000004040680BF048BE10B504460020FFF749
:101990001BFC04F11001122208F00EFA002818BFF7
:1019A0004FF0FF3010BD000080B50246012001213C
:1019B0000BF076FE0138B0FA80F0400980BD0000DF
:1019C000704700000000000080B54FF4806003F015
:1019D000CFFA4FF48050BDE8804003F0C9BA000050
:1019E000EFF3108072B600BFFEE7000000000000B9
:1019F00044F60400C5F60200816841F002018160EE
:101A00000168890409D4016889045CBF01685FEA40
:101A1000814102D401688904F2D5704700000000BA
:101A200041F26840C2F2004002F0EEBC000000004B
:101A300041F26840C2F2004002F0E6BC0000000043
:101A400041F20850C2F2004002F0DEBC000000008B
:101A500041F20850C2F2004002F0D6BC0000000083
:101A600041F2A850C2F2004002F0CEBC00000000DB
:101A700041F2A850C2F2004002F0C6BC00000000D3
:101A800070470000000000007047000000000000E8
:101A900070470000000000007047000000000000D8
:101AA0007047000000000000B0B582B090F85C20E4
:101AB000012A03D10221084602B0B0BD42F2083229
:101AC00000230193C4F202020093A2F5427403685A
:101AD000A34227D14FF6006C4FF60055CFF6FF7C9E
:101AE000CFF6FF7552F80C40535923435B0719D4C6
:101AF000D1F800E01368BEF1000F23F440441DD07C
:101B00004B6823431360535952F80C502B43DB07A7
:101B100022D1136840F61F758968AB4341EA0E0174
:101B2000194316E0016E41F02001016601210022F7
:101B300080F85C20084602B0B0BD00BF1460515967
:101B400052F80C301943C90708D1116840F61F73C9
:101B5000994311600021EAE70021E8E70021E6E768
:101B60002DE9F04181B00022009290F85C20012A1A
:101B700004D10221084601B0BDE8F08103680122CA
:101B800080F85C209A68520700F1FC8246F2083C1B
:101B90004FF6FF78C5F6020CC0F20F08ACF5427E96
:101BA0000A68734516D0B2F1FF3F13DD92FAA2F531
:101BB00012EA080FB5FA85F54FF0010608BF950E39
:101BC000920E05F01F0506FA05F5DE693543DD6165
:101BD00001E000BF920E4D681F2402F01F02C5F302
:101BE000012605F01F05AC4003EB8606AA40376BC3
:101BF00027EA0404224332639A689C68E40844EAB2
:101C00009202D20740F029810A6807268D68734541
:101C1000C2F34064C2F3045203EB840406FA02F6F2
:101C2000676905FA02F227EA060642EA06026261DD
:101C300010D041F20002C5F60042126802F0704274
:101C4000B2F1805F6ED14A69DC680E2505EA540660
:101C50009CE000BF4FF604540A69CFF6FF74042AD3
:101C60004D695CF8046067D14FF65852CFF6FF72A9
:101C70005CF802201C6E0E68C4F3846416EA080245
:101C8000C6F3846596FAA6F6B6FA86F6374608BF16
:101C90002F46BC420CD11A6E22F000421A660C6824
:101CA00004EA0802C4F3846594FAA4F4B4FA84F64E
:101CB0005C6E37465C6E002A08BF2F46C4F384640E
:101CC000BC420CD15A6E22F000425A660C6804EAFB
:101CD0000802C4F3846594FAA4F4B4FA84F69C6E02
:101CE00037469C6E002A08BF2F46C4F38464BC426A
:101CF0000CD19A6E22F000429A660C6804EA08023F
:101D0000C4F3846594FAA4F4B4FA84F6DC6E002A71
:101D1000DC6E08BF2E46C4F38462B24200F09980A4
:101D20009BE000BFDC684A69DD68E4064FEA5505C0
:101D30002AD405F00E0629E00624ACF52A7704EA39
:101D400096040E6805FA04F406F0F8452C4357F89B
:101D5000226044F0004447F822400A69CC6957F8F1
:101D6000225025F080752C4347F822400A6991F8EB
:101D7000204057F82250012C25F0007508BF05F1CE
:101D8000007547F8225068E005F008060F6903F176
:101D90006005042F20D12A680C6802F0F842B2EBEB
:101DA000846F4FEA846241D12C6824F000442C6097
:101DB0005C6E04F0F84494423DD09C6E04F0F8440C
:101DC000944241D19C6E24F000449C66DC6E04F089
:101DD000F844944241D13CE00C68B24055F8276089
:101DE00004F0F84406F000462243324345F8272029
:101DF0000A6991F8214055F82260012C26F000462E
:101E000008BF06F1004645F822600A7E0C691D698C
:101E1000013A04F01F04B2FA82F225F4F0455209A7
:101E2000D202A2402A431A6117E000BF5C6E04F0A0
:101E3000F8449442C1D15C6E24F000445C669C6E10
:101E400004F0F8449442BDD0DC6E04F0F8449442AF
:101E500003D1DA6E22F00042DA669A68D20711D115
:101E600073450A68CD680FD005F01804D3F8C01088
:101E700028FA04F402EA0806B14314402143C3F8E7
:101E8000C01012E0002182E14FF6A85105F01806BB
:101E9000CFF6FF7128FA06F602EA080716405CF84A
:101EA0000140BC4334434CF801400021C4F252715C
:101EB00001F52D04A54240F0138146F20004C5F659
:101EC0000204A3422CD042F20014C4F20204A34242
:101ED0003CD042F20004C4F20204A34250D11F24B9
:101EE000C1F2F044A24275DD40F2FF74C2F63064E4
:101EF000A2425FDD40F60004C2F63064A24200F068
:101F0000BF8041F20004C3F26024A24200F0B2801C
:101F10000024C4F22134A24200F0CD80B6E000BF1C
:101F20001F21C1F2F0418A422CDC0721C0F690410A
:101F30008A426DDC0221C0F230418A4254D0042131
:101F4000C0F660018A4216D0AAE000BF1F21C1F28C
:101F5000F0418A4228DC0721C0F690418A4245DCE4
:101F60000221C0F230418A423ED00421C0F6600115
:101F70008A4240F08B804021C1F620119BE000BFD7
:101F8000002198E040F2FF71C2F630618A4253DCD2
:101F90002021C1F2F0418A4234D040F20041C2F621
:101FA00000218A4211D07BE040F2FF71C2F630611D
:101FB0008A4253DC2021C1F2F0418A4222D040F211
:101FC0000041C2F600218A4260D140F60001C2F60B
:101FD000306170E00721C0F690418A4206DC0221A0
:101FE000C0F230418A42C0D1012164E00821C0F62C
:101FF00090418A421CD01021C1F2C0018A4211D006
:1020000044E000BF40F20021C2F2B05153E000BFF3
:102010000821C0F690418A420AD01021C1F2C001C5
:102020008A423DD140F20011C2F2801143E000BF6C
:102030008021C1F650513EE040F60001C2F6306109
:102040008A421DD042F20001C3F290618A4227D138
:1020500044F20001C3F6C0212DE000BF40F60001AC
:10206000C2F630618A420BD041F20001C3F2602116
:102070008A420BD142F20001C3F290611BE000BF23
:1020800041F20001C3F2602115E000BF00240021ED
:10209000C4F68434A24204BF0021C4F6B8710AE039
:1020A00044F200040021C3F6C024A24204BF48F257
:1020B0000001C3F6F061734512D091FAA1F44FF616
:1020C000C135B4FA84F4C0F20A05294208BF8C0E67
:1020D00004F01F01012404FA01F1DC692143D961F4
:1020E000B2F1FF3F02DD002151E000BF42F20001EA
:1020F00042F20016C4F20201C4F2020601F5807435
:1021000001F54275A342644608BF2C468B4208BFC6
:102110002C4643F48075B54225682BD18C68D1F8E4
:1021200008112143C9072DD1002105F0E074CCF23C
:1021300052718A4208BF15F400012FD00021CCF261
:1021400021318A4208BF15F080712BD00021CCF6D6
:1021500084318A424FF0000119D115F4800208BF82
:10216000734514D1DCF8001021F0E071214341F4F3
:10217000800156E04FF60051CFF6FF715CF8011078
:10218000C907D1D0016E41F0200101660121002272
:1021900080F85C20084601B0BDE8F081734505D0A9
:1021A0000021F4E7734535D00021F0E7DCF800109A
:1021B00042F6635221F0E071C0F23E52214341F4F5
:1021C0000001CCF8001040F20801C2F20041096899
:1021D0008909A1FB02129109022202EB410100913F
:1021E000009919B3009901390091009901B3009940
:1021F000013900910099E9B10099013900910099E4
:10220000D1B1009901390091009900294FF00001E6
:10221000E8D1BCE7DCF8001021F0E071214341F087
:102220008071CCF800100021B1E700BF0021AEE7BB
:102230000021ACE70021AAE70021A8E70000000088
:102240007047000000000000704700000000000020
:102250002DE9F04F81B046F2083942F200080446F9
:102260000068C5F60209C4F2020808F5807B08F58B
:1022700042774A460168584508BF3A464045436898
:1022800008BF3A4603EA0105A90716680CD5206E77
:10229000C00603D4206E40F4006020662046FFF79D
:1022A000EFFB20680221016015F00C0F06F01F0AF9
:1022B00044D0216EC90603D4216E41F40071216619
:1022C000C16811F4406F33D10146584508BF4146FB
:1022D000814218BF0946BAF1000F08BF0146BAF1A2
:1022E000050F08BF0146BAF1090F08BF0146C968CA
:1022F00089041DD4016809071AD5816849070FD4DC
:10230000416821F00C014160206E20F4807020664D
:10231000206EC0040CD4206E40F00100206607E05F
:10232000206E40F010002066606E40F00100606694
:102330002046FFF785FF20680C21016015F0600F33
:1023400022D0216EC90603D4216E41F400512166CA
:102350000146584508BF414606F01E02814218BF9B
:102360000946BAF1000F08BF0146062A08BF014618
:10237000C26C12F4C07FC268C9686BD02046FFF7F8
:1023800083FB20686021016029060BD4E90515D480
:10239000A90520D4E9062BD4690549D401B0BDE8CC
:1023A000F08F00BF206E40F480302066204600F0A1
:1023B00003FA206880210160E905E9D5206E40F428
:1023C000003020662046FFF767FB20684FF48071DD
:1023D0000160A905DED5206E40F4802020662046ED
:1023E000FFF75EFB20684FF400710160E906D3D56A
:1023F000E16B69B1BAF1000F52D0584508BFB94638
:10240000404508BFB946D9F8001011F4404F0BD031
:10241000206E40F480602066606E40F002006066CE
:102420002046FFF711FF2068102101606905B5D52E
:10243000216E41F480412166616E41F008016166C0
:102440004FF480610160204601B0BDE8F04FFFF716
:102450001FBB00BF8B0106D502F4406201F400539C
:10246000D2187FF48BAF890201683FF587AF11F076
:1024700040013FF483AF8168090715D4416821F01A
:1024800060014160206E20F480502066206EC005FF
:102490003FF574AF206E40F0010020666EE700BF8C
:1024A000C1688907B4D1BFE7206E40F010002066F4
:1024B000606E40F00100606660E700000000000010
:1024C000B0B582B0044600284FF00000019009D05A
:1024D000206E58B120688168890012D48168C900D3
:1024E00019D54EE00125284602B0B0BD204600F0C7
:1024F00067F90020606684F85C00206881688900C4
:10250000ECD54FF6C0728168C5F6FF72114081604C
:102510008168C90035D44FF6C0718268C5F6FF7175
:1025200001F18051114042F6635201F18051816006
:1025300040F20801C0F23E52C2F200410968890926
:10254000A1FB0212012101EB921101910199C1B18C
:10255000019901390191019900291FBF01990139A0
:10256000019101991FBF00290199013901911CBFF7
:102570000199002905D0019901390191019900299A
:10258000E6D18168C90009D4216E012541F010010E
:102590002166616E41F00101616600E000258168FD
:1025A000226E02F01002C1F380018918216E07D05B
:1025B00041F0100001252066284602B0B0BD00BFE2
:1025C00021F4817146F2100C023121668168C5F652
:1025D000020CC90724D142F2001240F48071C4F207
:1025E0000202914242F20001C4F2020140F0A080D6
:1025F0008A68D1F808311A43D20711D101F58072E7
:1026000001F5427390421A4618BF0CF53E7288429B
:1026100008BF1A466168136823F47C1319431160DC
:10262000617EE36BACF1100E704543EA413121D07D
:10263000A268114394F82020012A41EA024306D1FE
:10264000616A0022CFF6FE7202EB41410B43A16AA0
:1026500029B101F47871E26A194341EA0203704535
:1026600016D04CF20302C168CFF6F0721140194344
:10267000C1601FE0D4E90232082B41EA02015DD0BB
:102680000C2B5FD01C2B61D110231943D2E700BF64
:1026900044F207025CF8041CCFF6F07211401943B3
:1026A0004CF8041CDCF80010626B21F0406111430F
:1026B000CCF8001081688268D20842EA9101C9070B
:1026C00065D1217E70454FEA813103D0226B1143E1
:1026D00004E000BF94F8382041EA4201C26844F2A5
:1026E00003039A431143C16094F84410012919D19E
:1026F0004FF61E017045CFF600412DD0026902EA67
:10270000010C0021D4E91223CFF6FF7101EB024145
:102710004CEA0302236D1143626D1943114341F0EA
:10272000010102E0016921F00101016123E000BF24
:102730005CF8082CD2073FF461AF71E7002319431E
:1027400078E700BF0823194374E700BF182B18BFB0
:10275000002319436EE700BFDCF800201140D4E9E4
:1027600012231143226D1943636D1143194341F044
:102770000101CCF800100169226C21F07041704514
:1027800041EA0201016102D02046FEF76DFC20689B
:102790002169026B012922F00F0102D1E269013A9D
:1027A000114301630121206E61F301002066284678
:1027B00002B0B0BD00000000704700000000000043
:1027C0002DE9F04186B0044646F20002C5F6020249
:1027D0000020216805909142049067D042F20000E9
:1027E000C4F20200814240F0948044F2E0400025AF
:1027F000C5F60200C5F6020501AE4FF0030850F819
:10280000081C002741F0200140F8081C50F8081C63
:1028100001F0200100910099016841F0010101607F
:10282000016801F0010100910099016841F0040183
:1028300001600068314600F00400009000982020FC
:1028400001902846CDF80880039702F09DFB1020E8
:102850003146CDE9010805F50060039702F094FBCD
:1028600041F220151020C2F20045C4F20200286097
:102870000920C5E901074FF4806028614FF400602A
:1028800068614FF40050A8614FF48070EF60C5E9B3
:10289000070728466F6201F057F808B1FFF7A0F864
:1028A000A565AC6306B0BDE8F08100BF44F2E0412D
:1028B00041F29815C5F60201C2F200450A6842F0DD
:1028C00080720A600A6801F6287102F08072009234
:1028D000009A29601121E860C5E901104FF4806178
:1028E00029614FF4006169614FF400512862C5E924
:1028F0000610284601F028F808B1FFF771F87F208C
:1029000005210022A565AC6302F0FEFC7F2002F0E9
:10291000EBFC06B0BDE8F0812DE9F041044602F081
:102920002FFC0CB3054694F83500022820D140F264
:102930000F472668C4F2020740F26F48BE42C4F255
:1029400002081DDC6F20C4F2020086422ADC3F2010
:10295000C4F20200864241DC1020C4F2020086422A
:1029600063D028205CE000BF0120BDE8F08100BFFB
:10297000802060650120002184F83410BDE8F081DA
:1029800046451BDC40F23F40C4F2020086422DDC8B
:1029900040F21040C4F20200864246D040F2284085
:1029A0003EE000BF9F20C4F20200864228DC702077
:1029B000C4F20200864238D0882031E040F29F40C5
:1029C000C4F20200864223DC40F27040C4F20200EE
:1029D00086422AD040F2884022E000BF4020C4F264
:1029E0000200864221D058201AE000BF40F2404049
:1029F000C4F20200864218D040F2584010E000BFF6
:102A0000A020C4F2020086420FD0B82008E000BF28
:102A100040F2B840C4F20200864206D040F2A04024
:102A2000C4F20200864240F099813146306820F0BD
:102A30001E0041F8140B6FF080000A68464500EA5A
:102A4000020008601ADC9F20C4F20200864233DCD8
:102A50005720C4F2020086425ADC1020C4F2020061
:102A6000864200F097802820C4F20200864200F0DF
:102A700091804020C4F202008AE000BF45F22F405E
:102A8000C5F6020086422DDC40F2B740C4F20200D7
:102A900086424BDC40F27040C4F20200864279D09C
:102AA00040F28840C4F20200864273D040F2A04057
:102AB000C4F202006CE000BF40F22740C4F2020002
:102AC000864243DCA020C4F20200864262D0B820D5
:102AD000C4F2020086425DD040F21040C4F202000F
:102AE00056E000BF45F26B40C5F6020086423FDC6F
:102AF00045F23040C5F6020086424BD045F24440D4
:102B0000C5F60200864245D045F258403EE000BF7F
:102B10005820C4F2020086423CD07020C4F2020069
:102B2000864237D08820C4F2020031E040F2B8403B
:102B3000C4F2020086422DD045F20840C5F60200DC
:102B4000864227D045F21C4020E000BF40F22840DA
:102B5000C4F2020086421DD040F24040C4F202009E
:102B6000864217D040F25840C4F2020010E000BF85
:102B700045F26C40C5F6020086420BD045F2944007
:102B8000C5F60200864205D045F28040C5F6020037
:102B9000864204D1206E016821F4807101603068A2
:102BA00020F00100306000BF3068C00710D002F094
:102BB000E7FA401B0628F7D320206065032084F83D
:102BC00035000120002184F83410BDE8F08100BFF9
:102BD0002068B84210DC6F21C4F2020188421DDC7B
:102BE0003F21C4F20201884234DC1021C4F2020108
:102BF000884255D028214FE040451BDC40F23F4140
:102C0000C4F2020188422DDC40F21041C4F20201FC
:102C1000884245D040F228413EE000BF9F21C4F2E7
:102C20000201884228DC7021C4F20201884237D0B8
:102C3000882131E040F29F41C4F20201884223DC46
:102C400040F27041C4F20201884229D040F288412A
:102C500022E000BF4021C4F20201884220D0582166
:102C60001AE000BF40F24041C4F20201884217D08E
:102C700040F2584110E000BFA021C4F20201884296
:102C80000ED0B82108E000BF40F2B841C4F2020102
:102C9000884205D040F2A041C4F20201884261D1CD
:102CA000D4E9161202F01F023F2303FA02F28A60EF
:102CB000404561DC9F21C4F20201884214DC5721A7
:102CC000C4F20201884227DC1021C4F202018842CA
:102CD00000F0A8802821C4F20201884200F0A280FE
:102CE0004021C4F202019BE040F22741C4F20201FC
:102CF000884221DCA021C4F20201884200F09280C7
:102D0000B821C4F20201884200F08C8040F21041E8
:102D1000C4F2020184E000BF5821C4F202018842DB
:102D200000F080807021C4F2020188427AD08821AC
:102D3000C4F2020174E000BF40F22841C4F2020173
:102D400088426FD040F24041C4F20201884269D00B
:102D500040F25841C4F2020162E000BF6FF00E0081
:102D600031466AE6D4E9161202F01F02012303FA83
:102D700002F24A6040459DDD45F22F41C5F6020151
:102D8000884217DC40F2B741C4F20201884227DCD6
:102D900040F27041C4F20201884243D040F28841BF
:102DA000C4F2020188423DD040F2A041C4F20201C7
:102DB00036E000BF45F26B41C5F6020188421FDCD8
:102DC00045F23041C5F6020188422BD045F244411C
:102DD000C5F60201884225D045F258411EE000BFE9
:102DE00040F2B841C4F2020188421BD045F20841CA
:102DF000C5F60201884215D045F21C410EE000BF25
:102E000045F26C41C5F6020188420BD045F294416F
:102E1000C5F60201884205D045F28041C5F602019F
:102E200088420BD1616EA26EE06E4A6030B10168DB
:102E300021F480710160D4E91C014160012084F813
:102E400035000020002184F83410BDE8F081000036
:102E500080B5D8B190F83510022919D140F20F424F
:102E60000168C4F20202914216DC6F23C4F202032D
:102E7000994227DC3F23C4F2020399423EDC10232F
:102E8000C4F2020399425FD0282359E0012080BD9B
:102E900080214165012080BD40F26F43C4F20203EE
:102EA00099421BDC40F23F43C4F2020399422DDCFD
:102EB00040F21043C4F20203994245D040F2284345
:102EC0003EE000BF9F23C4F20203994228DC702336
:102ED000C4F20203994237D0882331E040F29F4385
:102EE000C4F20203994223DC40F27043C4F20203AD
:102EF000994229D040F2884322E000BF4023C4F227
:102F00000203994220D058231AE000BF40F2404308
:102F1000C4F20203994217D040F2584310E000BFB8
:102F2000A023C4F2020399420ED0B82308E000BFE8
:102F300040F2B843C4F20203994205D040F2A043E4
:102F4000C4F20203994275D191424FF0040280F815
:102F5000352011DC6F20C4F20200814222DC3F20C8
:102F6000C4F20200814239DC1020C4F20200814226
:102F700059D0282054E000BF40F26F40C4F2020054
:102F800081421BDC40F23F40C4F2020081422DDC52
:102F900040F21040C4F20200814244D040F2284086
:102FA0003EE000BF9F20C4F20200814228DC702076
:102FB000C4F20200814236D0882031E040F29F40C6
:102FC000C4F20200814223DC40F27040C4F20200ED
:102FD000814228D040F2884022E000BF4020C4F265
:102FE000020081421FD058201AE000BF40F240404A
:102FF000C4F20200814216D040F2584010E000BFF7
:10300000A020C4F2020081420DD0B82008E000BF29
:1030100040F2B840C4F20200814204D040F2A04025
:10302000C4F202008142086820F00100086000201C
:1030300080BD00BF0A6822F00E020A6045F25742C6
:10304000C5F6020291420A6822F001020A600FDC12
:1030500045F22F42C5F60202914219DC45F20842C0
:10306000C5F60202914229D045F21C4222E000BF7F
:1030700045F27F42C5F60202914213DC45F2584206
:10308000C5F60202914219D045F26C4212E000BF2F
:1030900045F23042C5F6020291420FD045F2444259
:1030A00008E000BF45F29442C5F60202914205D005
:1030B00045F28042C5F6020291421AD1D0E9181CAD
:1030C000D0E916E30A6822F480720A6003F01F0157
:1030D000012202FA01F1CEF80410816ECCF804103E
:1030E000C16E31B10A6822F480720A60D0E91C1204
:1030F0004A60012180F83510026D002180F83410FB
:103100000AB190470021084680BD00000000000081
:103110002DE9F04782B00021019140F208010446F8
:10312000C2F2004148F2B512C1F64E32A56D0968EF
:1031300040F26F490068C4F20209A1FB0218484539
:103140002E68296816DC9F21C4F2020188422DDC1A
:103150005721C4F20201884252DC1021C4F202015C
:1031600088427BD02821C4F20201884276D04021D7
:1031700070E000BF45F22F42C5F60202904229DC02
:1031800040F2B742C4F20202904245DC40F2704184
:10319000C4F20201884261D040F28841C4F20201C7
:1031A00088425BD040F2A04154E000BF40F227418A
:1031B000C4F2020188423FDCA021C4F2020188422D
:1031C0004CD0B821C4F20201884247D040F21041ED
:1031D00040E000BF45F26B42C5F60202904275DC4A
:1031E00045F23042C5F60202904200F0818045F27D
:1031F0004442C5F6020290427AD045F2584273E04A
:103200005821C4F20201884228D07021C4F2020180
:10321000884223D088211DE040F2B842C4F2020265
:1032200090421BD045F20842C5F6020290425FD0A0
:1032300045F21C4258E000BF40F22841C4F20201AE
:1032400088420BD040F24041C4F20201884205D0CE
:1032500040F25841C4F20201884261D1E16D082276
:1032600001F01F0140F20F4A8A40C4F2020A3242C2
:1032700000F0E98050454FF0040313DC6F27C4F2DF
:103280000207B8426CDC3F27C4F20207B84200F3E1
:10329000A7801027C4F20207B84200F0C880282790
:1032A000C0E000BF484567DC40F23F47C4F2020778
:1032B000B84200F39D8040F21047C4F20207B842C2
:1032C00000F0B58040F22847ACE000BF45F26C4208
:1032D000C5F6020290420BD045F28042C5F60202CA
:1032E000904205D045F29442C5F60202904217D1B1
:1032F0000268E36D570703F01F0315D504279F40AD
:1033000017EA010610D011046F6045D4910603D46A
:10331000016821F004010160216C002940F0F6826F
:1033200002B0BDE8F08700BF97073DD502279F4058
:1033300017EA010638D011046F6000F1ED829106A2
:1033400009D4016821F00A010160012084F83500E8
:10335000002084F83400E16B002940F0D782DFE7D9
:103360009F27C4F20207B8424CDC7027C4F2020760
:10337000B8425CD0882755E040F29F47C4F202076C
:10338000B84247DC40F27047C4F20207B8424ED060
:1033900040F2884746E000BFD00300F1C382A16C31
:1033A000002940F0B382BBE71207B9D508229A4042
:1033B0001140B5D0016821F00E010160012000FA32
:1033C00003F16960606584F835000020E16C84F8E1
:1033D00034000029A4D02046884702B0BDE8F08719
:1033E0004027C4F20207B84221D058271AE000BF94
:1033F00040F24047C4F20207B84218D040F25847A2
:1034000010E000BFA027C4F20207B8420FD0B827CF
:1034100008E000BF40F2A047C4F20207B84206D05D
:1034200040F2B847C4F20207B84218BF0823076841
:103430001F4208D0036823F004030360AA60626D92
:1034400042F00102626501228A4032426FD050454B
:1034500010DC6F23C4F2020398421DDC3F23C4F248
:103460000203984234DC1023C4F20203984256D07F
:1034700028234FE048451BDC40F23F43C4F20203DF
:1034800098422DDC40F21043C4F20203984246D029
:1034900040F228433EE000BF9F23C4F2020398425B
:1034A00028DC7023C4F20203984238D0882331E02C
:1034B00040F29F43C4F20203984223DC40F270437F
:1034C000C4F2020398422AD040F2884322E000BFAF
:1034D0004023C4F20203984221D058231AE000BFCF
:1034E00040F24043C4F20203984218D040F25843DD
:1034F00010E000BFA023C4F2020398420FD0B8230B
:1035000008E000BF40F2A043C4F20203984206D094
:1035100040F2B843C4F20203984240F00B82436980
:103520001B0604D5AA60626D42F0020262650422A5
:103530008A4032426FD0504510DC6F23C4F2020340
:1035400098421DDC3F23C4F20203984234DC10236E
:10355000C4F20203984256D028234FE048451BDCB2
:1035600040F23F43C4F2020398422DDC40F2104384
:10357000C4F20203984246D040F228433EE000BF26
:103580009F23C4F20203984228DC7023C4F2020392
:10359000984238D0882331E040F29F43C4F20203BE
:1035A000984223DC40F27043C4F2020398422AD0CE
:1035B00040F2884322E000BF4023C4F20203984255
:1035C00021D058231AE000BF40F24043C4F2020366
:1035D000984218D040F2584310E000BFA023C4F234
:1035E000020398420FD0B82308E000BF40F2A04386
:1035F000C4F20203984206D040F2B843C4F2020378
:10360000984240F09F8103689B0704D5AA60626DD1
:1036100042F004026265102202FA01F1314200F028
:10362000818050454FF0080210DC6F23C4F2020382
:1036300098421DDC3F23C4F20203984234DC10237D
:10364000C4F20203984256D028234FE048451BDCC1
:1036500040F23F43C4F2020398422DDC40F2104393
:10366000C4F20203984246D040F228433EE000BF35
:103670009F23C4F20203984228DC7023C4F20203A1
:10368000984238D0882331E040F29F43C4F20203CD
:10369000984223DC40F27043C4F2020398422AD0DD
:1036A00040F2884322E000BF4023C4F20203984264
:1036B00021D058231AE000BF40F24043C4F2020375
:1036C000984218D040F2584310E000BFA023C4F243
:1036D000020398420FD0B82308E000BF40F2A04395
:1036E000C4F20203984206D040F2B843C4F2020387
:1036F000984218BF04220368134213D0A9600168DE
:103700004903016808D4C90508D4016821F00801FB
:103710000160216C21B905E008034FD4216C09B187
:1037200020468847E06D00F01F01202000FA01F2DA
:10373000324200F0AB8020681023504510DC6F2728
:10374000C4F20207B8421DDC3F27C4F20207B842A8
:1037500038DC1027C4F20207B8425AD0282753E0B9
:1037600048451BDC40F23F47C4F20207B84231DC57
:1037700040F21047C4F20207B8424AD040F228474C
:1037800042E000BF9F27C4F20207B8422CDC70273A
:10379000C4F20207B8423CD0882735E040F29F4788
:1037A000C4F20207B84227DC40F27047C4F20207B5
:1037B000B8422ED040F2884726E000BFA16C002915
:1037C000AED1AFE74027C4F20207B84221D0582754
:1037D0001AE000BF40F24047C4F20207B84218D0D6
:1037E00040F2584710E000BFA027C4F20207B842D9
:1037F0000FD0B82708E000BF40F2A047C4F202078C
:10380000B84206D040F2B847C4F20207B84218BF27
:10381000022307681F4239D0AA6094F83520042A91
:1038200002681BD122F016020260426922F0800277
:103830004261226C0AB9A26C1AB1026822F0080235
:1038400002603F208840A860012084F83500216D87
:103850000020002984F8340058D161E55103016843
:103860000CD4C9050ED4016821F0100101600120BB
:1038700084F83500002084F8340003E0080301D404
:10388000616C00E0E16B09B120468847606D00285B
:103890003FF446AD606DC00734D0042084F8350095
:1038A00020684FEA9821026822F001020260019A22
:1038B000013201928A421AD80268D20717D0019ABF
:1038C000013201928A4212D80268D2070FD0019ABF
:1038D000013201928A420AD80268D20707D0019ABF
:1038E000013201928A4202D80268D207DFD1006811
:1038F000C0074FF0030008BF012084F83500002006
:1039000084F83400E16C00293FF40AAD2046884772
:1039100002B0BDE8F08700BFD00307D4616C002976
:10392000F4D1FDE4216C0029F0D1F9E4E16B002928
:10393000ECD1F5E4026804228A4032427FF4FBAD08
:1039400069E600BF026866E62DE9F04381B00446EF
:1039500001F016FC002C00F0128140F26F48054681
:103960002068C4F20208404516DC9F21C4F202011F
:1039700088422DDC5721C4F20201884254DC102118
:10398000C4F20201884200F07E802821C4F20201C4
:10399000884278D0402171E045F22F41C5F60201FE
:1039A000884229DC40F2B741C4F20201884247DC78
:1039B00040F27041C4F20201884264D040F2884172
:1039C000C4F2020188425ED040F2A04156E000BF3E
:1039D00040F22741C4F20201884241DCA021C4F236
:1039E000020188424FD0B821C4F2020188424AD075
:1039F00040F2104142E000BF45F26B41C5F60201C2
:103A0000884200F3C18045F23041C5F60201884288
:103A100000F0CD8045F24441C5F60201884200F035
:103A2000C68045F25841BDE05821C4F202018842E7
:103A300029D07021C4F20201884224D088211DE0DF
:103A400040F2B841C4F2020188421CD045F208415C
:103A5000C5F60201884200F0AA8045F21C41A1E0AF
:103A600040F22841C4F2020188420CD040F24041A9
:103A7000C4F20201884206D040F25841C4F2020169
:103A8000884240F09782022184F83510002184F8A2
:103A90003410016821F0010101600168C90708D0F4
:103AA00001F06EFB401B052864D820680168C90737
:103AB000F6D148F23F0204F108060168CFF6106221
:103AC0001140D4F818C06CCE1143D4F82490194397
:103AD000E3692943256A0E43B9F1040F46EA0C064F
:103AE00043EA060343EA050303D1D4E90B653343F4
:103AF0002B43666843F48011A6F13F07A6F1290520
:103B0000042FA6F1470238BF0B46062DA6F14F0E33
:103B100038BF0B46022A26F0030238BF0B46BEF11F
:103B2000040F38BF0B46742A08BF0B46B9F1040FC7
:103B30000360416921F0070141EA090140F0F48086
:103B4000D4E90A53002B41EA050100F0ED80BCF5F1
:103B5000005F00F0CF80BCF1000F40F0D780022D55
:103B600000F0D780012D00F0CB80002D00F0D18037
:103B7000DAE000BF20206065032084F835000120D2
:103B800001B0BDE8F08300BF45F26C41C5F602010B
:103B900088420CD045F28041C5F60201884206D029
:103BA00045F29441C5F60201884240F003820221A9
:103BB00084F83510002184F834100168A268A2F15D
:103BC0008003E768B3FA83F3402A4FEA53134FEABE
:103BD00083336FF3101108BF1023226941EAD70124
:103BE00067691943A36941EAD201E26941EAD70151
:103BF00041EAD3014CF6CD4341EAD2014AF6F8320C
:103C0000CAF2FD72276A0244CCF6CC43A2FB03231E
:103C100041EA171101606FF0030000EA9300E065CC
:103C20002046FDF755FBE16D012201F01F0102FA6C
:103C300001F141602068404540F3858045F22F4105
:103C4000C5F60201884217DC40F2B741C4F2020116
:103C5000884229DC40F27041C4F20201884200F03F
:103C6000BC8040F28841C4F20201884200F0B58075
:103C700040F2A041ACE000BF45F26B41C5F6020145
:103C8000884223DC45F23041C5F60201884200F04B
:103C9000A48045F24441C5F60201884200F09D80AF
:103CA00045F2584122E000BF40F2B841C4F202019F
:103CB000884200F0928045F20841C5F60201884230
:103CC00000F08B8045F21C4110E000BF45F26C41D2
:103CD000C5F60201884200F0808045F29441C5F6A5
:103CE0000201884200F0798045F28041C5F6020168
:103CF00070E000BF032D17D8DFE805F00E0B0E02B1
:103D0000A3F1C072B2FA82F2520904E0032D03D388
:103D10000AD1C3F300623AB140206065012084F803
:103D2000350001B0BDE8F08341612046FDF7D0FACF
:103D3000E16D3F2201F01F0102FA01F1816020686C
:103D400040453FF77BAF9F21C4F20201884211DC5E
:103D50005721C4F20201884220DC1021C4F2020182
:103D600088423AD02821C4F20201884235D040214D
:103D70002EE000BF40F22741C4F20201884219DC64
:103D8000A021C4F20201884227D0B821C4F2020166
:103D9000884222D040F210411AE000BF5821C4F2FC
:103DA0000201884219D07021C4F20201884214D065
:103DB00088210DE040F22841C4F2020188420CD073
:103DC00040F24041C4F20201884206D040F258411C
:103DD000C4F20201884240F0E58045F2574C45F6B6
:103DE000FC0EC5F6020CC5F6020E604512DC45F26B
:103DF0002F41C5F60201884220DC45F20841C5F694
:103E00000201884234D045F21C41C5F602018842C5
:103E10002ED085E045F27F41C5F6020188421BDCC9
:103E200045F25841C5F60201884221D045F26C4165
:103E3000C5F6020188421BD072E000BF45F2304156
:103E4000C5F60201884213D045F24441C5F602018D
:103E500088420DD064E000BF45F29441C5F60201EE
:103E6000884205D045F28041C5F60201884257D10B
:103E70006FF007014CF6CD4251FA80F1CCF6CC42FE
:103E8000A1FB0212AEF1FC05AEF17C061309A2689B
:103E900003F01F01802A4FF0010205EB8305256620
:103EA00002FA01F26666A26602D10021616000E0BA
:103EB0006168CBB2013907292B60726016D85E1E8B
:103EC000082E19D260450EF1440219DC45F22F414B
:103ED000C5F60201884245DC45F20841C5F60201FB
:103EE000884255D045F21C414EE000BF002060677B
:103EF000C4E91B0056E000BFD4E91B02616F4EE02D
:103F000045F27F41C5F60201884235DC45F2584151
:103F1000C5F6020188423BD045F26C4134E000BF57
:103F20006FF00F014AF6AB2251FA80F1CAF6AA22CD
:103F3000A1FB021240F20F43C4F20203082511094B
:103F4000984203F1AA060B4688BF05EB121340F610
:103F50000005B042C4F2020505F1800628BF0B46F9
:103F600095E700BF45F23041C5F6020188420FD007
:103F700045F2444108E000BF45F28041C5F6020128
:103F8000884205D045F29441C5F60201884213D11A
:103F900001210EEB8300B140E066226761670023D8
:103FA0000360516000206065012184F8351001B084
:103FB000BDE8F0834020DEE540F60000C4F20200D8
:103FC00000F1FC0E00F5A072E2E700000000000026
:103FD000B0B500283CD0054690F83400012801D146
:103FE0000220B0BD012085F8340095F83500012885
:103FF00028D1022085F8350000206865286804680B
:1040000024F0010404602846FDF7FAF940F20F425B
:104010002868C4F2020240F26F419042C4F20201E9
:1040200018DC6F23C4F20203984225DC3F23C4F25C
:10403000020398423CDC1023C4F2020398425ED093
:10404000282357E04FF400606865002085F83400AD
:104050000120B0BD88421BDC40F23F43C4F20203A2
:1040600098422DDC40F21043C4F20203984246D03D
:1040700040F228433EE000BF9F23C4F2020398426F
:1040800028DC7023C4F20203984238D0882331E040
:1040900040F29F43C4F20203984223DC40F2704393
:1040A000C4F2020398422AD040F2884322E000BFC3
:1040B0004023C4F20203984221D058231AE000BFE3
:1040C00040F24043C4F20203984218D040F25843F1
:1040D00010E000BFA023C4F2020398420FD0B8231F
:1040E00008E000BF40F2B843C4F20203984206D091
:1040F00040F2A043C4F20203984240F02F810368CB
:104100000B2464F3440303602B6C1BB1036843F07E
:1041100008030360884219DC9F23C4F2020398421B
:1041200032DC5723C4F20203984259DC1023C4F254
:104130000203984200F096802823C4F202039842BA
:1041400000F090804023C4F2020389E045F22F433F
:10415000C5F6020398422DDC40F2B743C4F20203D5
:1041600098424BDC40F27043C4F20203984279D08B
:1041700040F28843C4F20203984273D040F2A04355
:10418000C4F202036CE000BF40F22743C4F2020312
:10419000984243DCA023C4F20203984262D0B823C1
:1041A000C4F2020398425DD040F21043C4F202030D
:1041B00056E000BF45F26B43C5F6020398423FDC70
:1041C00045F23043C5F6020398424BD045F24443D2
:1041D000C5F60203984245D045F258433EE000BF81
:1041E0005823C4F2020398423CD07023C4F2020365
:1041F000984237D08823C4F2020331E040F2B8433A
:10420000C4F2020398422DD045F20843C5F60203DA
:10421000984227D045F21C4320E000BF40F22843DB
:10422000C4F2020398421DD040F24043C4F202039C
:10423000984217D040F25843C4F2020310E000BF86
:1042400045F26C43C5F6020398420BD045F2944305
:10425000C5F60203984205D045F28043C5F6020335
:10426000984274D12B6E1C68E40303D51C6844F497
:1042700080741C60EB6E1BB11D6845F480751D6079
:10428000904211DC6F21C4F2020188421EDC3F2102
:10429000C4F20201884235DC1021C4F202018842D6
:1042A00055D0282150E000BF88421BDC40F23F413E
:1042B000C4F2020188422DDC40F21041C4F2020136
:1042C000884244D040F228413EE000BF9F21C4F222
:1042D0000201884228DC7021C4F20201884236D0F3
:1042E000882131E040F29F41C4F20201884223DC80
:1042F00040F27041C4F20201884228D040F2884165
:1043000022E000BF4021C4F2020188421FD05821A0
:104310001AE000BF40F24041C4F20201884216D0C8
:1043200040F2584110E000BFA021C4F202018842CF
:104330000DD0B82108E000BF40F2B841C4F202013C
:10434000884204D040F2A041C4F2020188420168D0
:1043500041F0010101600020B0BD00BF03680524E9
:1043600064F3430303602B6C002B3FF4D3AE03686C
:1043700043F00403CDE60000B0B5044600F000FFB2
:1043800040F200010546C2F20041621C097818BFE4
:104390000C4400BF00F0F4FE401BA042FAD3B0BDB5
:1043A000704700000000000010B34AF200010068EE
:1043B000C4F2000188420FD04DF20041C4F2000166
:1043C00088420BD04AF20041C4F20001884218BF73
:1043D0007047012003E000BF002000E0022040F60B
:1043E0006861C2F2004101EB4010C06A00B10047B1
:1043F000704700000000000070470000000000004F
:1044000070470000000000002DE9F04F87B004461F
:104410004AF61000C4F2000001684AF61400C4F223
:1044200000000268206802EA010A056DD0F8549085
:10443000076DD0F85480036D0293436D0193036DB3
:104440000693436D0593036D0493436D0393436D8E
:10445000066D06EA030B5FEACB530BD54FF4807170
:1044600001654AF610010020C4F2000108602046F0
:10447000FFF7C6FF05EA09064AF610095FEA4B5046
:10448000C4F200094FEA8A750ED52068D0F8DC1016
:10449000D0F8E42011404FF4806202650020C9F892
:1044A0000000204600F08CFC08EA070806F470467D
:1044B00055B12068002101650AF00300C9F8000029
:1044C00020462946FFF76CFFDDE9011000EA0107ED
:1044D00008F00F0546B12068314606650020C9F88E
:1044E0000000204600F0BCFC07F0F00645B1206853
:1044F000294605650020C9F80000204600F0F8FBB9
:1045000046B12068314606650020C9F80000204603
:1045100000F016FC5FEA0B5000F1B6805FEA8B50AA
:1045200000F1C0805FEA0B3000F1CF805FEACB3052
:1045300000F1D9805FEA4B30DDE9031000EA0105A4
:1045400009D520684FF4802101650020C9F80000DA
:10455000204600F02DFC5FEA8B30DDE9051000EA13
:10456000010005F060710CD522684FF4003313652B
:104570000022C9F80020D4F89C2042F08002C4F840
:104580009C2000F0715539B1206801650020C9F800
:1045900000002046FFF730FF206845B10565002187
:1045A000C9F80010D4F89C102943C4F89C10A9F550
:1045B000016188425ED16068816889075AD0016ACA
:1045C000426A036A476A114003EA070202F03005B3
:1045D000D0F82080D0F82490026A049211F00F01E4
:1045E000D0F824B0026A0692426A0592466AD0F870
:1045F00020A003D00162204600F0CEFB08EA0907A4
:104600002DB1606829460562204600F0CDFB06EA20
:104610000A0007F4C0754006049800EA0B060AD5A4
:1046200060684023C16BC26B090C02F03F02036259
:10463000204600F0B5FBDDE9051000EA010706F4AD
:10464000FC462DB1606829460562204600F0A0FBBB
:1046500007F4F02036B161680E62D4F89C10314343
:10466000C4F89C1030B161680862D4F89C1008430B
:10467000C4F89C00D4F89C00002847D0204607B01E
:10468000BDE8F04FFFF790BE20684FF40061016570
:104690000020C9F80000204600F00AFC5FEA8B50B9
:1046A0007FF540AF2068D0F8D810D0F8E020114056
:1046B0004FF4007202650020C9F80000204600F0A7
:1046C000A7FB5FEA0B307FF531AF20684FF4002184
:1046D00001650020C9F80000204600F005FB5FEAF4
:1046E000CB307FF527AF20684FF480310165002083
:1046F000C9F80000204600F05FFB5FEA4B30DDE9BF
:10470000031000EA01053FF51CAF24E707B0BDE840
:10471000F08F0000000000002DE9F04F85B0A8B335
:104720004AF200080446C4F200080068404531D04F
:1047300094F89810A9B3816921F01001816100F00B
:104740001FFD054620688169090705D500F018FDA1
:10475000401B0B28F6D310E0816941F00101816113
:1047600000F00EFD054600BF20688169C90721D110
:1047700000F006FD401B0B28F6D3D4F89C0040F057
:104780000100C4F89C00032084F89800012005B0C3
:10479000BDE8F08F08F58071616094F898100029E9
:1047A000C9D1002084F89900204600F0B9F92068AA
:1047B000C1E700BF816941F002018161217C82690A
:1047C00022F04002012918BF40328261617C826977
:1047D00022F48042012908BF02F580428261A17C57
:1047E000826922F48052012918BF02F58052826149
:1047F000816921F44073D4E902120B438361836918
:1048000023F0A4038361036923F010030361AAB1B9
:10481000022A0FD0012A03D1826942F004020CE07F
:104820008369032A43F080038361036943F0100224
:10483000026103D1826942F020028261D4E90572EB
:10484000E369561E6FF0FF02256A02EB0323B1F500
:10485000407F43EA4663A5F1010646EA030640F2BB
:104860000003CFF6FF7303EB074746EA0701C16178
:1048700010D1D4E90B65D4E90917013F02EB0622F8
:104880006FF00F063A4306EB05173A4303EB01417D
:104890001143C160236E2BB1616ED0F8C02011436B
:1048A000C0F8C010E16DCDE90313D94240F2F02108
:1048B000C0F6010109D0D0F8C820A36E22F007028B
:1048C00051F823301A43C0F8C820D4F840A0BAF1F8
:1048D000000F09D0D0F8BC20636C22F0070251F819
:1048E00023301A43C0F8BC20A76C57B1D0F8BC20C5
:1048F000E36C22F0700251F8233042EA0312C0F850
:10490000BC20D4F850C0BCF1000F0AD0D0F8BC20B5
:10491000636D22F4E06251F8231042EA0121C0F8ED
:10492000BC10404504D161688A6822F003028A60A5
:104930000021C4F89410C4F89C10012184F8981048
:104940004FF6FC72D0F88410D4F83C9021EA0203B0
:10495000656CD4E90D120292019543EA8103C0F817
:104960008430D0F8843023F47F0343EA0243C0F854
:1049700084305318D0F888606FF38F0646EA8306B8
:10498000C0F88860D0F8886003EB490326F4FE067F
:1049900046EA0946C0F88860D0F8A0606FF38F0639
:1049A00046EA8306C0F8A060D0F8A06005FB0A3391
:1049B00026F4FE0646EA0A46C0F8A060D0F8B060C9
:1049C0006FF38F0646EA8306C0F8B060D0F8B06097
:1049D00026F4FE0646EA0746C0F8B060E66CD0F85A
:1049E000AC506FF38F0506FB07337E4345EA830522
:1049F000C0F8AC50D4F8548008FB0C35D0F8F03037
:104A00006FF38F0308FB0CFC43EA8503C0F8F0301A
:104A1000D0F8F0E0A36D2EF47C1242EA0342C0F815
:104A2000F02005EB4302D0F8C0506FF38F0545EA44
:104A30008202C0F8C020D0F8C020DDF80CB022F40B
:104A40007C1242EA0B42C0F8C020019AD0F8C05054
:104A500025F07C5502FB0AFE4AF20002C4F2000275
:104A6000DDF810A002EB8101029A01F5406145EAF0
:104A70000A6501EB8207C0F8C05007EBC902A56EBA
:104A800002EB8E00626700EB86060BFB05F22767E0
:104A900006EB8C07C4E91E060AFB05F007EBC3030F
:104AA00003EB8202C4F884304DF2FC33E16602EB82
:104AB0008000C4F200039842C4F88070C4F88820D3
:104AC000C4F8900004D9D4F89C0040F0200058E6C7
:104AD000814221D20A46002042F8040BD4F89030DB
:104AE0009A4215D2486001F10802D4F890309A42F7
:104AF0003FBF0020886001F10C02D4F8903038BF2D
:104B00009A4205D2C8601031D4F890209142E1D386
:104B100005B0BDE8F08F00BF002005B0BDE8F08F04
:104B2000B0B5B6B0044602A8B8210025CDE9345589
:104B3000CDE932553195FCF7D6F84DF200412068A9
:104B4000C4F20001884241D04AF20041C4F200019F
:104B5000884273D04AF20001C4F20001884240F05A
:104B6000BF80002003904FF4004002904FF080502F
:104B70001D9002A801F074FE08B1FCF731FF40F669
:104B8000707144F2E040C2F20041C5F602000A68CA
:104B9000002A02F101020A6008D1C16841F4807163
:104BA000C160C16801F48071019101990168152407
:104BB00041F0080101600068132500F00800019031
:104BC000019803203190092133E000BF4FF40040E9
:104BD00002904FF080501D9002A8039501F040FE16
:104BE00008B1FCF7FDFE40F6707144F2E040C2F2FD
:104BF0000041C5F602000A68002A02F101020A60BB
:104C000008D1C16841F48071C160C16801F480714C
:104C1000019101990168A02441F008010160006838
:104C20009F2500F008000190052101984FF44050A5
:104C3000319040F60040C5F6020038E000200390B5
:104C40004FF4004002904FF080501D9002A801F0F8
:104C500007FE08B1FCF7C4FE40F6707144F2E04074
:104C6000C2F20041C5F602000A68002A02F1010200
:104C70000A6008D1C16841F48071C160C16801F463
:104C80008071019101990168162441F002010160CF
:104C90000068142500F00200019001986020319016
:104CA00040F60040C5F602000921A0F500603591EC
:104CB00031A9022232920022CDE9332200F064F9B8
:104CC00005210022284600F01FFB284600F00CFBBF
:104CD00005210022204600F017FB204600F004FBCF
:104CE00036B0B0BD000000007047000000000000BA
:104CF00010B34AF200010068C4F2000188420FD0EC
:104D00004DF20041C4F2000188420BD04AF200414A
:104D1000C4F20001884218BF7047012003E000BFC1
:104D2000002000E0022040F66861C2F2004101EB81
:104D30004010C06900B1004770470000000000004B
:104D400010B34AF200010068C4F2000188420FD09B
:104D50004DF20041C4F2000188420BD04AF20041FA
:104D6000C4F20001884218BF7047012003E000BF71
:104D7000002000E0022040F66861C2F2004101EB31
:104D80004010406A00B1004770470000000000007A
:104D900070470000000000007047000000000000A5
:104DA0007047000000000000704700000000000095
:104DB0007047000000000000704700000000000085
:104DC00010B34AF200010068C4F2000188420FD01B
:104DD0004DF20041C4F2000188420BD04AF200417A
:104DE000C4F20001884218BF7047012003E000BFF1
:104DF000002000E0022040F66861C2F2004101EBB1
:104E00004010806900B100477047000000000000BA
:104E100010B34AF200010068C4F2000188420FD0CA
:104E20004DF20041C4F2000188420BD04AF2004129
:104E3000C4F20001884218BF7047012003E000BFA0
:104E4000002000E0022040F66861C2F2004101EB60
:104E50004010406900B100477047000000000000AA
:104E600010B34AF200010068C4F2000188420FD07A
:104E70004DF20041C4F2000188420BD04AF20041D9
:104E8000C4F20001884218BF7047012003E000BF50
:104E9000002000E0022040F66861C2F2004101EB10
:104EA0004010006900B1004770470000000000009A
:104EB0007047000000000000B0B540F630750446B1
:104EC000C007C2F2004502D0286800B18047A007A1
:104ED00002D5686800B18047600702D5A86800B1B4
:104EE0008047200702D5E86800B18047E00602D578
:104EF000286900B18047A00602D5686900B18047E3
:104F0000600602D5A86900B18047200602D5E8698D
:104F100000B18047E00502D5286A00B18047A005AE
:104F200002D5686A00B18047600502D5A86A00B161
:104F30008047200502D5E86A00B18047E00402D529
:104F4000286B00B18047A00402D5686B00B1804790
:104F5000600402D5A86B00B18047200406D5E86B39
:104F6000002808BFB0BDBDE8B0400047B0BD00009C
:104F70008821C5F600010A68024208BF7047086030
:104F8000FFF79ABF000000002DE9F04F85B00D68D3
:104F90000290002D00F0E68002988E4600F1264235
:104FA0000A2102F1FF7342F20042C5F60202002418
:104FB00090424FEAB32208BF0921082A4FF00107A7
:104FC00038BF4FEAB32100264FF000080091CDF81A
:104FD0000CE00DE0DEF8005008F1010835FA07F0AA
:104FE00006F1020607F1010704F1040400F0BA809B
:104FF000A7F1010A012000FA0AF315EA0309E9D032
:10500000DEF804B00BF003056A1E012A22D80298CC
:105010004FEA4801D0F808C00191032101FA06F2D5
:1050200003992CEA020CD1F80CE00EFA06F1DDF837
:105030000CE041EA0C01816041686FEA020CCBF39D
:10504000001299430346019802FA0AF2114359608B
:105050000CE000BF0320032D00FA06F0029B6FEA6C
:10506000000C304602D13046032526E0D968DEF830
:10507000082001EA0C018240022D41EA0201D960B8
:105080001BD102466FF0030000EA5A010F201944B9
:1050900004F01C0300FA03F51046D1F820E0039A4F
:1050A0002EEA0505DDF80CE012699A40029B2A43BE
:1050B0000A62DEF804B00BF00305196805FA00F087
:1050C00001EA0C011BF4403F40EA010018603FF484
:1050D00081AF44F2F44140F20845C5F60201C5F63D
:1050E00000050F23086840F002000860086800F01F
:1050F000020004902AF00300049904F00C014259C4
:105100008B409A43009B03FA01F1114341514FF048
:10511000B0452868DEF8041040EA0902CB0258BF07
:1051200020EA09028B022A6040F20405C5F6000558
:10513000286840EA090258BF20EA09028B032A6066
:10514000D5F8800040EA090258BF20EA0902C903E5
:10515000C5F88020E86F40EA090258BF20EA09023A
:10516000EA6737E705B0BDE8F08F000000000000F7
:10517000002A08BF09048161704700000000000098
:1051800042F2B870C2F201400068704700000000AF
:1051900040F2000042F2B871C2F20040C2F2014196
:1051A00000780A68104408607047000000000000A2
:1051B00080B5032000F0D8F802F092FA44F21841CA
:1051C00040F23C33C5F60201C0F601030A680968E3
:1051D00001F00F01C2F30322595C9A5C01F01F0138
:1051E00002F01F02D04040F20C02C2F2004220FA4C
:1051F00001F1116040F20801C2F2004108600F2085
:1052000000F00AF800281CBF012080BD00F054F80F
:10521000002080BD00000000B0B58AB00F283ED845
:105220000446A12000222146002500F06DF8A120AF
:1052300000F05AF840F20400C2F20040046044F268
:10524000EC40C5F60200016841F080710160006821
:1052500001A900F080700290029802A802F08CF977
:1052600002F00EFA4DF683614000C4F21B314EF29B
:105270000002A0FB010141F67C50C2F200404FF059
:10528000FF33C4F20002026003EB9141C0E9011553
:1052900040F2E731C0E9031503F01AFA10B101201A
:1052A0000AB0B0BD41F67C50C2F2004003F044FAAF
:1052B0000AB0B0BD0000000081B044F2F44000220A
:1052C000C5F60200016841F00201016000680F218B
:1052D00000F0020000906FF00100009B01B000F0B0
:1052E00013B8000000000000002848BF704700F01D
:1052F0001F01012202FA01F14EF200124009CEF222
:10530000000242F82010704770B54EF60C5C4FF06A
:10531000FF36CEF2000C00F16045DCF80030C3F33C
:10532000022E8EF00703042B28BF0423BEF10304D2
:1053300006FA03F321EA030100F00F0338BF00244B
:10534000043BB0F1FF3F634406FA04F003F10C03A1
:1053500001FA04F1C8BF05F5644322EA00000843DE
:105360000001187070BD00004EF60C514FF6FF039F
:10537000CEF200010A681A4060F30A2242F080600F
:1053800040F0FD70086070472DE9F04F8EB04BF291
:1053900004430022C5F200230492CDE902220592C3
:1053A00045F200090692C5F20029D0F800E01A681B
:1053B000BEEB090C02F0030018BF4FF0010C0128EE
:1053C00076D10120029002F03000102875D002F44E
:1053D0004070B0F5807F01D10120049002F4A0203C
:1053E00040F20108B0F5803FC0F200186ED1900382
:1053F000404658BF4FF00110059002F0A060B0F198
:10540000807F68D05A6802F0030001286ED1022024
:10541000029002F0300010286CD002F44070B0F519
:10542000807F01D10220049002F4A020B0F5803FDB
:1054300040F20200C0F2010005D19503054648BFC5
:1054400008F10105059502F0A065B5F1807F05D151
:105450009201024648BF08F10102069200250C9510
:10546000CDE90A55CDE9085553F8042C1E68D2073A
:105470004FF4007204BF40F22222C0F20442F70748
:1054800005D086EA0207BF073CD401250895F70638
:105490003BD586EA0207BF0637D44FF0010BCDF8A3
:1054A00024B006F44077B7F5407F37D134E000BF31
:1054B00002F0300010287FF48AAF0120039002F43C
:1054C0004070B0F5807F3FF487AF87E702F0A060BF
:1054D000B0F1807F96D19001404658BF4FF0011047
:1054E00006905A6802F00300012890D002F03000C4
:1054F000102892D10220039002F44070B0F5807F12
:1055000090D091E70025F706C3D44FF0000B06F4C6
:105510004077B7F5407F01D101270A97F7030DD5F2
:1055200086EA02077F0309D4B70319D44FF0011AA2
:10553000CDF82CA0F70118D504E000BF4FF0000A09
:10554000F70112D586EA02077F010ED4B70141D4D4
:105550004FF001140C945F68FE070AD10FE000BF02
:10556000CDF82C80C246F701ECD400245F68FE071A
:1055700005D087EA0206B60701D402250895FE0683
:1055800007D587EA0206B60603D44FF0020BCDF822
:1055900024B007F44076B6F5407F01D102260A9682
:1055A000FE0307D587EA0206760303D4BE0319D4A7
:1055B00082460B90FE011BD57A40520118D4BA01E5
:1055C0001ED404460C90D9F80000C007AEEB0900C9
:1055D00014D01EE0CDF8308044465F68FE07CED080
:1055E000C7E700BF08F1010ACDF82CA0FE01E3D403
:1055F000D9F80000C007AEEB09000AD100220FE085
:1056000008F101040C94D9F80000C007AEEB0900C2
:10561000F4D0D9F8002022F00102C9F800200122BC
:105620004AF200060192B0FA80F7C5F20026D04691
:10563000CA463268CDF800E0D207A646484606D0F2
:10564000306820F0010030600198023001900CEBCE
:105650004C000DF108097F0909EBC006B26803EBA5
:10566000820252F804CC2CF4807442F8044C53F8B3
:10567000042CD2072AD159F8300000285BD003EB64
:10568000800050F8042C22F0010240F8042C7068CD
:1056900038B103EB800050F8042C22F0100240F8DF
:1056A000042CF06840B1012222EA000053F82020C7
:1056B00022F4803243F820203069E0B3012222EA4C
:1056C000000053F8202022F0807232E053F8040CDE
:1056D000009A524520F0010043F8040C2BD103EB53
:1056E0008500BBF1000F50F8042C42F0020240F894
:1056F000042C07D003EB8B0050F8042C42F020025E
:1057000040F8042CB8F1000F08D0012020EA08006E
:1057100053F8202042F4802243F82020BEF1000FED
:1057200009D00120724620EA0E0053F8202042F0F2
:10573000806243F8202007EB4705086859F8356078
:1057400009EBC502B04215D148685768B842DDF888
:1057500000E034D1CF68D468A7422FD10F69126915
:10576000974207462BD153F8040C40F0010043F850
:10577000040C57E088689768B84203D15768DDF891
:1057800000E01CE04868576860B1B8420AD103EBFA
:10579000860252F8047C27F0010742F8047CDDF809
:1057A00000E016E0C868D468A042DDF800E006D04A
:1057B00008691269904202D034E000BF074603EB4B
:1057C000860050F8042C22F0010240F8042C3846E0
:1057D0003FB103EB800050F8042C22F0100240F897
:1057E000042C09EBC500826803EB820252F8047CAA
:1057F00027F4807742F8047CC26842B1012727EA87
:10580000020253F8227027F4803743F822700069AF
:1058100040B1012222EA000053F8202022F08072D9
:1058200043F8202088684FF44072D64503EB80008F
:1058300050F8047C08BF4FF4807227F440773A4454
:1058400040F8042C486953F8042C471EC2F3074261
:1058500097420BD9002753F8042CCFF6FF7722F498
:105860007F0207EB0040104343F8040C53F8042C6C
:10587000086801384AF20005D207C5F2002553F83E
:10588000207027F003022BD10327D64508BF01273C
:105890003A4343F82020486860B103EB800030228F
:1058A000D64550F8047C08BF102227F020073A4361
:1058B00040F8042CC868C2032AD4019ED0B3012248
:1058C000D64522EA000053F8202003EB80044FF075
:1058D000A06022F0E06208BF4FF0807028E000BFB7
:1058E00042F0010243F82020486840B103EB8000F9
:1058F000012750F8042C67F3051240F8042CC868FF
:10590000C20329D4A8B34FF080726FF0E06727E09C
:105910000122D64522EA000003EB800453F8202040
:105920004FF4A02022F4E02208BF4FF48030019E03
:10593000104320600869C1032AD4C8B30121D645A9
:1059400021EA00004FF0E06153F8202022F0E062ED
:1059500008BF4FF0407128E04FF480326FF4E02729
:10596000012626EA000053F8206037403A4343F806
:1059700020200869C10323D4019EC8B1012103225C
:1059800021EA000053F8201062F31A610EE000BF14
:105990000121D64521EA00004FF4E02153F82020F0
:1059A00008BF4FF4403122F4E022114443F82010A4
:1059B000F00712D1B00718D400200EB0BDE8F08F68
:1059C0000121032221EA000053F8201062F3124162
:1059D00043F82010019EF007ECD0DAF8000040F008
:1059E0000100CAF80000B007E6D5286840F00100C1
:1059F000286000200EB0BDE8F08F0000000000001D
:105A0000F0B581B00446FFF7BBFB002C00F08980A5
:105A1000054600206065216D11B101B0F0BD00BFE9
:105A2000204600F081F8206841F28836A6654FF6DE
:105A3000F40ED4E903C263698168CFF6E00E002753
:105A4000CFF6FF7701EA0E0107EB024241EA0C01B3
:105A50006FF0FF0E676B11430EEB03223943E369CE
:105A6000114319438160C168226A21F4E021114386
:105A7000C160216BA26B42EA01410161E16B4161AE
:105A80000168626821F4F8510EEB022211430160B3
:105A9000016A890609D500BFFFF772FB401BB042BF
:105AA00038D82068016A8906F6D4C168A268D4E9AA
:105AB000097621F0FF01013FA3693943C160022B40
:105AC000016821F0400141EA02010160D0F80811AB
:105AD000E26A21F0A04141EA060141EA0201C0F870
:105AE0000811016841F00101016003D1816841F0B2
:105AF00002018160E068B0F1806F05D1012020656E
:105B0000002001B0F0BD00BF02202065002001B0E0
:105B1000F0BD00BF4FF400702065606D40F00100E3
:105B20006065012001B0F0BD2DE9F04FB5B004462D
:105B300002A80830B02100253095CDE93355CDE9D4
:105B40003155FBF7D0F845F200012068C5F200217D
:105B5000884203D035B0BDE8F08F00BF4FF0007031
:105B6000029002A80395159500F07AFE08B1FBF7A4
:105B700037FF44F2E04040F20008C5F60200C5F6E7
:105B8000020830AC022750F80C1C4FF0000941F419
:105B9000001140F80C1C50F80C1C4FF0030B01F4E2
:105BA00000110191019950F80C1C41F4804140F81A
:105BB0000C1C50F80C1C4FF0090A01F480410191B3
:105BC0000199016841F001010160016801F00101E2
:105BD00001910199016841F002010160016801F041
:105BE000020101910199016841F010010160016811
:105BF00001F0100101910199016841F00801016073
:105C00000068214600F00800019001984046CDE967
:105C10003077CDF8C890CDF8CCB0CDF8D0A0FFF754
:105C2000B3F930A9082081E8810A06203490404663
:105C30002146FFF7A9F930A9012008F5806604255F
:105C400081E8810A304621463495FFF79DF930A856
:105C50002146CDF8D0A080E8A00A3046FFF794F99D
:105C600030A84FF40065214680E8A00A0B2034904C
:105C700008F58050FFF788F930A82146CDF8D0A06C
:105C800080E8A00A08F54060FFF77EF935B0BDE86E
:105C9000F08F00000000000001680122C0F8D82445
:105CA000002280F8CC24886940F000608861486D4B
:105CB00040F08052002042F003024A657047000025
:105CC000F0B581B0002800F02781044690F89504D3
:105CD00028B9002084F89404204600F035F9032008
:105CE00084F89504206807F0EBF8D4E90001267CDD
:105CF000D4E90223009606F023FE002840F0098133
:105D00002068002107F0E4F8002840F002812179A2
:105D1000002900F0F580A1F1010C01F0030EBCF1A7
:105D2000030F4FF0000345D301F0FC0204F19A0089
:105D30000126002500F8865C6F1C20F86C5C00F8DA
:105D4000627C20F8487CAF1C00F83E7C20F8247C64
:105D5000EF1C043500F8856C00F8823CAA4240F83C
:105D60007E3C40F87A3C40F8763C00F8616C00F8E4
:105D70005E3C40F85A3C40F8563C40F8523C00F833
:105D80003D6C00F83A3C40F8363C40F8323C40F874
:105D90002E3C00F8196C00F81A7C078000F8163CBD
:105DA00040F8123C40F80E3C40F80A3C00F19000EC
:105DB000C0D12B46BEF1000F2DD003EBC300012252
:105DC000BEF1010F04EB80054FF000006A752B75E2
:105DD000EB852876C5E9070068621CD05D1CBEF122
:105DE000020F05EBC50604EB860672753575F58561
:105DF0003076C6E9070070620DD0981C012300EBD5
:105E0000C00204EB820253751075D0850020107615
:105E1000C2E907005062BCF1030F4FF0000237D314
:105E200001F0FC0004F53471002300BF01F87C3C54
:105E30005F1C01F8587C9F1C01F8347CDF1C043384
:105E400001F87B2C01F8782C984241E91D2241F899
:105E50006C2C01F8572C01F8542C41E9142241F81C
:105E6000482C01F8332C01F8302C41E90B2241F881
:105E7000242C01F80F2C01F8107C01F80C2C41F8AF
:105E8000082C41F8042C0A6001F19001CED11A4689
:105E9000BEF1000F34D002EBC200BEF1010F04EBE3
:105EA00080014FF0000081F8550281F8542281F8FA
:105EB0005802C1E99700C1F8640221D0511CBEF11B
:105EC000020F01EBC10304EB830383F8550283F84F
:105ED000541283F85802C3E99700C3F864020FD044
:105EE000901C002200EBC00104EB810181F85522D7
:105EF00081F8540281F85822C1E99722C1F864223E
:105F0000D4E90001277CD4E90223009706F040FE83
:105F100030B1022084F89504012001B0F0BD00BF2B
:105F200000206074012084F89504207B012802D1B0
:105F30002046FFF7B1FE206806F01AFE002001B0EF
:105F4000F0BD00000000000010B5B0B002A904468A
:105F500001F10800B021FAF7C6FE00212068C4F262
:105F60000401884202D030B010BD00BF0020039071
:105F70004FF4802002904FF44010239002A800F0CC
:105F80006FFC08B1FBF72CFD00F03AF844F2D84062
:105F9000C5F60200016841F000710160006800F080
:105FA00000700190019830B010BD000000000000AA
:105FB000B0B544F60C05C5F60205296849072968FD
:105FC00006D401F00701081A18BF0120B0BD00BFB8
:105FD00021F0070108432860FFF7D2F8044600BF0C
:105FE00055F8080C800407D4FFF7CAF8001BB0F579
:105FF0007A7FF5D90120B0BD0020B0BD00000000BF
:1060000044F60C00C5F60200016841F080710160A1
:10601000704700000000000080B501F0D9FA44F29A
:10602000204140F23C32C5F60201C0F60102096887
:10603000C1F30211515C01F01F01C84080BD000096
:1060400080B544F2304EC5F6020E5EF8083C5EF8AC
:10605000081CC1F3051C5EF8041CBCF1000FDEF83F
:10606000042017D0C2F3CC0201F00101514303F028
:106070000303022B00EE101AB8EE400A10D0012BD9
:1060800012D01BB95EF8301C890611D49FED361A68
:106090001CE000BF00218160C0E9001180BD00BF8D
:1060A0009FED301A12E000BF9FED2D1A0EE000BFE9
:1060B0005EF8301C49F20002C0F2D032C1F3C101D7
:1060C00022FA01F101EE101AB8EE411ADEF80010C2
:1060D0009FED263A6FF35F2102EE101ADEF80010F2
:1060E000C1F34621B8EE422A00EE032A00EE10CAA0
:1060F000B7EE003AB8EE400A81EE000A32EE031A1B
:1061000002EE101AB8EE422A20EE010A32EE031A0D
:1061100080EE011ABCEEC11A80ED001ADEF8001004
:10612000C1F3064101EE101AB8EE411A31EE031A1E
:1061300080EE011ABCEEC11A80ED011ADEF80010E3
:10614000C1F3066101EE101AB8EE411A31EE031ADE
:1061500080EE010ABCEEC00A10EE101A816080BD0C
:106160000024744A001BB74B0024744C0000003913
:1061700080B544F2384EC5F6020E5EF8103C5EF86B
:10618000101CC1F3053C5EF80C1CBCF1000FDEF8DE
:10619000042015D0C1F30011C2F3CC02514300EE2C
:1061A000101A03F003010229B8EE400A0ED089B993
:1061B0005EF8381C890611D49FED361A1CE000BF2A
:1061C00000218160C0E9001180BD00BF9FED301A41
:1061D00012E000BF9FED2D1A0EE000BF5EF8381CE4
:1061E00049F20002C0F2D032C1F3C10122FA01F13A
:1061F00001EE101AB8EE411ADEF800109FED263AB3
:106200006FF35F2102EE101ADEF80010C1F3462191
:10621000B8EE422A00EE032A00EE10CAB7EE003AAA
:10622000B8EE400A81EE000A32EE031A02EE101AAE
:10623000B8EE422A20EE010A32EE031A80EE011A6D
:10624000BCEEC11A80ED001ADEF80010C1F3064161
:1062500001EE101AB8EE411A31EE031A80EE011A5F
:10626000BCEEC11A80ED011ADEF80010C1F3066120
:1062700001EE101AB8EE411A31EE031A80EE010A4F
:10628000BCEEC00A10EE101A816080BD0024744A72
:10629000001BB74B0024744C0000003900000000C4
:1062A00080B544F2404EC5F6020E5EF8183C5EF82A
:1062B000181CC1F3055C5EF8141CBCF1000FDEF87D
:1062C000042015D0C1F30021C2F3CC02514300EEEB
:1062D000101A03F003010229B8EE400A0ED089B962
:1062E0005EF8401C890611D49FED361A1CE000BFF1
:1062F00000218160C0E9001180BD00BF9FED301A10
:1063000012E000BF9FED2D1A0EE000BF5EF8401CAA
:1063100049F20002C0F2D032C1F3C10122FA01F108
:1063200001EE101AB8EE411ADEF800109FED263A81
:106330006FF35F2102EE101ADEF80010C1F3462160
:10634000B8EE422A00EE032A00EE10CAB7EE003A79
:10635000B8EE400A81EE000A32EE031A02EE101A7D
:10636000B8EE422A20EE010A32EE031A80EE011A3C
:10637000BCEEC11A80ED001ADEF80010C1F3064130
:1063800001EE101AB8EE411A31EE031A80EE011A2E
:10639000BCEEC11A80ED011ADEF80010C1F30661EF
:1063A00001EE101AB8EE411A31EE031A80EE010A1E
:1063B000BCEEC00A10EE101A816080BD0024744A41
:1063C000001BB74B0024744C000000390000000093
:1063D00010B584B0024641F6FF7300209B1A70EBA3
:1063E00001032DDA47F6FF739B1A70EB010380F26D
:1063F000798082F400430B4300F0A08082F4803364
:106400000B4300F0E38082F40022114340F01E8130
:1064100044F20040C5F60200816D01F44031B1F54F
:10642000003F00F01F81B1F5803F00F0FD800029A2
:1064300040F0E1810068000100F17D81DBE100BFF7
:1064400040F2FF739B1A70EB010325DB82F480732B
:106450000B4300F0878082F48062114340F0F680A5
:1064600044F20041C5F60201886DC0F34252042A8D
:1064700000F2C18148F20000C0F2BB00DFE812F078
:10648000060000010601E6000C0100BF086880015B
:1064900040F1B181E0E000BF82F400630B4300F003
:1064A0007B8082F48052114340F0D08044F200415E
:1064B000C5F60201086DC0F30232042A00F29B8186
:1064C00048F20000C0F2BB00DFE812F00600F8005E
:1064D000FE00C000040100BF0868800140F18B810C
:1064E000BAE000BF82F400530B4300F07B8082F4DB
:1064F0008042114340F0AA8044F20044C5F60204F1
:10650000A06DC0F30270052800F27581DFE810F07D
:106510000600420146014A015001520101F058F8BB
:10652000216A40F23C32C0F60102C1F30211515C13
:1065300001F01F01C84004B010BD00BF44F200408C
:10654000C5F60200016D01F04051B1F1005F00F0AD
:106550007580B1F1805F00F07B80002940F04B81B5
:1065600060E000BF44F20041C5F60201086D00F092
:106570000702042A00F23F8148F20000C0F2BB008B
:10658000DFE802F004BAC064C40000BF08688001FC
:1065900040F1318160E000BF44F20041C5F60201E4
:1065A000886DC0F30262042A00F2258148F20000DF
:1065B000C0F2BB00DFE802F004BCC64AD00000BF56
:1065C0000868800140F1178146E000BF44F20040B6
:1065D000C5F60200C16C0068C90319D4800140F1FE
:1065E0000A8139E044F20040C5F60200016DC1F3B2
:1065F0000241052900F2FF80DFE811F00600E60005
:10660000F000FA000001140001F00AF804B010BD17
:10661000000140F1F08001A8FFF7AAFD039804B043
:1066200010BD00BF0068C6E00068800040F1E38054
:1066300001A8FFF735FE039804B010BD0068000103
:1066400040F1D98001A8FFF793FD029804B010BD76
:106650000068800140F1CF8001A8FFF7F1FC0298AB
:1066600004B010BDC16C036811F04051026840F0E5
:10667000CF8013F0040300F0CB80C2F3C100D6E05A
:106680000868000140F1B78055E000BF086880004D
:1066900040F1B18059E000BFC86C0B6810F0405267
:1066A000086803D113F0040340F0BF80B2F1805FAB
:1066B00061D110F4807040F0B1805CE008680001A6
:1066C00040F1998037E000BF0868800040F1938076
:1066D0003BE000BFC86C0B6810F04052086803D163
:1066E00013F0040340F0A180B2F1805F43D110F4B5
:1066F000807040F093803EE00868000140F17B80AC
:1067000019E000BF0868800075D51EE0C86C0B68F2
:1067100010F04052086803D113F0040340F0858064
:10672000B2F1805F27D110F4807077D123E000BFF1
:10673000086800015FD501A8FFF71AFD019804B0B1
:1067400010BD00BF0868800055D501A8FFF7A8FD5F
:10675000019804B010BD00BFC86C0B6810F0405227
:10676000086802D113F004035FD1B2F1805F02D157
:1067700010F4807052D1086810F400301CBF43F24E
:106780000060C0F26E10B2F1005F18BF002004B0CC
:1067900010BD00BF206800012DD518E020688000E2
:1067A00029D51EE02068400725D520683DE000BFC0
:1067B000206824E0206843F200618003C0F26E117B
:1067C00001EAE07004B010BD0068000113D501A813
:1067D000FFF7CEFC029804B010BD00BF0068800037
:1067E00009D501A8FFF75CFD029804B010BD00BFF9
:1067F0000168490718D4002004B010BD006840F6B5
:106800000011C005C0F23D0101EAE07004B010BD06
:10681000B1F1805F14D112F4807211D040F60010F3
:10682000C0F23D0004B010BD0068C0F3C10049F2E1
:106830000001C0F2D03121FA00F004B010BD00BF59
:10684000006810F400301CBF43F20060C0F26E100C
:10685000B1F1005F18BF002004B010BD00000000BF
:106860002DE9F0470446C07844F22C480007C5F6ED
:10687000020833D5606E4FEA305103290CD8DFE8A7
:1068800001F003111D2600BFD8F8001041F40031BB
:10689000C8F800101BE000BF01266078C0070BD0CD
:1068A00020E000BF04F10800022104F06DFB064661
:1068B00060B16078C00715D1354646E004F1280084
:1068C000022104F0F5FB06460028F2D1606ED8F8EC
:1068D000241021F440110843C8F8240000266078F1
:1068E000C007E9D0A06D04280ED83546DFE800F0D7
:1068F0000412181E1E0000BFD8F80000354640F4F0
:106900000030C8F8000011E0012501276078400739
:106910001FD453E004F10800002104F035FB04E02B
:1069200004F12800002104F0C3FB05462F461DB1E9
:10693000607840070DD441E0D8F82400A16D20F024
:10694000070000250843C8F8240037466078400750
:1069500034D5D4F8A4004FEA705005280CD8DFE8ED
:1069600000F00311171D1D1DD8F8000040F4003081
:10697000C8F8000012E000BF01250126607800077A
:1069800020D455E004F10800002104F0FDFA04E0F1
:1069900004F12800002104F08BFB05462E461DB1B2
:1069A000607800070ED443E0D8F82C00D4F8A41087
:1069B00020F4600000250843C8F82C003E466078AB
:1069C000000735D5D4F8A8004FEA306005280DD867
:1069D000DFE800F00412181E1E1E00BFD8F80000E9
:1069E00040F40030C8F8000012E000BF0125012784
:1069F000E078800720D44EE004F10800002104F084
:106A0000C3FA04E004F12800002104F051FB05461C
:106A10002F461DB1E07880070ED43CE0D8F82C005A
:106A2000D4F8A81020F0E06000250843C8F82C0036
:106A30003746E07880072ED5E06C4FEA3010032807
:106A40000ED8DFE800F00903130900BFD8F80000F2
:106A500040F40030C8F800002E467DB912E000BFB7
:106A6000012501266078C00619D44CE004F1080025
:106A7000022104F089FA05462E461DB16078C00651
:106A80000DD440E0D8F82000E16C20F03000002563
:106A90000843C8F820003E466078C00633D5E06D54
:106AA0004FEA303004280DD8DFE800F00412181E39
:106AB0001E0000BFD8F8000040F40030C8F8000005
:106AC00012E000BF01250127607880061FD44EE048
:106AD00004F10800002104F057FA04E004F1280052
:106AE000002104F0E5FA05462F461DB160788006C6
:106AF0000DD43CE0D8F82400E16D20F4E0400025FE
:106B00000843C8F824003746607880062FD5206EE9
:106B10004FEA3040052809D8DFE800F0040E1404DD
:106B2000040400BF2E46ADB918E000BF01250126C0
:106B3000607840061FD44FE004F10800012104F002
:106B400023FA04E004F12800012104F0B1FA05461B
:106B50002E461DB1607840060DD43DE0D8F82400E3
:106B6000216E20F4E02000250843C8F824003E46AA
:106B70006078400630D5D4F8AC004FEA3070052874
:106B800008D8DFE800F0030D130303032F46ADB967
:106B900018E000BF012501276078000620D442E0FC
:106BA00004F10800012104F0EFF904E004F12800E9
:106BB000012104F07DFA05462F461DB160780006DC
:106BC0000ED430E0D8F82C00D4F8AC1020F0E0401F
:106BD00000250843C8F82C0037466078000622D507
:106BE000E06E58B1B0F1005F0CD0B0F1805F2FD1F2
:106BF000D8F8000040F40030C8F800002E469DB9D7
:106C000008E000BF04F10800012104F0BDF90546C9
:106C10002E464DB9D8F82400E16E20F040500025F2
:106C20000843C8F824003E46E078C00733D0A06C83
:106C3000032813D8DFE800F008021A08D8F800008B
:106C400040F40030C8F80000A946BDB91AE000BF02
:106C500001250126E078C007E9D11CE001254FF0AD
:106C60000109A07840061AD51CE000BF04F1080015
:106C7000022104F089F90546A9461DB1A078400615
:106C80000DD50FE0D8F82000A16C20F003000025FE
:106C90000843C8F82000B146A078400602D44F4609
:106CA00018E000BFD8F8D40340F48070C8F8D403CB
:106CB000FEF766FA064600BFD8F8D403C00507D42D
:106CC000FEF75EFA801B6428F6D90325032701E04E
:106CD0002F468DB12078C00761D0A06F4FEAF00039
:106CE00005283BD8DFE800F004404604040400BF58
:106CF000002D2E4646D149E0D8F84410D4F8B00013
:106D0000414011F4407F11D0D8F84410D8F8442005
:106D100042F48032C8F84420D8F8442021F440716D
:106D200022F48032C8F84420C8F84410B0F5807FBF
:106D300040F0D082FEF724FA064641F2883A032555
:106D4000032700BFD8F84400800700F1C182FEF796
:106D500017FA801B5045F5D9BCE700BF0125012675
:106D6000207880071FD44CE004F10800012104F0D2
:106D70000BF904E004F12800012104F099F905461B
:106D80002E461DB1207880070DD43AE0D8F82800AF
:106D9000A16F20F0380000250843C8F828003E46BF
:106DA000207880072DD5606F052809D8DFE800F02E
:106DB000040E1404040400BF2F46ADB918E000BF50
:106DC00001250127207840071FD44DE004F1080079
:106DD000012104F0D9F804E004F12800012104F0B5
:106DE00067F905462F461DB1207840070DD43BE0DA
:106DF000D8F82800616F20F0070000250843C8F884
:106E000028003746207840072ED5D4F89000052872
:106E100008D8DFE800F0030D130303032E46ADB9D5
:106E200018E000BF012601252078800620D451E01B
:106E300004F10800012104F0A7F804E004F128009F
:106E4000012104F035F905462E461DB12078800653
:106E50000ED43FE0D8F82C00D4F8901020F00700B2
:106E600000250843C8F82C003E462078800631D51E
:106E7000D4F88C004FEA3070052809D8DFE800F01C
:106E8000040E1404040400BF2F46ADB918E000BF7F
:106E9000012701252078400620D451E004F10800A4
:106EA000002104F071F804E004F12800022104F04C
:106EB000FFF805462F461DB1207840060ED43FE06E
:106EC000D8F82800D4F88C1020F0E04000250843C2
:106ED000C8F8280037462078400631D5D4F8980005
:106EE0004FEAB020052809D8DFE800F0040E1404AA
:106EF000040400BF2E46ADB918E000BF01260125ED
:106F00002078000620D454E004F10800002104F0A9
:106F10003BF804E004F12800022104F0C9F805461A
:106F20002E461DB1207800060ED442E0D8F82C0081
:106F3000D4F8981020F4E05000250843C8F82C003D
:106F40003E462078000634D5D4F89C004FEA7030D5
:106F500005280FD8DFE800F004141A04040400BF69
:106F60002F46E5B12068010727D4C1063ED40003AF
:106F700055D475E00127012520680107F5D51CE0EF
:106F800004F10800002103F0FFFF04E004F12800F1
:106F9000022104F08DF80546002D2F46E2D1D8F8E5
:106FA0002C00D4F89C1020F4604000250843C8F859
:106FB0002C00374620680107D7D5D4F88010B1F5EA
:106FC000805F0AD104F12800022104F071F8002842
:106FD00018BF01272068D4F88010D8F8282022F4A0
:106FE00040521143C8F82810C106C0D5D4F89410F7
:106FF000B1F5807F0AD104F12800022104F058F88D
:10700000002818BF01272068D4F89410D8F82C2045
:1070100022F440721143C8F82C10000320D5D4F894
:10702000A000B0F5003F0FD0B0F5803F06D078BB90
:1070300004F10800002103F0A7FF04E004F1280098
:10704000022104F035F805462E4655B9D8F82C0033
:10705000D4F8A01020F4403000250843C8F82C00D4
:107060003E46A07840072BD5D4F88400B0F5401FE9
:107070000BD0B0F5001F11D0B0F5801F2AD1D8F881
:10708000000040F40030C8F800002F46CDB90DE0F4
:1070900001260125A0784007E6D411E004F128007C
:1070A000012104F005F805462F4655B9D8F8280007
:1070B000D4F8841020F4401000250843C8F82800B4
:1070C0003746A078C0070AD13E462168880016D509
:1070D00033E000BF01270125A078C007F4D0206D60
:1070E000B0F5803F10D018BBD8F8000040F4003055
:1070F000C8F800002E4685B1216888001DD460685C
:107100008A0326D467E000BF04F10800022103F0DF
:107110003BFF0546002D2E46EED1D8F82000216D0C
:1071200020F4803000250843C8F82000CCE700BFD9
:107130000126012521688800E1D504F128000221FB
:1071400003F0B6FF002818BF0126D4E900108A0317
:1071500041D5E26F6FF0010303EB3223022B0BD317
:107160004FEA322343B1012B40F0AC80D8F8003015
:1071700043F40033C8F8003035B3CA022ED48A0273
:1071800036D44A003ED4B1F1FF3F4BDD090253D45F
:10719000C1075CD1810765D441076ED4010778D45B
:1071A000C10600F18280800607D504F12800022183
:1071B00003F07EFF002818BF0125002D18BF012510
:1071C0002846BDE8F08700BFD8F8283023F4407384
:1071D0001A43C8F828203546CA02D0D5D8F824204A
:1071E000236F22F000421A43C8F824208A02C8D52F
:1071F000D8F82420A36E22F080721A43C8F8242005
:107200004A00C0D558F81C2C22F4004248F81C2C27
:10721000D4F8B42058F81C3C1A4348F81C2CB1F19F
:10722000FF3FB3DCD8F82020636D22F040521A43B0
:10723000C8F820200902ABD5D8F82810D4F8882047
:1072400021F440011143C8F82810C107A2D004F16D
:107250000800002103F098FE002818BF054660686A
:10726000810799D504F10800012103F08DFE002863
:1072700018BF05466068410790D504F10800022157
:1072800003F082FE002818BF0546606801077FF5FD
:1072900087AF04F12800002103F00AFF002818BF7F
:1072A00005466068C1067FF57EAF04F12800012124
:1072B00003F0FEFE002818BF0546606880067FF5D3
:1072C0007CAF72E70125CA027FF559AF86E700BFA0
:1072D000D4F8B0004FF6CF7358F81C2CC0F2FF035F
:1072E00000F4407122F47C5203EA10136FF31F3054
:1072F000B1F5407F08BF1A43002548F81C2CD8F888
:1073000044100843C8F84400FFF7C9BC000000005F
:107310002DE9F04381B0002800F02A8142F20008F4
:107320000446C5F200288946D8F8000000F00F0096
:1073300088420ED2D8F8000020F00F0040EA090081
:10734000C8F80000D8F8000000F00F00484540F0F1
:107350000F81206844F218474107C5F602070AD595
:1073600021693A6802F07002914204D93A6822F029
:1073700070021143396001070AD561697A6802F029
:107380007002914204D97A6822F070021143796048
:10739000C1060AD5A1697A6802F4E062914204D973
:1073A0007A6822F4E0621143796081060AD5E169C6
:1073B000BA6802F07002914204D9BA6822F07002F1
:1073C0001143B96010F002010AD0E2683B6803F093
:1073D0000F039A4204D93B6823F00F031A433A6023
:1073E000C20746D0386820F47061D4E90102012850
:1073F00041EA0201396009D003280DD0022811D1D9
:1074000057F8181C890340F1B38010E057F8181C96
:10741000C90540F1AD800AE057F8181C890140F118
:10742000A78004E057F8181C490740F1A18057F8DD
:10743000081C21F00701084347F8080CFDF7A0FEDF
:10744000064641F2883500BF57F8080C616800F025
:107450003800B0EBC10F09D0FDF792FE801BA842A7
:10746000F2D9032001B0BDE8F08300BF206800F02E
:10747000020151B1E1683A6802F00F02914204D270
:107480003A6822F00F0211433960D8F8001001F079
:107490000F0149450DD9D8F8001021F00F0141EA3C
:1074A0000901C8F80010D8F8001001F00F01494593
:1074B0005ED141070AD521693A6802F07002914213
:1074C00004D23A6822F070021143396001070AD5EC
:1074D00061697A6802F07002914204D27A6822F0FF
:1074E000700211437960C1060AD5A1697A6802F475
:1074F000E062914204D27A6822F4E062114379603A
:1075000080060AD5E069B96801F07001884204D2AA
:10751000B96821F070010843B86000F0E1F83968FB
:1075200040F23C333A68C0F60103C1F3032102F094
:107530000F02595C9A5C01F01F0120FA01F102F080
:107540001F0040F20C0221FA00F0C2F2004210606B
:1075500040F2040040F20802C2F20040C2F20042CF
:107560000068116001B0BDE8F043FDF755BE00BFF3
:10757000012001B0BDE8F0833F22026044F21842CE
:10758000C5F6020252F8083C03F007034360136893
:1075900003F470638360136803F00F03C360136820
:1075A00003F070030361536803F070034361536891
:1075B00003F4E0638361926802F07002C26142F2F8
:1075C0000000C5F20020006800F00F00086070475E
:1075D00080B500F085F844F2184140F23C33C5F61E
:1075E0000201C0F601030A68096801F00F01C2F345
:1075F0000322595C9A5C02F01F0220FA02F201F0A9
:107600001F0040F20C0122FA00F0C2F200410860B3
:1076100040F20801C2F200410A6080BD0000000093
:1076200080B500F05DF844F2184C40F23C31C5F6EC
:10763000020CC0F60101DCF80020DCF8003003F099
:107640000F03C2F30322CB5C8A5C02F01F02D0401E
:1076500003F01F0240F20C0320FA02F2C2F20043D0
:107660001A6040F20803C2F200431860DCF804001C
:10767000C0F30210085C00F01F0022FA00F080BD89
:1076800080B500F02DF844F2184C40F23C31C5F6BC
:10769000020CC0F60101DCF80020DCF8003003F039
:1076A0000F03C2F30322CB5C8A5C02F01F02D040BE
:1076B00003F01F0240F20C0320FA02F2C2F2004370
:1076C0001A6040F20803C2F200431860DCF80400BC
:1076D000C0F30220085C00F01F0022FA00F080BD19
:1076E00044F20041C5F602010869C0F3C200032854
:1076F00010D002282CD088BB0868800649F2000010
:10770000C0F2D03058BF70470968C1F3C101C8400A
:10771000704700BF8A6A886AC0F3051CC86ABCF15A
:10772000000F4B6B20D0C3F3CC0300F00100584393
:1077300002F00302022A00EE100AB8EE400A15D049
:10774000C2B90868800619D49FED281A23E000BF4B
:1077500043F20060C0F26E10704700BF40F60010A8
:10776000C0F23D00704700BF002070479FED1E1A19
:1077700011E000BF9FED1B1A0DE000BF086849F241
:107780000002C0F2D032C0F3C10022FA00F001EED4
:10779000100AB8EE411A086B9FED153A6FF35F209F
:1077A00002EE100A086BC0F34620B8EE422A013000
:1077B00000EE032A00EE10CAB7EE003AB8EE400A17
:1077C00081EE000A32EE031A20EE010A01EE100AE1
:1077D000B8EE411A80EE010ABCEEC00A10EE100AA3
:1077E000704700BF0024744A001BB74B0024744C40
:1077F000000000390000000070B586B0002844F297
:10780000E04640F2000014460D46C5F60206C5F6F5
:1078100002001DD0316800F5006041F004013160C4
:10782000316801F00401019101994FF40071019157
:10783000022102910321049100210391059101A9E4
:10784000FDF7A2FB56F8D00CE40120F07E4019E0D1
:10785000316841F001013160316801F001010191AD
:1078600001994FF480710191022102910321049149
:1078700000210391059101A9FDF786FB56F8D00C74
:1078800020F0FE7044EA0501084346F8D00C06B02B
:1078900070BD000000000000F0B581B0002800F0CD
:1078A000D5800446007844F20046C007C5F60206BB
:1078B00022D12078800768D5306910F03801B06A8D
:1078C00042D0182908BF5FEA80703DD0E068316877
:1078D000002800F0258121F0190108433060FDF7F0
:1078E0004FFC05463068400748D4FDF749FC401B73
:1078F0000228F7D977E100BF306900F03801B06A9B
:10790000102905D018290BD100F00300022807D157
:1079100030688003CDD560680028CAD196E000BFEA
:107920006068002800F03281B0F5A02F00F0468199
:10793000B0F5803F00F04681306820F48030306040
:10794000306820F4802040E130684007E06801D5CD
:1079500000287BD0316821F0190108433060FDF721
:107960000FFC05463068400708D4FDF709FC401BB2
:1079700002284FF00300F5D901B0F0BD706821690D
:1079800020F0FE4040EA016070602078C00619D502
:10799000306900F03801B06A082906D0182940F093
:1079A000818000F0030001287CD13068C00502D539
:1079B000E06980284AD1F068216A20F07C5040EAD2
:1079C0000160F0602078000744D42078800655D408
:1079D0002078400700F17E80656A9DB3306900F031
:1079E0003800182840F01481012DB16A306B2DD079
:1079F00001F00302A36A9A4228D1C1F30511E26A99
:107A0000914223D10146226B6FF35F21013A9142EB
:107A10001CD1C0F34622616B01398A4216D1C0F3F2
:107A20000642A16B01398A4210D1C0F30660E16BB6
:107A3000013988420AD1706BA16CC0F3CC0081423D
:107A400040F09C81002001B0F0BD00BF012001B0DA
:107A5000F0BD00BF60690028706F4FD040F001009A
:107A60007067FDF78DFB0546706F8007ADD4FDF79D
:107A700087FB401B0228F7D9B5E000BFA0690028AA
:107A8000306871D040F480503060FDF779FB0546D6
:107A9000306880049CD4FDF773FB401B0228F7D9A3
:107AA000A1E000BFE0690028306800F09F8040F04E
:107AB00080003060FDF764FB054600BF3068C005FC
:107AC0003FF579AFFDF75CFB401B02284FF0030048
:107AD000F4D951E7D6F8000440F48070C6F80004E9
:107AE000FDF74EFB054600BFD6F80004C00529D4BB
:107AF000FDF746FB401B6428F6D974E020F0010036
:107B00007067FDF73DFB0546706F80077FF55DAF41
:107B1000FDF736FB401B02284FF00300F4D92BE79A
:107B200021F001003060FDF72BFB0546306840076F
:107B30007FF52BAFFDF724FB401B02284FF003001D
:107B4000F4D919E7A068002800F08480052800F027
:107B50009B80012800F09C80306F20F0010030678E
:107B6000306F20F0040096E020F480503060FDF784
:107B700007FB0546306880047FF52AAFFDF700FB60
:107B8000401B02284FF00300F4D9F5E6306820F4DA
:107B900080303060306820F480203060FDF7F0FAEB
:107BA000054600BF306880037FF583AEFDF7E8FA35
:107BB000401B64284FF00300F4D9DDE6306840F440
:107BC00080203060306840F480303060FDF7D8FAB3
:107BD000054600BF306880033FF56BAEFDF7D0FA75
:107BE000401B6428F6D9032001B0F0BD20F08000CE
:107BF0003060FDF7C5FA05463068C0057FF5E2AE96
:107C0000FDF7BEFA401B02284FF00300F4D9B3E69B
:107C1000306820F080703060FDF7B2FA022D054622
:107C20000CD100BF3068800148D5FDF7A9FA401B90
:107C300002284FF00300F5D99EE600BF30688001AE
:107C40007FF500AFFDF79CFA401B02284FF00300C0
:107C5000F4D991E6306F20F001003067306F20F0EA
:107C600004003067FDF78CFA054641F28837306F23
:107C700080077FF5B1AEFDF783FA401BB8424FF0A5
:107C80000300F4D978E600BF306F40F0040030679D
:107C9000306F40F001003067FDF772FA054641F29F
:107CA000883700BF306F80073FF596AEFDF768FA62
:107CB000401BB8424FF00300F4D95DE604F12807F9
:107CC000B06A40F2F33188438ECF0843591E40EA30
:107CD00002104FF47E426FF35F21B06202EB472047
:107CE0004FF4FE0280B2E36B0844A16B02EB01414A
:107CF0004FF0FE4201F4FE0102EB0362084402F081
:107D0000FE4108443063F06A4FF6F87120F001003C
:107D1000F062706BA26C884340EAC2007063F06A44
:107D2000216C20F00C000843F062F06A616C20F0D6
:107D300002000843F062F06A40F48030F062F06ABA
:107D400040F40030F062F06A40F48020F062F06AA3
:107D500040F00100F062306840F080703060FDF764
:107D60000FFA0446306880013FF56CAEFDF708FA63
:107D7000001B02284FF00300F4D9FDE5F06A20F063
:107D80000100F062FDF7FCF90546FDF7F9F9A8429C
:107D9000FBD0706B4FF6F871A26C884340EAC200CA
:107DA0007063F06A40F00100F062002001B0F0BDA5
:107DB000F0B581B0F8B10446D0F888001E461546EB
:107DC0000F4628B9002084F88400204601F0DCFD2D
:107DD0002420C4F888002068A16A0268002922F0E3
:107DE0000101016002D0204603F09EFD204604F010
:107DF000ABF8012802D1012001B0F0BD20688168F4
:107E000041F480418160816821F4004139438160FF
:107E10003104026841EA45516FF319421143016090
:107E2000016841F001010160204601B0BDE8F04069
:107E300003F0EABD0000000043F600010068C4F250
:107E40000001884208D140F67870C2F20040806993
:107E5000002808BF7047004770470000000000007E
:107E60002DE9F04381B00446066830697169D6F89F
:107E7000089094F8818002070CD511F4006209D0B3
:107E8000B06940F40060B061204601B0BDE8F04345
:107E900000F006BB01EA000505F06407042F05D1D8
:107EA000616F20468847216F2046884705F04500CE
:107EB000012807D1216F2046884705F026000228B7
:107EC00004D00BE005F02600022805D1616F2046A2
:107ED00001B0BDE8F0430847042F03D101B0BDE86D
:107EE000F08300BF280715D415F4587FF6D015F09D
:107EF000400065D1A80570D4E80505F020007CD4C9
:107F0000002840F08880D4F88400002840F0938056
:107F1000E4E700BF2068816941F00801816181695F
:107F200041F010018161816941F400618161016961
:107F300021F008010161806810F4404F27D02046ED
:107F400003F052F9012084F88100D4F8840000285D
:107F500040F0AB80B8F1030F00F0AE80B8F1040F31
:107F600000F0B080B8F1050FB8D1204601B0BDE8EF
:107F7000F04300F0ADBA00BF2068616E006B41F8BD
:107F8000040B6166B4F86A000138A4F86A00B4F81A
:107F90006A000028D3D0E0681028EDD2082805D365
:107FA000308E616E21F8020BEBE700BF206890F87D
:107FB0003000616E0870606E01306066E2E700BFFD
:107FC0002068D4F8841041F00401C4F88410816959
:107FD00041F040018161A8058ED52068D4F8841055
:107FE00041F00101C4F88410816941F4007181619C
:107FF000E80505F020007FF583AF2168D4F88420E0
:1080000042F00802C4F884208A6942F480728A61CE
:1080100000283FF478AF2068D4F8841041F0800144
:10802000C4F88410816941F020018161D4F8840092
:1080300000283FF453AF206809F4404240F26B330C
:10804000B2F5404F016821F001010160016921EAA8
:108050000301016126D181684BF2B92521F4404129
:108060008160E06FC0F6000548B10565FAF7F0FEE3
:1080700028B1D4F8840040F04000C4F88400A06F18
:1080800000283FF42BAF0565FAF7E2FE00283FF425
:1080900025AFD4F8840040F04000C4F8840001B05B
:1080A000BDE8F083012084F88100204601B0BDE8DE
:1080B000F043FFF7C1BE00BF204601B0BDE8F0436A
:1080C00000F0F2B9204601B0BDE8F04300F0D4B9A9
:1080D0002DE9F047002858D043F600030446006815
:1080E000C4F2000343F2000E43F6004C9842C4F27F
:1080F000010EC4F2000C4FF00001A16203D06045F4
:1081000018BF70453ED1E16B0122E568984202EB51
:10811000511105F108024FEAD20202FB01F118BF2A
:10812000704525D1102930D894F8811031B900203C
:1081300084F88000204600F09FF82068022184F82F
:108140008110016821F0010101608168D4F8188074
:10815000B8F1806F01F4F81ED4F804A020D1BAF170
:10816000000F15D0BAF5800F1AD1A36B03BB13E033
:10817000604518BF082908D8704518BF6045D1D0A0
:10818000D2E700BFE1680F29BDD90120BDE8F08723
:10819000A36BB3F1805F06D1036843F4805303609F
:1081A0005FEA4A2304D4D4F80C904FF0010C0FE09E
:1081B000D4F80C90B9F1070F08D3056825F4807C3A
:1081C000256D45EA0C054FF0000C04E04FF0000C63
:1081D000056825F480750560BAF1000FE769A26AA9
:1081E00047EA0E07E36B42EA0702A56842EA030288
:1081F0002669676942EA090282604AEA0803626BFB
:10820000616A42EA0302A36B41EA020141EA030107
:10821000226A41EA0601E36C41EA070141EA0201F0
:10822000A26C41EA0301A36D41EA050141EA0201A2
:1082300041EA0301C16009D18168012262F3CC21C6
:1082400081608168022262F34A218160016DBCF184
:10825000000F21F00101016505D1C168626D21F0B7
:1082600000411143C1600020C4F88400012184F85A
:108270008110BDE8F08700002DE9F04FB5B004464D
:1082800002A8B8210025CDE93355CDE93155309507
:10829000F8F729FD43F600012068C4F20001884286
:1082A00056D043F20001C4F20101884240F0DF8061
:1082B0004FF48050029002A84FF00008CDF80C80D7
:1082C000CDF86480FEF7CCFA08B1F9F789FB44F2E7
:1082D000E04040F20044C5F60200C5F6020430ADAD
:1082E0004FF002090169032641F4805101610169DF
:1082F000052701F4805101910199016841F00801BD
:108300000160016801F0080101910199016841F0E3
:10831000020101600068294600F002000190019806
:108320008020309004F50060CDE931983396349781
:10833000FCF72AFE08202946CDE93009204634976B
:10834000CDE93286FCF720FE35B0BDE8F08F00BFE6
:108350004FF48050029002A803951995FEF780FA19
:1083600008B1F9F73DFB44F2E04040F20045C5F6A4
:108370000200C5F6020530AE40F228088168C4F25A
:10838000020841F48041816081684FF0020901F4E4
:10839000804101910199016841F004010160016887
:1083A000002701F0040101910199016841F00201E7
:1083B00001600068314600F002000190019806203B
:1083C000309005F58060CDF8C4904FF0030A3297E5
:1083D0004FF0050BCDF8CCA0CDF8D0B0FCF7D4FD14
:1083E0004FF400503146CDE9300932A880E8800CC6
:1083F0002846FCF7C9FD41F210252720C2F20045AE
:108400004FF48066C5E901072846C5F80080EF6093
:10841000C5E90467C5E90677C5E90877FBF794FA6B
:1084200008B1F9F7DDFAE56708F11800AC6341F22D
:108430008825C2F200452860282068604020C5E9F0
:1084400002072846C5E90467C5E90677C5E9087744
:10845000FBF77AFA08B1F9F7C3FA242005210022C4
:10846000A567AC63FCF750FF2420FCF73DFF35B057
:10847000BDE8F08F0000000043F600010068C4F280
:108480000001884208D140F67870C2F2004040688E
:10849000002808BF70470047704700000000000038
:1084A000704700000000000043F600010068C4F2BD
:1084B0000001884208D140F67870C2F2004000689E
:1084C000002808BF70470047704700000000000008
:1084D00043F600010068C4F20001884208D140F66A
:1084E0007870C2F200408068002808BF70470047DB
:1084F000704700000000000040F20442C5F6000290
:10850000136823EA00000843106070470000000071
:1085100070470000000000007047000000000000ED
:108520007047000000000000B0B590F83C20012A20
:1085300002D10220B0BD00BFD1E9022323F47C5355
:1085400022F4705242EA030548F2FF73D1E900CEEB
:10855000CEF6F0730EEA030203F5006445EA020E5C
:108560000CEA04050C6903F5C05245EA0E052240E9
:108570002A434D692A4303F560550C6B03F5F0431C
:108580002A4023401343026840F2004C42F48065C5
:10859000C4F2010C8C69654540F2000CCEF6FF7CFC
:1085A000CD690CEA044443EA050343EA040318D105
:1085B0004FF6FF7540F2000CCDF60F458C6ACDF6F4
:1085C000F04C03EA050E0D6A0CEA04544B6A44EAC7
:1085D0000E0425F0085523F000532543C96A2B43A8
:1085E0000B430021536480F83C100846B0BD0000E6
:1085F000B0B590F83C20012A4FF0020263D080F819
:108600003D2040F2004C0268C4F2010C42F4806349
:1086100063455368D2F808E002BF23F470034C6846
:1086200023434DF6FF740D68C4F2000423F0700379
:10863000A24243EA0503536014DC40F2FF73C4F224
:1086400000039A4222DD40F60003C4F200039A427E
:108650002ED040F60043C4F200039A4228D041F6DF
:10866000000321E04FF6FF73C4F200039A4213DDCA
:108670000023C4F201039A421AD044F20003C4F268
:1086800001039A4214D0624512D016E0B2F1804F35
:108690000ED040F2004307E04EF20003C4F20003A4
:1086A0009A4205D04EF20043C4F200039A4204D12C
:1086B0002EF080038968194391600022012180F81F
:1086C0003D1080F83C201046B0BD000000000000C6
:1086D00060B310B5044690F83D0028B9002084F836
:1086E0003C00204600F024F8022084F83D00206879
:1086F000211D02F001FF012084F8480084F83E00AB
:1087000084F83F0084F8400084F8410084F8420077
:1087100084F8430084F8440084F8450084F8460057
:1087200084F8470084F83D00002010BD0120704708
:10873000704700000000000090F83D10012923D18F
:10874000022180F83D1001684DF6FF70C4F2000070
:108750008142C86840F00100C86017DC40F2FF7039
:10876000C4F20000814227DD40F60000C4F20000A0
:10877000814233D040F60040C4F2000081422DD047
:1087800041F6000026E000BF012070474FF6FF7061
:10879000C4F20000814215DD0020C4F201008142D4
:1087A0001CD044F20000C4F20100814216D040F215
:1087B0000040C4F201000FE0B1F1804F0ED040F252
:1087C000004007E04EF20000C4F20000814205D0F4
:1087D0004EF20040C4F2000081420BD107228868AB
:1087E000C0F2010202400020062A18BFB2F5803F05
:1087F00000D17047086840F0010008600020704711
:108800007047000000000000F0B581B00446006829
:10881000C768066906EA0705A9071BD468072FD4AD
:10882000280745D4E8065BD4E80772D117F0800723
:1088300018BF16F402507AD1002F18BF16F48070BA
:1088400040F08280680600F18980A80600F19080DF
:1088500001B0F0BD6FF00201016101212177806953
:10886000800703D02046FFF7CBFF05E0204600F04D
:1088700033F9204600F01CFC002020776807CFD594
:1088800020686FF00401016102212177806910F4F2
:10889000407F03D02046FFF7B3FF05E0204600F0FD
:1088A0001BF9204600F004FC002020772807B9D5EA
:1088B00020686FF00801016104212177C0698007F9
:1088C00004D02046FFF79CFF06E000BF204600F0E2
:1088D00003F9204600F0ECFB00202077E806A3D542
:1088E00020686FF01001016108212177C06910F440
:1088F000407F03D02046FFF783FF05E0204600F0CD
:10890000EBF8204600F0D4FB00202077E8073FF486
:108910008DAF20686FF001010161204600F0CCFBB3
:1089200017F0800718BF16F402503FF485AF206897
:108930006FF4025101612046FFF7EEFD002F18BFD2
:1089400016F480703FF47EAF20686FF4807101618F
:108950002046FFF7DDFD68067FF577AF20686FF0F2
:1089600040010161204600F0B3FBA8067FF570AF1F
:1089700020686FF020010161204601B0BDE8F040A1
:10898000FFF7CEBD0000000070B586B041F2FF7267
:108990000068C4F20002002190420591CDE9031164
:1089A000CDE9011136DCB0F1804F5BD040F20041DF
:1089B000C4F20001884240F08D8044F2E04000247F
:1089C000C5F60200C5F6020402250026016841F042
:1089D00001010160016801F0010100910099016845
:1089E00041F002010160006801A900F0020000905E
:1089F00000988020019020460295CDE903660595F8
:108A0000FCF7C2FACDE90155CDE90366059504F5F9
:108A100080605CE041F60001C4F2000188423BD076
:108A20000021C4F20101884254D144F2E040C5F66D
:108A30000200016841F0100101600068002100F0AF
:108A400010000090C5F6020100984FF40850019004
:108A5000022002900020CDE903000120059001F5DD
:108A6000805034E044F2E040C5F60200016841F075
:108A700001010160006800F00100009000980520ED
:108A80000190022002900020CDE903000120059012
:108A90000020C5F602001AE044F2E040C5F60200EC
:108AA000016841F0020101600068002100F002004D
:108AB000009000984FF40040CDE90311002101908F
:108AC000C5F6020102200290059001F5806001A91F
:108AD000FCF75AFA06B070BD7047000000000000B5
:108AE0002DE9F04190F83C30012B03D10220BDE884
:108AF000F08100BF4FEAB202052A31D8DFE812F058
:108B0000060038007600B400DA000001036843F67E
:108B1000FF76C4F201061C6AB3421A6A24F002040A
:108B200022F001021A621A46D3F804E052F818CF74
:108B30008D6844EA0504D1F8008040F3078144F2CF
:108B40000007C4F20107BB4200F00B8144F60007A6
:108B5000C4F20107BB4200F0048144F20047FCE08C
:108B60000121002280F83C200846BDE8F08100BFCA
:108B7000036840F2004E43F48067C4F2010E1C6AA1
:108B800077451A6A24F0200422F010021A621A466D
:108B90005D6852F818CF8E6844EA061407D1CE6893
:108BA0006FF0400724F0C00407EA0616344343F68A
:108BB000FF76D1F80080C4F20106B34240F3EC80A6
:108BC00044F20007C4F20107BB4200F0EC8044F617
:108BD0000007C4F20107BB4200F0E58044F2004701
:108BE000C4F20107BB4200F0DE80E4E0036840F21B
:108BF000004E43F48067C4F2010E1C6A77451A6A7E
:108C000024F4007422F480721A621A465D6852F8E5
:108C10001CCF8E6844EA062407D1CE6840F2FF4795
:108C2000360224F44064BE43344343F6FF76D1F861
:108C30000080C4F20106B34240F3D48044F200073E
:108C4000C4F20107BB4200F0D48044F60007C4F22E
:108C50000107BB4200F0CD8044F20047C4F2010797
:108C6000BB4200F0C680CCE0036843F6FF77C4F255
:108C70000107D3F820C0BB421A6A22F480521A625C
:108C80001A465C6852F81C6F0D68D1F808E040F392
:108C9000CF8044F20007C4F20107BB4200F0D3804A
:108CA00044F60007C4F20107BB4200F0CC8044F256
:108CB0000047C4E0036843F6FF77C4F20107D3F826
:108CC00020C0BB421A6A22F480321A621A465C68DB
:108CD00052F8546F0D68D1F808E040F3D38044F2A5
:108CE0000007C4F20107BB4200F0D78044F600073A
:108CF000C4F20107BB4200F0D08044F20047C8E054
:108D0000036843F6FF77C4F20107D3F820C0BB42E3
:108D10001A6A22F480121A621A465C6852F8546F7A
:108D20000D68D1F808E040F3D98044F20007C4F29E
:108D30000107BB4200F0DD8044F60007C4F20107E2
:108D4000BB4200F0D68044F20047CEE00027C4F2D8
:108D50000107BB4205D040F20047C4F20107BB4205
:108D600005D1CF6824F00C0427F004073C43B3423C
:108D700040F3E28044F20006C4F20106B34200F080
:108D8000E68044F60006C4F20106B34200F0DF803C
:108D900044F20046D7E000BF0027C4F20107BB42FF
:108DA00001D0734507D14F6925F440658E6945EAC6
:108DB000870747EA860548F6FF475D60CFF6FF67FD
:108DC00007EA0C0747EA08279F614F6809699F6314
:108DD0001C629F6947F400679F619F6927F4806761
:108DE0009F61A6E00027C4F20107BB4201D0734592
:108DF00007D14F6925F440558E6945EA071747EAC0
:108E000006154FF68C775D60CFF6FE7707EA0C0704
:108E100047EA0807DF614F680969DF631C62DF69A1
:108E200047F00807DF61DF6927F00407DF61ACE086
:108E30000027C4F20107BB4205D040F20047C4F24C
:108E40000107BB4204D14F6924F4804444EA8714EB
:108E500048F6FF475C60CFF6FF673E402CF40057B2
:108E600046EA0524DC614E6809691E6447EA0E374C
:108E70001F62DF6947F40067DF61DF6927F48067FD
:108E8000DF6156E00027C4F20107BB4205D040F283
:108E90000047C4F20107BB4204D14F6924F4803477
:108EA00044EA07244FF68C775C60CFF6FE770337F1
:108EB0003E402CF4003746EA05045C654E680969BB
:108EC0009E6547EA0E471F625F6D47F008075F65C2
:108ED0005F6D27F004075F6557E000BF0027C4F20D
:108EE0000107BB4205D040F20047C4F20107BB4274
:108EF00004D14F6924F4802444EA872448F6FF47CC
:108F00005C60CFF6FF6707F540773E402CF4001712
:108F100046EA05245C654E680969DE6547EA0E5736
:108F20001F625F6D47F400675F655F6D27F48067C0
:108F30005F65090229E000BF0026C4F20106B342C2
:108F400005D040F20046C4F20106B34206D12EF429
:108F50004077D1E90565374347EA050E4FF68C7532
:108F6000C3F804E0CFF6FE750CEA050747EA0807E8
:108F70009F614F6809695F631C629F6947F008073A
:108F80009F619F6927F004079F611368194311606F
:108F90000021002280F83C200846BDE8F081000056
:108FA00060B310B5044690F83D0028B9002084F85D
:108FB0003C00204600F024F8022084F83D002068A0
:108FC000211D02F099FA012084F8480084F83E003F
:108FD00084F83F0084F8400084F8410084F842009F
:108FE00084F8430084F8440084F8450084F846007F
:108FF00084F8470084F83D00002010BD0120704730
:1090000081B041F2FF710068C4F20001884217DCB0
:10901000B0F1804F2AD040F20041C4F200018842F2
:1090200041D144F2E840C5F60200016841F0020176
:109030000160006800F002000090009801B07047E5
:1090400041F60001C4F2000188421FD00021C4F2A1
:109050000101884227D144F2E840C5F60200816848
:1090600041F001018160806809E000BF44F2E840FE
:10907000C5F60200016841F001010160006800F0DE
:1090800001000090009801B0704700BF44F2E84032
:10909000C5F60200016841F040010160006800F07F
:1090A00040000090009801B07047000000000000F0
:1090B00070470000000000004EF200010068C4F29A
:1090C0000001884218BF7047FCF762B8000000003A
:1090D000704700000000000090F88410012901D1C1
:1090E000022070472421C0F88810026813681168B4
:1090F00023F0005321F0010111600021416613604B
:109100002022C0F8882080F88410084670470000AC
:1091100070470000000000007047000000000000E1
:1091200070B590F88420012A02D1022070BD00BFE2
:109130002422C0F888200268D0F864E0BEF1000F55
:10914000D2F800C0136823F001031360936823F082
:10915000606341EA030191601AD0916840F2AC3E2D
:109160009368C0F6010E5B0F40F2B435C1F342665E
:10917000C0F601051EF80340E95C2301B3FBF1F1E1
:109180001EF80630AE5D1B01B3FBF6F302E000BF34
:1091900001210123A0F86A102021A0F86830C2F84C
:1091A00000C0C0F88810002180F88410084670BD07
:1091B00070B590F88420012A02D1022070BD00BF52
:1091C0002422C0F888200268D0F864E0BEF1000FC5
:1091D000D2F800C0136823F001031360936823F0F2
:1091E000604341EA030191601AD0916840F2AC3EBD
:1091F0009368C0F6010E5B0F40F2B435C1F34266CE
:10920000C0F601051EF80340E95C2301B3FBF1F150
:109210001EF80630AE5D1B01B3FBF6F302E000BFA3
:1092200001210123A0F86A102021A0F86830C2F8BB
:1092300000C0C0F88810002180F88410084670BD76
:1092400070470000000000007047000000000000B0
:1092500045F200010068C4F20001032301F5404219
:10926000904208BF0123401A18BF1846032808BFC0
:10927000704700EBC00040F69871C2F2004101EB6C
:109280008000006900B10047704700000000000046
:10929000B0B50446006840F62F01C2690568114068
:1092A000D0F808E020290BD105F020010EF0805302
:1092B000C91823D0616FD1B32046BDE8B04008473C
:1092C00040F60F010A4219D0012140F22013C1F2E9
:1092D0000001C0F200430EEA010C05EA030111EBA4
:1092E0000C010BD0D10718BF15F4807140F0C68176
:1092F00091070EF0010300F1CD81D4E105EA0203EC
:10930000D906E16E14D5012912D1102101628168BC
:10931000490600F19D80B4F85C10B4F85E20B4F802
:109320005E30002B1CBF891A5FEA01422FD1B0BD0D
:10933000D10240F159811EF4800100F055814FF4B3
:10934000801101622046BDE8B040FFF77DBF00BF3D
:10935000206850E8000F226820F4907042E8000373
:10936000002B1FBF206850E8000F226820F4907087
:109370001CBF42E80003002B12D0206850E8000F09
:10938000226820F4907042E800034BB1206850E856
:10939000000F226820F4907042E80003002BD7D120
:1093A0004FF6FE70CEF6FF70226852E8022F236857
:1093B000024043E80225002D1FBF226852E8022F19
:1093C000236802401CBF43E80225002D10D022680C
:1093D00052E8022F2368024043E8022545B1226883
:1093E00052E8022F2368024043E80225002DDBD11A
:1093F0002020C4F88C000020E0666067206850E8F8
:10940000000F226820F0100042E80003002B1FBF6D
:10941000206850E8000F226820F010001CBF42E8CE
:109420000003002B12D0206850E8000F226820F0C3
:10943000100042E800034BB1206850E8000F22689A
:1094400020F0100042E80003002BD7D189B227E2B8
:10945000D4F8803019684A68B4F85CC091B2002929
:1094600000F01682614580F01382A4F85E20D9696D
:10947000B1F5807F00F0AC8050E8000F216820F447
:10948000807041E80002FAB1206850E8000F2168BE
:1094900020F4807041E80002002A1FBF206850E8D5
:1094A000000F216820F480701CBF41E80002002AF0
:1094B0000AD0206850E8000F216820F4807041E84D
:1094C00000020AB12068D7E7206850E8020F21683F
:1094D00020F0010041E80202002A1FBF206850E886
:1094E000020F216820F001001CBF41E80202002A9F
:1094F00026D0206850E8020F216820F0010041E8E2
:109500000202EAB1206850E8020F216820F0010051
:1095100041E80202002AD7D112E000BF206850E8DB
:10952000020F216820F0400041E80202EAB1206801
:1095300050E8020F216820F0400041E80202A2B189
:10954000206850E8020F216820F0400041E8020244
:10955000002A1FBF206850E8020F216820F0400059
:109560001CBF41E80202002AD8D12020C4F88C0098
:109570000020E066206850E8000F216820F010000D
:1095800041E80002002A1FBF206850E8000F216850
:1095900020F010001CBF41E80002002A12D0206811
:1095A00050E8000F216820F0100041E800024AB1A5
:1095B000206850E8000F216820F0100041E8000208
:1095C000002AD7D1D4F88000F9F7A6F9B4F85CC026
:1095D00002202067B4F85E00ACEB000081B22046A8
:1095E000BDE8B040FFF794BD11060BD505F0800C27
:1095F0000EF4000111EB0C0104D0A16F00297FF4DF
:109600005BAE94E659060BD4100240F17D8115F053
:10961000804000F079812046BDE8B040FFF710BEE1
:1096200050E8000F216820F0400041E80002002AC5
:1096300000F04681206850E8000F216820F04000CB
:1096400041E80002002A1FBF206850E8000F21688F
:1096500020F040001CBF41E80002002A00F03081E9
:10966000206850E8000F216820F0400041E8000227
:10967000002A00F025812068D2E700BF01210162A5
:10968000D4F8901041F00101C4F8901091070EF049
:10969000010308D53BB102210162D4F8901041F0DA
:1096A0000401C4F89010510708D53BB104210162B0
:1096B000D4F8901041F00201C4F8901011070CD5B5
:1096C00005F0200151EA0C0107D008210162D4F80D
:1096D000901041F00801C4F8901011050BD515F059
:1096E000806108D04FF400610162D4F8901041F01D
:1096F0002001C4F89010D4F8901000293FF417AE60
:1097000012F020010AD005F020010EF080528918D5
:1097100004D0616F11B1204688472068D4F89010BA
:10972000826802F0400201F02801891800F0C08030
:1097300050E8000F216820F4907041E80002FAB16F
:10974000206850E8000F216820F4907041E8000282
:10975000002A1FBF206850E8000F216820F4907095
:109760001CBF41E80002002A0AD0206850E8000F20
:10977000216820F4907041E800020AB12068D7E720
:109780004FF6FE70CEF6FF70216851E8021F226886
:10979000014042E80213002B1FBF216851E8021F5D
:1097A000226801401CBF42E80213002B10D0216840
:1097B00051E8021F2268014042E8021343B12168C8
:1097C00051E8021F2268014042E80213002BDBD15E
:1097D000E06E012828D100BF206850E8000F216802
:1097E00020F0100041E80002002A1FBF206850E866
:1097F000000F216820F010001CBF41E80002002A81
:1098000012D0206850E8000F216820F0100041E8D5
:1098100000024AB1206850E8000F216820F01000D3
:1098200041E80002002AD7D12020C4F88C00002192
:10983000E16620686167816849065FD550E8020FDC
:10984000216820F0400041E80202002A42D020684E
:1098500050E8020F216820F0400041E80202002A8F
:109860001FBF206850E8020F216820F040001CBF95
:1098700041E80202002A2DD0206850E8020F21683A
:1098800020F0400041E8020222B32068D6E700BF82
:109890008C457FF44CADD869B0F5807F7FF447AD3F
:1098A000022020672046BDE8B040FFF731BC00BF72
:1098B0002046FFF7CDFC0020C4F89000B0BD00BFEB
:1098C0002020C4F888000020A0672046BDE8B040F2
:1098D00000F0AABBD4F8800080B14BF68131C0F60D
:1098E00000010165F9F7B4FA00283FF420ADD4F87F
:1098F0008000016DBDE8B040084700BF2046BDE8CC
:10990000B040FFF7A5BC00BFD0017FF510ADB5F1A9
:10991000FF3FC8BFB0BD2046BDE8B040FFF7FCBB6D
:1099200010B5E0B10446D0F8880028B9002084F8CA
:109930008400204600F028F82420C4F8880020681D
:10994000A16A0268002922F00101016002D02046CC
:1099500001F0EAFF204602F0F7FA012802D10120C7
:1099600010BD00BF2068416821F4904141608168CA
:1099700021F02A018160016841F001010160204667
:10998000BDE8104002F040B82DE9F043B5B0002129
:109990000446CDE93311CDE93111309102A8B82147
:1099A000F7F7A1F947F2FF712068C4F2000188427D
:1099B00000F3808044F20041C4F20001884200F0CC
:1099C000CF8044F60001C4F20001884200F0FA8022
:1099D00045F20001C4F20001884240F0EA8102A889
:1099E000002703974FF00208CDF808801F97FCF777
:1099F00037FF08B1F7F7F4FF44F2E04040F60045C6
:109A0000C5F60200C5F6020530AE4FF008098168C0
:109A100041F480118160816801F480110191019904
:109A2000016841F004010160016801F00401019145
:109A30000199016841F0080101600068314600F0B9
:109A40000800019001984FF48050CDE93008A5F549
:109A50008060CDF8D090CDE93277FBF795FA0420FD
:109A60003146CDE930082846CDF8D090CDE932779F
:109A7000FBF78AFA41F200355820C2F20045C4F2E1
:109A8000020028604120C5E901074FF48060EF60C3
:109A9000C5E904072846C5E90677C5E90877F9F757
:109AA00053FF08B1F7F79CFFC4F88050AC6335242E
:109AB00077E100BF47F60001C4F20001884200F0E0
:109AC000CD8041F20001C4F20101884200F0FA8029
:109AD00041F60041C4F20101884240F06A81012050
:109AE000029002A8002603962096FCF7B9FE08B162
:109AF000F7F776FF44F2E04030ADC5F602000227EA
:109B0000016941F080010161016901F08001019169
:109B10000199016841F0100101600068294600F0D8
:109B200010000190019804203090349040F60040DD
:109B3000C5F60200339600F580642046CDE9317603
:109B4000FBF722FA08202946CDE930070B20349094
:109B50002046CDE93266FBF717FA9C2421E100BFCD
:109B600002A800240394022502951F94FCF778FEB6
:109B700008B1F7F735FF44F2E040C5F6020081680E
:109B800041F400318160816801F400310191019953
:109B9000016841F008010160006830A900F0080088
:109BA000019001987020CDE930050720349040F6EF
:109BB0000040C5F60200CDE93244FBF7E5F9262462
:109BC000EFE000BF02A8002603964FF00208CDF890
:109BD00008801F96FCF744FE08B1F7F701FF44F236
:109BE000E04040F60044C5F60200C5F6020430AD80
:109BF0000727816841F480218160816801F4802118
:109C000001910199016841F002010160016801F0D0
:109C1000020101910199016841F0080101600068A9
:109C2000294600F00800019001984FF48040CDE9EA
:109C30003008A4F500603497CDE93266FBF7A4F94B
:109C40004FF440702946CDE9300820463497CDE9DD
:109C50003266FBF799F92724A3E000BF02A800248D
:109C60000394022502951F94FCF7FAFD08B1F7F75B
:109C7000B7FE44F2E040C5F60200816841F0804141
:109C80008160816801F0804101910199016841F092
:109C900010010160006840F6004100F010000190E2
:109CA000C5F6020101984FF4C070CDE930050720D8
:109CB000349001F5806030A9CDE93244FBF764F9B6
:109CC00052246EE00120029002A8002603962096FE
:109CD000FCF7C6FD08B1F7F783FE44F2E04040F21E
:109CE0005808C5F60200C4F20208016941F01001EB
:109CF0000161016901F0100101910199016841F0D0
:109D000001010160006840F6004100F0010001908F
:109D1000C5F6020101984FF4C060309002203396DE
:109D2000CDE9310607203490A1F5406030A9FBF75A
:109D30002BF941F2F03508F11800C2F200454FF45A
:109D4000806728602A2068604020C5E9020628460E
:109D5000C5E90476C5E90666C5E90866F9F7F4FDC4
:109D600008B1F7F73DFEE56708F13000AC6341F25A
:109D70007835C2F200452860292068600020C5E9D6
:109D80000200C5E90470C5E90600C5E908002846D7
:109D9000F9F7DAFD08B1F7F723FEC4F88050AC6399
:109DA0002524052100222046FBF7AEFA2046FBF7CA
:109DB0009BFA35B0BDE8F083B0B50446D0F88C000E
:109DC000202807D115460A460120002918BF002D7A
:109DD00002D1B0BD0220B0BD4FF0000CC4F86CC081
:109DE00040F600402168C5F60000814234D0486842
:109DF000000231D551E8000FD4F800E040F0806057
:109E00004EE8000141B300BF206850E8000F216810
:109E100040F0806041E80003002B1FBF206850E83D
:109E2000000F216840F080601CBF41E80003002B58
:109E300012D0206850E8000F216840F0806041E8AF
:109E400000034BB1206850E8000F216840F08060AB
:109E500041E80003002BD7D1A2652220A4F85C5072
:109E6000C4F890C0C4F88C00D4F88000F0B14BF670
:109E7000A9514BF62973C0F60001C0F60003C0E9F2
:109E80000F134BF691310023C0F60001C164216825
:109E9000036524312B46FAF79BF838B11020C4F83B
:109EA00090002020C4F88C000120B0BD206938B398
:109EB000206850E8000F216840F4807041E80002FB
:109EC000002A1FBF206850E8000F216840F480700E
:109ED0001CBF41E80002002A12D0206850E8000FA1
:109EE000216840F4807041E800024AB1206850E8DF
:109EF000000F216840F4807041E80002002AD7D1A9
:109F0000206850E8020F216840F0010041E8020299
:109F1000002A1FBF206850E8020F216840F00100AE
:109F20001CBF41E80202002A1DD0206850E8020F41
:109F3000216840F0010041E80202A2B1206850E827
:109F4000020F216840F0010041E80202002AD7D147
:109F500009E000BF206850E8020F216840F040008F
:109F600041E80202EAB1206850E8020F216840F09F
:109F7000400041E80202A2B1206850E8020F2168C7
:109F800040F0400041E80202002A1FBF206850E86C
:109F9000020F216840F040001CBF41E80202002A85
:109FA000D8D10020B0BD000045F200010068C4F225
:109FB0000001032301F54042904208BF0123401AEB
:109FC00018BF1846032808BF704700EBC00040F6D2
:109FD0009871C2F2004101EB8000C06800B10047F7
:109FE000704700000000000045F200010068C4F264
:109FF0000001032301F54042904208BF0123401AAB
:10A0000018BF1846032808BF704700EBC00040F691
:10A010009871C2F2004101EB8000806800B10047F6
:10A02000704700000000000045F200010068C4F223
:10A030000001032301F54042904208BF0123401A6A
:10A0400018BF1846032808BF704700EBC00040F651
:10A050009871C2F2004101EB8000406800B10047F6
:10A060007047000000000000FEE700000000000054
:10A07000F0B583B00027002818BF002902D1384668
:10A0800003B0F0BDB5EE400AF1EE10FA06DA02298F
:10A0900006DB01272D23037003E000BF002702E049
:10A0A0000027B1EE400A22EAE2740125062CA8BF7F
:10A0B0000624012A05DB012CC8BF2546022C33DA11
:10A0C0000A25B6EEC01A02EE105AB6EE003A002388
:10A0D00030EE411AB8EEC22ABDEEC00A01EE023AD5
:10A0E000BDEEC31A11EE106AB542D8BF0123012A92
:10A0F00010EE102A134409DB751B3844B8BF3546EF
:10A10000C91B009417A2019506E000BF40F2F1328E
:10A110003844C91BC0F60102F6F7FCF90028C8BF95
:10A120000744384603B0F0BDAB1E032B0AD86425A4
:10A13000DFE803F002040E12C3E700BF4FF47A75A4
:10A14000BFE700BF44F24025C0F20F05B9E700BFEA
:10A1500042F21075B5E700BF48F2A065C0F20105F4
:10A16000AFE700BF25642E25302A64000000000000
:10A170002DE9F04700284FF0FE0449D08A46002917
:10A1800046D040F21008C2F2004898F8005A3F2D1D
:10A1900004D9FF2460B2BDE8F08700BF06469146AF
:10A1A0006DB140F210072C46C2F2004738463146E6
:10A1B000F6F7EEFD80B3013C07F12807F6D1D8F899
:10A1C0000C0D28B14FF0FF3105F0B2FA98F8005AA3
:10A1D00005EB85001F22314608EBC000F6F7AAFD0B
:10A1E00098F8001A002401EB8100013188F8001A68
:10A1F00008EBC002D8F80C0DD477C2F820A0C2F842
:10A20000249028B1002100220023002404F0E4FF60
:10A2100060B2BDE8F08700BFFD2460B2BDE8F08702
:10A2200081B080B581B0039303AB009302F0D8FEF8
:10A2300001B0BDE8804001B07047000000000000A0
:10A2400010B58CB06846242100240B94CDE9094454
:10A25000F6F749FD41F2400042F20001C2F200402F
:10A26000C4F20201042201604FF41011C0E901148C
:10A270000121016142614FF4807202830222C261B6
:10A28000032280F82040C0E90A440263C0E90F4479
:10A2900080F844408164F8F713F908B1F7F7A0FBA0
:10A2A00041F2400009A9C2F200400994F7F7FCFB13
:10A2B00008B1F7F795FB102040F2FF71C1F2C00022
:10A2C00000900620019004200290CDE903100020A8
:10A2D00005908DF8210041F24000C2F2004069462D
:10A2E000F7F73EFC08B1F7F77BFB00206946C4F6A0
:10A2F000B87000900C20019041F24000C2F2004082
:10A30000F7F72EFC08B1F7F76BFB0CB010BD00009F
:10A31000B0B58AB041F2B00046F20001C2F200408E
:10A3200000240994C5F60201CDE90744CDE90544AE
:10A33000C0E9001408210461C0E902140425456144
:10A3400004830121C16180F82040C0E90F4480F8F6
:10A350004440846480F83840C0E90A44C0E90C44B1
:10A36000F8F7AEF808B1F7F73BFB002001A9CCF2F3
:10A370002130019006200694CDE9020440F2FF70DE
:10A380000894CDE9040541F2B000C2F20040F7F7AD
:10A39000E7FB08B1F7F724FB0AB0B0BD00000000EE
:10A3A00080B582B044F2E0400022C5F602000168A8
:10A3B00041F4001101600068052100F400100190D3
:10A3C00001988120FAF7A0FF812002B0BDE880400B
:10A3D000FAF78ABF0000000080B582B044F2D8408E
:10A3E0000022C5F60200016841F001010160006829
:10A3F000052100F00100019001980B20FAF784FF7D
:10A400000B20FAF771FF0C2005210022FAF77CFFE0
:10A410000C20FAF769FF0D2005210022FAF774FFDE
:10A420000D20FAF761FF0E2005210022FAF76CFFDC
:10A430000E20FAF759FF0F2005210022FAF764FFDA
:10A440000F20FAF751FF102005210022FAF75CFFD8
:10A45000102002B0BDE88040FAF746BF00000000BF
:10A4600080B541F268404AF20001C2F20040C4F2F5
:10A4700000010122182301600021C0E902110282BB
:10A480008174C0E905320323C163C0E90732C0E922
:10A490000922C0E90B22C0E90D1220220264042324
:10A4A000C0E91131C0E91331C0E91531C0E9171213
:10A4B000C0E91913FAF730F9002808BF80BDBDE8DC
:10A4C0008040F7F78DBA000080B541F208504AF29B
:10A4D0000041C2F20040C4F20001012218230160D1
:10A4E0000021C0E9021102828174C0E90532032310
:10A4F000C163C0E90732C0E90922C0E90B2240F27A
:10A500000643C0E90D32202202640423C0E911325F
:10A51000C0E91331C0E91531C0E91712C0E91913B8
:10A52000FAF7FAF8002808BF80BDBDE88040F7F7C9
:10A5300057BA00000000000080B541F2A8504DF26B
:10A540000041C2F20040C4F2000101221823016060
:10A550000021C0E9021102828174C0E9053203239F
:10A56000C263C0E90732C0E90922C0E90B2240F604
:10A570001203C0E90D32202202640423C0E9113223
:10A58000C0E91331C0E91531C0E91712C0E9191348
:10A59000FAF7C2F8002808BF80BDBDE88040F7F791
:10A5A0001FBA00000000000080B54BF2F92040F215
:10A5B000BC32C0F60000C0F60102002103F028F909
:10A5C00040F6E07C4BF27163C2F2004CC0F600032F
:10A5D00040F264320021C0F60102CCF800001846B7
:10A5E000BDE8804003F014B92DE9F04F87B044F284
:10A5F000E0400027C5F60200069740F2004901221C
:10A600000168C5F6020941F010010160016809F511
:10A61000806601F0100101910199016841F0040187
:10A62000016001684FF0010B01F0040101910199F3
:10A63000016841F080010160016801F08001019131
:10A640000199016841F001010160016801F0010117
:10A6500001910199016841F002010160016801F076
:10A66000020101910199016841F00801016000684F
:10A670004EF2290100F00800019001983046FAF7E7
:10A6800077FD09F540644FF4004100222046FAF7B7
:10A690006FFD4FF4406100224846FAF769FD4FF420
:10A6A000805101224846FAF763FD09F500684FF42E
:10A6B000806100224046FAF75BFD02AD4FF4604036
:10A6C000CDE9020B30462946CDE90477FAF75CFC68
:10A6D00029202946CDE9020B304604974FF0030AA2
:10A6E000CDF814A0FAF750FC4FF4A05002904FF4AC
:10A6F00088102946CDE903072046FAF745FC204695
:10A7000029464FF40046CDE9026BCDE90477FAF70C
:10A710003BFC4FF440602946CDE9020B4846CDE9A9
:10A720000477FAF731FC4FF480502946CDE9020B4B
:10A730004846CDE904BAFAF727FC4FF48060294671
:10A74000CDE9020B4046CDE90477FAF71DFCA9F5E7
:10A7500080644FF4807002900220CDE90307204608
:10A760002946CDE90577FAF70FFC20462946CDE9C1
:10A7700002670497FAF708FC4FF000600021FDF72C
:10A78000BBFE282005210022FAF7BEFD2820FAF79B
:10A79000ABFD07B0BDE8F08F10B586B041F2486060
:10A7A00045F20002C2F200400021CDE90411CDE9DA
:10A7B0000211CDE90011C5F2002202600124C1603E
:10A7C000C0E9014120220163C0E90424C0E9061167
:10A7D000C0E90814C0E90A110822C163C0E90D21CB
:10A7E000FBF70EF908B1F7F7FBF84FF001100390F3
:10A7F00041F248606946C2F2004041F2883200945A
:10A800000294FAF7C1FD08B1F7F7EAF806B010BDF7
:10A8100010B541F6883443F20000C2F20044C4F29D
:10A8200001004FF0806120604FF4800060604FF4C1
:10A830000030A0600720E0604FF000702061002031
:10A840006061A1614FF08051C4E90710C4E90900BB
:10A85000E0624FF08040606304F138002421F6F795
:10A8600042FA2046FDF734FC002808BF10BDBDE8C1
:10A870001040F7F7B5B8000010B541F6104443F6A4
:10A880000000C2F20044C4F20000072120604FF42F
:10A89000800060600020A060E1604FF000712161E5
:10A8A0004FF0807161614FF08061A1614FF0804194
:10A8B000C4E90710C4E90900E06204F138006163EB
:10A8C0002421F6F710FA2046FDF702FC002808BF05
:10A8D00010BDBDE81040F7F783B80000000000008D
:10A8E00010B58AB041F6E44041F60001C2F20040E2
:10A8F00000240894C4F200010694CDE90444CDE993
:10A900000244CDE9004401601721C0E9011440F27E
:10A91000CF718461C0E90314FEF742FB08B1F7F779
:10A920005FF841F6E44007A9C2F200400794099499
:10A93000FDF75EFE08B1F7F753F8602000900020A5
:10A940000490CDE9010041F6E4406946C2F20040BE
:10A950000422FEF7C5F808B1F7F742F841F6E440E3
:10A96000C2F20040FEF710F80AB010BD000000006F
:10A9700010B598B001A8342100241494CDE91244F4
:10A98000CDE91044CDE90E44F6F7ADF941F6984013
:10A990000021C2F20040C4F2010101601821C0E9A7
:10A9A000011442F21071C0E90314C0E90544FEF736
:10A9B000F7FA08B1F7F714F841F6984015A9C2F272
:10A9C00000401794CDE91544FDF712FE08B1F7F7E2
:10A9D00007F860200E9041F288300F90002014900C
:10A9E000CDE91000CDE9120041F698400EA9C2F25F
:10A9F00000400022FEF774F808B1F6F7F1FF41F6C7
:10AA000098400EA9C2F200400822FEF769F808B18A
:10AA1000F6F7E6FF00200590CDE90300CDE901003F
:10AA20004FF400510990CDE906104FF000710D90E0
:10AA3000CDE90A1041F6984001A9C2F20040FDF7A5
:10AA400073FD08B1F6F7CCFF41F69840C2F2004022
:10AA5000FDF79AFF18B010BD10B58AB041F630501E
:10AA60000024C2F20040089406944FF08041CDE9E2
:10AA70000444CDE90244CDE9004401601821C0E955
:10AA8000011442F210718461C0E90314FEF788FAE0
:10AA900008B1F6F7A5FF41F6305007A9C2F2004011
:10AAA00007940994FDF7A4FD08B1F6F799FF60201B
:10AAB000009041F28830019000200290049041F60D
:10AAC0003050C2F2004069460022FEF709F808B192
:10AAD000F6F786FF41F630506946C2F20040082280
:10AAE000FDF7FEFF08B1F6F77BFF41F63050C2F2EA
:10AAF0000040FDF749FF0AB010BD00000000000053
:10AB000010B58AB041F6C85040F20041C2F2004090
:10AB100000240894C4F200010694CDE90444CDE970
:10AB20000244CDE9004401601721C0E9011442F25A
:10AB30000F71C0E9031480218161FEF731FA08B179
:10AB4000F6F74EFF41F6C85007A9C2F2004007943D
:10AB50000994FDF74DFD08B1F6F742FF6020009023
:10AB600000200490CDE9010041F6C8506946C2F2C8
:10AB700000400422FDF7B4FF08B1F6F731FF41F6BB
:10AB8000C8506946C2F200400C22FDF7A9FF08B187
:10AB9000F6F726FF41F6C850C2F20040FDF7F4FE7A
:10ABA0000AB010BD0000000080B542F2640045F21A
:10ABB0000001C2F2004048F2A062C4F20001C0F2FB
:10ABC0000102C0E900124FF4805181604FF400513E
:10ABD000C1604FF480610161042141610021816203
:10ABE000C0E90611C0E90811FEF79AFE08B1F6F7B0
:10ABF000F7FE42F264000021C2F20040FEF7D8FAEC
:10AC000008B1F6F7EDFE42F264000021C2F2004006
:10AC1000FEF786FA08B1F6F7E3FE42F26400C2F2EC
:10AC20000040FEF759FA002808BF80BDBDE880400B
:10AC3000F6F7D6BE0000000080B542F2F80047F6F5
:10AC40000001C2F20040C4F200010C2201604FF486
:10AC5000612141600021C0E902110161C0E90521C3
:10AC6000C0E90711C0E90911FEF75AFE08B1F6F76D
:10AC7000B7FE42F2F8000021C2F20040FEF798FA57
:10AC800008B1F6F7ADFE42F2F8000021C2F2004032
:10AC9000FEF746FA08B1F6F7A3FE42F2F800C2F258
:10ACA0000040FEF719FA002808BF80BDBDE88040CB
:10ACB000F6F796BE0000000080B541F6A86041F6A8
:10ACC0000041C2F20040C4F201010C2201604FF4C5
:10ACD000612141600021C0E902110161C0E9052143
:10ACE000C0E90711C0E90911FEF71AFE08B1F6F72D
:10ACF00077FE41F6A8600021C2F20040FEF758FA44
:10AD000008B1F6F76DFE41F6A8600021C2F20040DE
:10AD1000FEF706FA08B1F6F763FE41F6A860C2F244
:10AD20000040FEF7D9F9002808BF80BDBDE880408B
:10AD3000F6F756BE0000000080B541F6146041F2FF
:10AD40000001C2F20040C4F201010C2201604FF484
:10AD5000612141600021C0E902110161C0E90521C2
:10AD6000C0E90711C0E90911FEF7DAFD08B1F6F7ED
:10AD700037FE41F614600021C2F20040FEF718FAD7
:10AD800008B1F6F72DFE41F614600021C2F2004032
:10AD9000FEF7C6F908B1F6F723FE41F61460C2F2D9
:10ADA0000040FEF799F9002808BF80BDBDE880404B
:10ADB000F6F716BE0000000080B541F63C7044F284
:10ADC0000041C2F20040C4F200010C2200230160E5
:10ADD0004FF4612141600021C0E902110161C0E925
:10ADE0000521C0E90711C0E9091100210022FCF783
:10ADF000DFFF08B1F6F7F4FD41F63C700021C2F226
:10AE00000040FEF7D5F908B1F6F7EAFD41F63C70CF
:10AE10000021C2F20040FEF783F908B1F6F7E0FD29
:10AE200041F63C70C2F20040FEF756F9002808BF18
:10AE300080BDBDE88040F6F7D3BD000000000000F3
:10AE400080B541F6D07044F60001C2F20040C4F271
:10AE500000010C22002301604FF4612141600021B8
:10AE6000C0E902110161C0E90521C0E90711C0E98B
:10AE7000091100210022FCF79BFF08B1F6F7B0FD95
:10AE800041F6D0700021C2F20040FEF791F908B1FE
:10AE9000F6F7A6FD41F6D0700021C2F20040FEF7A1
:10AEA0003FF908B1F6F79CFD41F6D070C2F20040C0
:10AEB000FEF712F9002808BF80BDBDE88040F6F714
:10AEC0008FBD00000000000080B541F2A4600021A9
:10AED000C2F20040C4F204010160092101714FF483
:10AEE0000071C1800221C0F809100021C1810174E4
:10AEF000FAF7E6FE002808BF80BDBDE88040F6F7FF
:10AF00006FBD000000000000FEE700000000000030
:10AF1000FEE700000000000000000000000000004C
:10AF2000EFF30980BFF36F8F154B1A681EF0100FF7
:10AF300008BF20ED108A20E9F04F10602DE90900CC
:10AF40004FF0500080F31188BFF34F8FBFF36F8F26
:10AF500003F006FF4FF0000080F31188BDE8090000
:10AF600019680868B0E8F04F1EF0100F08BFB0EC89
:10AF7000108A80F30988BFF36F8F704700BF00BF4E
:10AF8000880D002400000000F0B581B044F22C4789
:10AF9000C5F6020757F8042C02F00302032A03D176
:10AFA000012001B0F0BD00BF054657F82C0C0C463F
:10AFB00020F0806047F82C0CFAF7E2F8064600BF54
:10AFC00057F82C0C000105D5FAF7DAF8801B022897
:10AFD000F6D964E057F8040CEE6895E80E0020F40A
:10AFE0007C30012C40EA0130A2F101016FF35F21B6
:10AFF0004FF47E4202EB432247F8040C92B24FF02A
:10B00000FE4302EB01004FF4FE012A6901EB064109
:10B0100001F4FE0103EB0262084402F0FE41084421
:10B02000F8603868696920F0C00040EA01003860C3
:10B030003868A96920F0200040EA010038603868CB
:10B040004FF6F87120F0100038603869EA6920EA9C
:10B0500001004FF4001140EAC2003861386808BFAF
:10B060004FF4801140F01000002C386008BF4FF4FE
:10B07000002138680843386057F82C0C40F0806095
:10B0800047F82C0CFAF77CF8044600BF57F82C0C54
:10B09000000107D4FAF774F8001B0328F6D3032045
:10B0A00001B0F0BD002001B0F0BD000000000000C4
:10B0B000F0B581B044F22C47C5F6020757F8042CCE
:10B0C00002F00302032A03D1012001B0F0BD00BF4A
:10B0D000054657F82C0C0C4620F0805047F82C0CF5
:10B0E000FAF74EF8064600BF57F82C0C800005D53D
:10B0F000FAF746F8801B0228F6D964E057F8040CEA
:10B10000EE6895E80E0020F07C70012C40EA0150BA
:10B11000A2F101016FF35F214FF47E4202EB432263
:10B1200047F8040C92B24FF0FE4302EB01004FF4DB
:10B13000FE012A6901EB064101F4FE0103EB026204
:10B14000084402F0FE41084478613868696920F4D7
:10B15000406040EA010038603868A96920F4007056
:10B1600040EA0100386038684FF6F87120F48070CA
:10B170003860B869EA6920EA01004FF0807140EA5E
:10B18000C200B861386808BF4FF4000140F4807015
:10B19000002C386008BF4FF48001386808433860DD
:10B1A00057F82C0C40F0805047F82C0CF9F7E8FFCA
:10B1B000044600BF57F82C0C800007D4F9F7E0FFD5
:10B1C000001B0328F6D3032001B0F0BD002001B01E
:10B1D000F0BD00000000000041F61040C2F2004047
:10B1E000FCF73EBE00000000016840F26F32D1F86B
:10B1F00014C08B6943F008038B618B6943F0100323
:10B200008B610B6823F001030B600B6923EA0202D8
:10B210000A618A6822F440428A6090F881305FEACD
:10B220008C620BD5042B09D0D0F8842042F0800228
:10B23000C0F884208A6942F020028A6190F8813047
:10B240005FEA4C620BD5032B09D0D0F8842042F082
:10B250000402C0F884208A6942F040028A615FEAF1
:10B260008C5209D45FEACC5213D40021A0F86210AA
:10B27000A0F86A10704700BFD0F8842042F00102A5
:10B28000C0F884208A6942F400728A615FEACC5275
:10B29000EBD5D0F8842042F00802C0F884208A69F7
:10B2A00042F480728A610021A0F86210A0F86A104E
:10B2B0007047000000000000806B0021A0F86A10B9
:10B2C000A0F86210012180F88110FCF7B5BD0000E4
:10B2D000074B19680868B0E8F04F80F30988BFF39E
:10B2E0006F8F4FF0000080F31188704700BF00BFE0
:10B2F000880D00240000000080B502F085FABDE84A
:10B30000804002F0D5BA000080B54EF21000CEF2B7
:10B310000000006804F0ECFC012808BF80BDBDE817
:10B32000804003F041BE0000B0B59CB044F6180464
:10B33000022000251195CDE90F55CDE90D55CDE938
:10B340000B550895C5F60204CDE90655CDE904551F
:10B35000CDE902550195FAF72BFE0095206820F4FF
:10B3600040402060206800F440400090009800BFFA
:10B37000206880045FBF20685FEA804020685FEA41
:10B38000804002D420688004F2D5232009904FF435
:10B3900080300A9001200C900F9002212822402436
:10B3A000CDE9152004200D94CDE917010C2019904A
:10B3B00009A81491CDE912110025CDE91A55FCF721
:10B3C0006BFA28B1EFF3108072B600BFFEE700BF42
:10B3D0003F20019003200321CDE9020508200694B7
:10B3E000CDE904044FF48060CDE9070401A8FBF720
:10B3F0008FFF28B1EFF3108072B600BFFEE700BFE9
:10B40000002000214FF48022FCF7F6F91CB0B0BDFB
:10B410004EF6885042F2000CCEF20000C5F2002C2D
:10B42000026842F470020260DCF8000000F00F00D5
:10B43000062806D8DCF80000072262F30300CCF8E7
:10B44000000044F200404EF67F51C5F60200CEF6F1
:10B45000F621026842F001020260002202610368E4
:10B4600019400160DCF80010090706D5DCF800106F
:10B47000072363F30301CCF8001040F2002182613E
:10B48000C261C0F20221026281620021C0F2FF119A
:10B49000C16240F28021C0F2011101634263816305
:10B4A000C26301644264016821F480210160026684
:10B4B000D0F8D410C90448BF7047D0F8D41043F274
:10B4C000D20241F48051C0F8D41044F20001C5F218
:10B4D00000210A60D0F8D41021F48051C0F8D410B3
:10B4E000704700000000000041F67C50C2F20040AE
:10B4F000FDF78AB90000000010B540F6FF32D0F821
:10B5000000E0C4F20002904210DCB0F1804F1ED087
:10B5100040F20043C4F20003984218D040F6000302
:10B52000C4F20003984212D016E000BF40F6004378
:10B53000C4F2000398420AD040F20043C4F201036F
:10B54000984204D00023C4F20103984204D12EF0A3
:10B5500070024B6843EA020E4EF2FF3343F6FF7C63
:10B56000C4F20003C4F2010C984213DD60452BDCE9
:10B570004EF20043C4F20003984242D00023C4F2CA
:10B58000010398423DD040F20043C4F201039842C7
:10B5900037D03BE040F2FF73C4F20003984227DD4E
:10B5A00040F60003C4F2000398422AD040F600435C
:10B5B000C4F20003984224D04EF20003C4F2000308
:10B5C00098421ED022E000BF44F20003C4F20103FF
:10B5D000984216D044F60003C4F20103984210D0FA
:10B5E00044F20043C4F2010398420AD00EE000BFC7
:10B5F000B0F1804F05D040F20043C4F200039842FE
:10B6000004D12EF44072CB6843EA020E4B696045C8
:10B610000A688C68C462826212DD44F20002C4F2DD
:10B620000102904217D044F60002C4F20102904297
:10B6300011D044F20042C4F2010290420BD00CE05F
:10B640000022C4F20102904205D040F20042C4F24E
:10B650000102904201D109690163016841F00401CE
:10B660000160012141612EF080011943016010BD8C
:10B6700010B501F0C1FE4BF2097040F28832C0F6FD
:10B680000000C0F60102002102F0C2F842F2DC64C0
:10B690000A21C2F2004400222060022001F008FFCB
:10B6A000A06202200321002201F002FFA064022018
:10B6B0002421002201F0FCFEE06202201821002279
:10B6C00001F0F6FE206302201021002201F0F0FEBE
:10B6D000606302204FF4FB61002201F0E9FEA063E9
:10B6E00002200C21002201F0E3FE206402200C2144
:10B6F000002201F0DDFE606401F0B6FE02F084F885
:10B70000BDE8104002F0D4B882B040F20018C0F298
:10B71000010801F055FE00EE100A4FF4FA709FED9B
:10B720006E1BB8EE400B80EE010BBCEEC00B10EEB2
:10B73000106A01F011FE01F03BFE40F6E874054688
:10B74000C2F200442046F5F7E7FF4DF6E90264A097
:10B75000C0F600022146FEF70BFD019605EB060B35
:10B7600040F6E066B9EE048AB1EE049AC2F20046F1
:10B7700042F2DC6506F1040AC2F2004500279FEDA3
:10B780005BAA08F581399FED58BA9FED59CA12E0BE
:10B79000F070A86C86F80280771C01F029FFA86C75
:10B7A00000220023394601F0CFFE584601F0E4FDA7
:10B7B0000198002783442046F6F7E6F81420F6F7B0
:10B7C000F3F818B12046F5F7DBFF02E02046F5F765
:10B7D000C7FF94F83900032818BF022812D194F843
:10B7E000380002284FF0030038BF022094ED0B1AF6
:10B7F00094ED0C0A21EE081A307120EE090A86ED4C
:10B80000021A04E0B0EE4B0A01283771B760286CC9
:10B8100086ED030A01F0ECFE286C0022002351465D
:10B8200001F092FE94ED0D0A86F82470B4EE4A0AF7
:10B83000F1EE10FA09DBB4EE4C0AF1EE10FA0CDD71
:10B84000307850B1012086F824000020B4EE4A0A76
:10B85000F1EE10FAB8BF0120307094F83900374685
:10B8600080FE0B0A4FF000080138C0B2C100032867
:10B870004FF0000038BF29FA01F007F8100FD4E9A3
:10B8800009017960E16AC7E90201286B87ED040AC2
:10B8900001F0AEFE286B00220023394601F054FE71
:10B8A00094F838002278411E07F80F2CC8B20228FD
:10B8B0004FF000003FF66CAF4FF4FF6000EAC100AC
:10B8C00040F20011C0F2010121FA00F84FF480713A
:10B8D00021FA00F05CE700BF0000000000407F405C
:10B8E000647231360000000000000000666666BF2A
:10B8F0009A9999BE0000000010B542F26404C2F2A9
:10B9000000442046FDF7C4FC2046BDE81040F5F792
:10B910006BBC00000000000042F2F800C2F20040E0
:10B92000FDF7B6BC00000000816A0A070CD4CA0704
:10B9300015D18A071ED44A0727D4CA0630D48A06EE
:10B9400039D44A0655D541E00268D0F838C053686A
:10B9500023F4004343EA0C035360CA07E9D00268AA
:10B96000D0F82CC0536823F4003343EA0C0353602F
:10B970008A07E0D50268D0F830C0536823F48033DA
:10B9800043EA0C0353604A07D7D50268D0F834C0A5
:10B99000536823F4802343EA0C035360CA06CED5D0
:10B9A0000268D0F83CC0936823F4805343EA0C0348
:10B9B00093608A06C5D50268D0F840C0936823F426
:10B9C000005343EA0C0393604A0612D50268D0F88C
:10B9D00044C0BCF5801F536823F4801343EA0C0372
:10B9E000536006D1536823F4C00C836C43EA0C0304
:10B9F0005360090658BF70470168C06C4A6822F45A
:10BA00000022104348607047B0B582B00446002061
:10BA1000C4F89000F9F7B4FB216805460A681207DC
:10BA200037D54FF4001100226FF07E400090204681
:10BA30002B4600F0A9FD58B3206850E8000F21689C
:10BA400020F0800041E80002002A1FBF206850E873
:10BA5000000F216820F080001CBF41E80002002A8E
:10BA600012D0206850E8000F216820F0800041E8E3
:10BA700000024AB1206850E8000F216820F08000E1
:10BA800041E80002002AD7D12020C4F8880063E0F2
:10BA900021680868400765D54FF4800100226FF0E7
:10BAA0007E40009020462B4600F06EFD002859D0C5
:10BAB000206850E8000F216820F4907041E80002EF
:10BAC000002A1FBF206850E8000F216820F4907002
:10BAD0001CBF41E80002002A26D0206850E8000F71
:10BAE000216820F4907041E80002EAB1206850E833
:10BAF000000F216820F4907041E80002002AD7D19D
:10BB000012E000BF206850E8020F216820F0010019
:10BB100041E80202EAB1206850E8020F216820F0F3
:10BB2000010041E80202A2B1206850E8020F21683A
:10BB300020F0010041E80202002A1FBF206850E8FF
:10BB4000020F216820F001001CBF41E80202002A18
:10BB5000D8D12020C4F88C000320002184F8841060
:10BB600002B0B0BD2020C4F88800C4F88C000020CA
:10BB7000E0662067002184F8841002B0B0BD0000A8
:10BB8000806B0021A0F85E10FDF762BB0000000092
:10BB9000806B0268D0F88810D0F88CC02129936897
:10BBA00063D113F0800360D00023A0F8563052E830
:10BBB000002F036822F0C00243E80021E1B300BF78
:10BBC000016851E8001F026821F0C00142E800133B
:10BBD000002B1FBF016851E8001F026821F0C0015F
:10BBE0001CBF42E80013002B26D0016851E8001F5B
:10BBF000026821F0C00142E80013EBB1016851E88E
:10BC0000001F026821F0C00142E80013002BD7D1C9
:10BC100012E000BF016851E8021F026821F4000130
:10BC200042E80213EBB1016851E8021F026821F4F7
:10BC3000000142E80213A3B1016851E8021F026843
:10BC400021F4000142E80213002B1FBF016851E8F4
:10BC5000021F026821F400011CBF42E80213002BFE
:10BC6000D8D12021C0F888100268BCF1220F916859
:10BC700040F0908011F0400100F08C800021A0F88D
:10BC80005E1052E8001F00BF026821F4907142E884
:10BC900000130BB3016851E8001F026821F4907192
:10BCA00042E80013002B1FBF016851E8001F026823
:10BCB00021F490711CBF42E80013002B0CD00168E6
:10BCC00051E8001F026821F4907142E800131BB193
:10BCD000016851E8001FD7E74FF6FE7CCEF6FF7CE7
:10BCE000026852E8022F036802EA0C0243E80221CC
:10BCF00000291FBF016851E8021F026801EA0C0118
:10BD00001CBF42E80213002B12D0016851E8021F49
:10BD1000026801EA0C0142E802134BB1016851E8E4
:10BD2000021F026801EA0C0142E80213002BD7D17E
:10BD3000C16E012928D100BF016851E8001F0268C7
:10BD400021F0100142E80013002B1FBF016851E8E9
:10BD5000001F026821F010011CBF42E80013002BF5
:10BD600012D0016851E8001F026821F0100142E87A
:10BD700000134BB1016851E8001F026821F0100167
:10BD800042E80013002BD7D12021C0F88C100021ED
:10BD9000C1664167D0F8901041F01001C0F89010D2
:10BDA000FDF756BA00000000C169806BB1F5807FD5
:10BDB00000F0AC800021A0F85E1000BF016851E8DF
:10BDC000001F026821F4807142E80013002B1FBF9E
:10BDD000016851E8001F026821F480711CBF42E82D
:10BDE0000013002B12D0016851E8001F026821F4F3
:10BDF000807142E800134BB1016851E8001F0268EE
:10BE000021F4807142E80013002BD7D1016851E87A
:10BE1000021F026821F0010142E80213002B1FBF3C
:10BE2000016851E8021F026821F001011CBF42E8CD
:10BE30000213002B26D0016851E8021F026821F08E
:10BE4000010142E80213EBB1016851E8021F0268E8
:10BE500021F0010142E80213002BD7D112E000BF0C
:10BE6000016851E8021F026821F0400142E8021314
:10BE7000EBB1016851E8021F026821F0400142E87D
:10BE80000213A3B1016851E8021F026821F04001CA
:10BE900042E80213002B1FBF016851E8021F02682D
:10BEA00021F040011CBF42E80213002BD8D1202111
:10BEB000C0F88C10C16E012928D100BF016851E87B
:10BEC000001F026821F0100142E80013002B1FBF81
:10BED000016851E8001F026821F010011CBF42E810
:10BEE0000013002B12D0016851E8001F026821F0F6
:10BEF000100142E800134BB1016851E8001F0268CD
:10BF000021F0100142E80013002BD7D10021016776
:10BF1000C16E012904D1B0F85C10FDF7F9B800BF7B
:10BF2000FEF742B800000000806B01210167C16E7E
:10BF3000012905D1B0F85C104908FDF7E9B800BF48
:10BF4000FEF752B80000000070B584B004460068E7
:10BF500004F1080340F6004EE669C5F6000E0ECB6C
:10BF6000194363690B4346F6F3110568CCF6FF717C
:10BF7000334329401943016041684FF2FF4321F4E4
:10BF80004051704541EA02014160A269C1F2FF13CC
:10BF90001CBF216A0A43816844F2544C1940C5F61B
:10BFA000020C1143816047F6FF32C16AC4F20002FD
:10BFB00021F00F01656A90424FF0800341EA0501CC
:10BFC000C1622BDD41F2FF71C4F20101884251DCF4
:10BFD00047F60041C4F20001884200F08B8041F234
:10BFE0000001C4F20101884200F0948041F2004156
:10BFF000C4F20101884240F00E81DCF80010C1F368
:10C00000C202052A00F2EE800123DFE812F00401EB
:10C01000E300F300FB000301AB0100BF44F6FF3176
:10C02000C4F20001884247DD44F60041C4F2000139
:10C03000884200F07F8045F20001C4F2000188428E
:10C0400000F0888047F60001C4F20001884240F009
:10C05000E280DCF8001001F00702052A00F2C2803D
:10C060000023DFE812F0D800B700C700CF00D700E8
:10C070007F0100BF41F60001C4F20101884200F0D7
:10C08000798041F60041C4F20101884200F08280CB
:10C09000704540F0C080DCF8041001F00702052A6A
:10C0A00000F2A0800223DFE812F0B6009500A500A0
:10C0B000AD00B5005D0100BF44F20041C4F20001D3
:10C0C000884200F0778044F60001C4F20001884203
:10C0D00040F0A180DCF8001001F00702052A00F210
:10C0E00081800023DFE812F09700760086008E0042
:10C0F00096003E01DCF8001001F00702052A00F26C
:10C1000071800023DFE812F08700660076007E0071
:10C1100086002E01DCF80010C1F3C202052A00F2ED
:10C1200061800123DFE812F07700560066006E00A0
:10C1300076001E01DCF8001001F00702052A00F26B
:10C1400051800023DFE812F06700460056005E00D1
:10C1500066000E01DCF8001001F00702052A41D844
:10C160000023DFE812F05800370047004F00570067
:10C17000FF0000BFDCF80010C1F3C202052A31D86D
:10C180000123DFE812F04800270037003F00470096
:10C19000EF0000BFDCF80010C1F3C202052A21D86D
:10C1A0000123DFE812F03800170027002F003700C6
:10C1B000DF0000BFDCF8001001F00702052A11D8EB
:10C1C0000023DFE812F02800070017001F002700F7
:10C1D000CF0000BF0423704540F60010C0F23D00C0
:10C1E00020D1C7E08023704540F60010C0F23D002A
:10C1F00018D1BFE00823704540F60010C0F23D00A2
:10C2000010D1B7E01023704540F60010C0F23D0099
:10C2100008D1AFE02023704540F60010C0F23D0089
:10C2200000F0A880B6F5004F40F04E80402B4FF054
:10C23000010100F29E81DFE813F0410017019C012B
:10C240009C011D019C019C019C0125019C019C01FC
:10C250009C019C019C019C019C012D019C019C0165
:10C260009C019C019C019C019C019C019C019C01E6
:10C270009C019C019C019C019C013D019C019C0135
:10C280009C019C019C019C019C019C019C019C01C6
:10C290009C019C019C019C019C019C019C019C01B6
:10C2A0009C019C019C019C019C019C019C019C01A6
:10C2B0009C019C019C019C019C013B01FBF7B0F996
:10C2C000002840F0D480E3E0402B4FF0010100F261
:10C2D0005081DFE813F041000F014E014E011501BE
:10C2E0004E014E014E011D014E014E014E014E0107
:10C2F0004E014E014E0125014E014E014E014E01EF
:10C300004E014E014E014E014E014E014E014E01B5
:10C310004E014E014E0135014E014E014E014E01BE
:10C320004E014E014E014E014E014E014E014E0195
:10C330004E014E014E014E014E014E014E014E0185
:10C340004E014E014E014E014E014E014E014E0175
:10C350004E014E014E013301FBF762F9002840F017
:10C36000CC80DBE04023704540F60010C0F23D0079
:10C370007FF458AF9A1E01211E2A27D8DFE812F059
:10C380002000F9002C00F900F900F9003400F90050
:10C39000F900F900F900F900F900F9003C00F90092
:10C3A000F900F900F900F900F900F900F900F900C5
:10C3B000F900F900F900F900F900F900490000BF9F
:10C3C000F9F72AFEB0B1656A23E000BF402B40F0C8
:10C3D000D0804FF400401CE001A8F9F7C9FE029894
:10C3E0000028F0D106E000BF01A8F9F759FF029834
:10C3F0000028E8D10021BCE05CF8540C800649F22A
:10C400000000C0F2D03004D55CF8541CC1F3C10167
:10C41000C84040F24C316268C0F6010131F8151095
:10C42000B0FBF1F002EB420188424FF00101C0F095
:10C43000A0801303984200F29C80010E00230002AA
:10C4400010EB520041F10001F3F7ECFF4FF6FF4211
:10C45000A0F54071C0F20F02914203D82168C86074
:10C46000002186E0012184E0FBF70AF980B1656ACA
:10C4700020E000BF01A8F9F77BFE02980028F6D162
:10C4800006E000BF01A8F9F70BFF02980028EED1E3
:10C4900000216EE05CF8540C800649F20000C0F206
:10C4A000D03007D55CF8541CC1F3C101C84001E08D
:10C4B0004FF4004040F24C31C0F6010131F8151044
:10C4C000B0FBF1F061684A0802EB40004FF6EF72F2
:10C4D000B0FBF1F0A0F11001914209D84FF6F071D4
:10C4E00022680140C0F342000844D060002140E0CF
:10C4F00001213EE0FBF7C4F880B1656A20E000BF8F
:10C5000001A8F9F735FE02980028F6D106E000BF31
:10C5100001A8F9F7C5FE02980028EED1002128E015
:10C520005CF8540C800649F20000C0F2D03007D508
:10C530005CF8541CC1F3C101C84001E04FF4004055
:10C5400040F24C316268C0F6010131F81510B0FBC1
:10C55000F1F000EB5200B0FBF2F0A0F110014FF649
:10C56000EF72914204D82168C860002101E000BF49
:10C5700001214FF00110A0660020C4E91D0008460B
:10C5800004B070BD000000002DE9F0418046006855
:10C590000D46C7693940491BB1FA81F149099142F9
:10C5A00025D1069C34B31646611C29D1C1692940A6
:10C5B000491BB1FA81F14909B14218D1C169294039
:10C5C000491BB1FA81F14909B14201BFC169294052
:10C5D000491BB1FA81F104BF4909B14207D1C169D0
:10C5E0002940491BB1FA81F14909B142DED000204E
:10C5F000BDE8F081F8F7C4FD0320BDE8F08100BF7D
:10C600001F4607E0C0692840401BB0FA80F040098F
:10C61000B042ECD1F8F7B4FDC01BA04244D8D8F822
:10C62000000001684907EDD5402D18BF802DE9D0E5
:10C63000C16909073CD4C1690905E3D54FF400611C
:10C64000016250E8000FD8F8001020F4907041E823
:10C650000002002A62D0D8F8000050E8000FD8F895
:10C66000001020F4907041E80002002A1FBFD8F8A3
:10C67000000050E8000FD8F8001020F490701CBFA4
:10C6800041E80002002A49D0D8F8000050E8000F25
:10C69000D8F8001020F4907041E80002002A3DD044
:10C6A000D8F80000CDE700BF0320BDE8F08100BF4F
:10C6B0000821016250E8000FD8F8001020F49070B3
:10C6C00041E80002002A00F09D80D8F8000050E800
:10C6D000000FD8F8001020F4907041E80002002A02
:10C6E0001FBFD8F8000050E8000FD8F8001020F461
:10C6F00090701CBF41E80002002A00F08380D8F847
:10C70000000050E8000FD8F8001020F4907041E8C5
:10C710000002002A76D0D8F80000CBE74FF6FE7072
:10C72000CEF6FF70D8F8001051E8021FD8F80020AC
:10C73000014042E80213002B1FBFD8F8001051E857
:10C74000021FD8F8002001401CBF42E80213002B52
:10C7500014D0D8F8001051E8021FD8F8002001408A
:10C7600042E8021353B1D8F8001051E8021FD8F87C
:10C770000020014042E80213002BD3D1D8F86C000E
:10C7800001282FD1D8F8000050E8000FD8F8001089
:10C7900020F0100041E80002002A1FBFD8F8000076
:10C7A00050E8000FD8F8001020F010001CBF41E83E
:10C7B0000002002A16D0D8F8000050E8000FD8F880
:10C7C000001020F0100041E800025AB1D8F8000033
:10C7D00050E8000FD8F8001020F0100041E80002E7
:10C7E000002ACFD12020C8F88C000021C8F86C1096
:10C7F000C8F87410C8F89000032088F88410BDE8C9
:10C80000F08100BF4FF6FE70CEF6FF70D8F8001032
:10C8100051E8021FD8F80020014042E80213002B23
:10C820001FBFD8F8001051E8021FD8F800200140BF
:10C830001CBF42E80213002B14D0D8F8001051E8B6
:10C84000021FD8F80020014042E8021353B1D8F883
:10C85000001051E8021FD8F80020014042E80213FE
:10C86000002BD3D1D8F86C0001282FD1D8F80000C4
:10C8700050E8000FD8F8001020F0100041E8000246
:10C88000002A1FBFD8F8000050E8000FD8F80010A9
:10C8900020F010001CBF41E80002002A16D0D8F892
:10C8A000000050E8000FD8F8001020F0100041E818
:10C8B00000025AB1D8F8000050E8000FD8F8001074
:10C8C00020F0100041E80002002ACFD12020C8F853
:10C8D0008C000020C8F86C00C8F874000821C8F863
:10C8E000901088F884000120BDE8F081000000006D
:10C8F00041F6A860C2F20040FCF7CABC000000008C
:10C9000010B541F61464C2F200442046FCF7C0FCA6
:10C910002046BDE81040F4F767BC000000000000AE
:10C9200041F63C70C2F20040FCF7B2BC00000000CF
:10C9300041F6D070C2F20040FCF7AABC0000000033
:10C9400082B002F47F42B2F5807F40F08180836B39
:10C950004FF6BF7223F480338363DDF808C0C368E9
:10C96000CFF6BD721A40C2605FFA8CF2C368012A2A
:10C9700023F44012C26003D1C26842F48012C26044
:10C9800000220092009A01320092009AB2F1706F78
:10C9900000F2C4800269B2F1FF3F21DD009A01324A
:10C9A0000092009AB2F1706F00F2B8800269002A1A
:10C9B00016D4009A01320092009AB2F1706F00F220
:10C9C000AD800269002A0BD4009A01320092009ACD
:10C9D000B2F1706F00F2A2800269B2F1FF3FD1DCC8
:10C9E00000220092026942F001020261009A0132C3
:10C9F0000092009AB2F1706F00F290800269D20743
:10CA00001ED0009A01320092009AB2F1706F00F2CB
:10CA100085800269D20713D0009A01320092009AF1
:10CA2000B2F1706F7AD80269D20709D0009A013248
:10CA30000092009AB2F1706F70D80269D207D5D116
:10CA4000002201F47F01B1F5803F40F08D807AE053
:10CA5000C26842F04002C26000220192019A013293
:10CA60000192019AB2F1706F60D80269B2F1FF3F92
:10CA70001EDD019A01320192019AB2F1706F55D810
:10CA80000269002A14D4019A01320192019AB2F18A
:10CA9000706F4BD80269002A0AD4019A01320192C0
:10CAA000019AB2F1706F41D80269B2F1FF3FD5DC53
:10CAB00000220192026942F001020261019A0132F0
:10CAC0000192019AB2F1706F30D80269D2071DD07D
:10CAD000019A01320192019AB2F1706F26D802696F
:10CAE000D20713D0019A01320192019AB2F1706F0C
:10CAF0001CD80269D20709D0019A01320192019A29
:10CB0000B2F1706F12D80269D207D7D1002213F4A4
:10CB10007F4F836B0FD143F480330EE0032201F487
:10CB20007F01B1F5803F1FD10DE000BF032213F458
:10CB30007F4F836BEFD023F48033836301F47F0155
:10CB4000B1F5803F10D1C16D89B2C165C16D41F0B1
:10CB5000007141F0F771C165816841F006018160A3
:10CB6000816841F020018160104602B070470000EA
:10CB70000146D0F8000E20F00300C1F8000E00209E
:10CB8000D1F8042842F00202C1F8042870470000DE
:10CB90002DE9F04F82B0C3F3074C0027BCF1000F22
:10CBA000C0F80471C0F80871C0F80C71C0F81071B9
:10CBB000C0F81471C0F81871C0F81C71C0F8207169
:10CBC000C0F82471C0F82871C0F82C71C0F8307119
:10CBD000C0F83471C0F83871C0F83C7104D000F16D
:10CBE00038034FF400170FE0D0F80438802743F0E3
:10CBF0000203C0F80438836B23F4001383630368D3
:10CC000043F04003036003461E68374302F47F4647
:10CC10001F60B6F5807F4FF00003C0F8003E07D1DB
:10CC2000B3EB116FD0F8003806D043F0010303E0F6
:10CC3000D0F8003843F00303C0F800380023019314
:10CC4000019B01330193019BB3F1706F52D80369CB
:10CC5000B3F1FF3F1EDD019B01330193019BB3F153
:10CC6000706F47D80369002B14D4019B01330193E3
:10CC7000019BB3F1706F3DD80369002B0AD4019B6F
:10CC800001330193019BB3F1706F33D80369B3F1A2
:10CC9000FF3FD5DC002301934FF484630361019BC4
:10CCA00001330193019BB3F1706F23D803699B0695
:10CCB0001DD5019B01330193019BB3F1706F19D80E
:10CCC00003699B0613D5019B01330193019BB3F1CB
:10CCD000706F0FD803699B0609D5019B013301933F
:10CCE000019BB3F1706F05D803699B06D7D44FF051
:10CCF000000E01E04FF0010E00230093009B013372
:10CD00000093009BB3F1706F50D80369B3F1FF3FFC
:10CD10001EDD009B01330093009BB3F1706F45D87B
:10CD20000369002B14D4009B01330093009BB3F1E3
:10CD3000706F3BD80369002B0AD4009B013300932A
:10CD4000009BB3F1706F31D80369B3F1FF3FD5DCBD
:10CD50000023009310230361009B01330093009B89
:10CD6000B3F1706F22D80369DB0621D5009B013334
:10CD70000093009BB3F1706F18D80369DB0617D5D9
:10CD8000009B01330093009BB3F1706F0ED80369D1
:10CD9000DB060DD5009B01330093009BB3F1706F50
:10CDA00004D80369DB06D7D402E000BF4FF0010EC0
:10CDB0005FFA81FA4FF00009BAF1000FC0F810983D
:10CDC000C0F81498C0F81C984AD0D0F800394FF039
:10CDD0000068BAF1010F4FF67F3B08EA1313C0F861
:10CDE0000039C0F81099C0F808B916D0CAF1000788
:10CDF00000F512654FF09043002400BF2E68013704
:10CE000003EAE6762E602C617E1CC5F808B005F1B9
:10CE10002005F3D1BAF1000F22D0D0F8003BBAF1CF
:10CE2000010F08EA13134FF00008C0F8003BC0F8E8
:10CE3000108BC0F808BB13D0CAF1000400F53266AD
:10CE40004FF090434FF67F373568013403EAE575BC
:10CE50003560C6F81080651CB76006F12006F3D176
:10CE6000D0F8103811F47F0F23F48073C0F8103815
:10CE7000C0F818906FF08041416103D1816941F0A1
:10CE80001001816143F600038169C8F23C0312F48A
:10CE90007F0F41EA0301816103D0816941F00801FC
:10CEA0008161BCF1010F05D1816941F0804141F000
:10CEB00004018161704602B0BDE8F08F00000000FF
:10CEC00001468268002022F001028A60704700005B
:10CED000B0B50446C06820F0C040E060A1B10129AF
:10CEE0002AD1E06840F00050E060002005460A20AA
:10CEF000F7F742FABD2D05F10A00616916D811F065
:10CF00000101F3D012E000BFE06840F08040E06033
:10CF1000002000BF05460A20F7F72EFABD2D05F1C7
:10CF20000A00616902D811F00101F3D1C838B0FAE2
:10CF300080F04009B0BD00BF0120B0BD000000007E
:10CF4000FEE7000000000000704700000000000045
:10CF50002DE9F041B0B140F688550446C2F20045D3
:10CF60002868A04218D001F0F3FA6669EF69D5F895
:10CF7000208001F015FB0220BE4218BF46450FD1AC
:10CF8000BDE8F0814FF0500080F31188BFF36F8F40
:10CF9000BFF34F8FFEE700BF0020BDE8F08100BF68
:10CFA00005F1540086420BD0012005F14001002E0E
:10CFB00008BF04208E4208BF0420BDE8F08100BFF6
:10CFC000A06A00281CBF0220BDE8F08194F85C1024
:10CFD0000320012908BF0220BDE8F0810000000005
:10CFE0002DE9F04F81B0814600284FF0000003D0BA
:10CFF000002918BF002A03D101B0BDE8F08F00BF9F
:10D000004E1E4C4600F02D811D4613784C46002BD9
:10D0100000F027814FF0250B4C46701E002700BF03
:10D02000252B04EB070802F1010A0BD19AF8003016
:10D03000252B15D188F800B00232B84207F1010162
:10D0400008D10DE1524688F80030B84207F10101DD
:10D0500000F0068113780F46002BE1D100E100BFFC
:10D060002E2B3FD192461AF8023FA3F13001092935
:10D070003AD802F1030A002202EB820103EB4101DC
:10D080009AF80030A3F130020A2AA1F1300233D21B
:10D0900002EB820103EB41019AF80130A3F1300267
:10D0A000092AA1F1300221D802EB820103EB4101F0
:10D0B0009AF80230A3F13002092AA1F1300219D8FE
:10D0C00002EB820103EB41019AF803300AF1040AF2
:10D0D000A3F130020A2AA1F13002CDD3AAF1010A4C
:10D0E0000AE000BF02220AE0002208E00AF1010A79
:10D0F00002E000BF0AF1020A052A00DD0622A3F1C0
:10D100005801F61B202900F27D80DFE801F01D7B2D
:10D110007B7B7B7B7B7B7B7B7B25117B2B7B7B11D9
:10D120007B7B397B7B7B7B7B7B5F7B6B7B7B730040
:10D1300040F2F13255F8043B40463146C0F6010258
:10D14000F3F7E8F97EE000BF55F8043B404631466E
:10D150004EA2F3F7DFF975E055F8040B88F80000EC
:10D1600001206FE0E81D314620F0070000F10805BE
:10D1700090ED000B4046B7EEC00BFCF779FF61E085
:10D18000544614F8010FA0F15801202900F24A80FA
:10D19000DFE801F0124848484848484848484848AD
:10D1A0004A484848484A48484848484848484848FB
:10D1B00048504848120000BF78282EA22CA055F8ED
:10D1C000043B08BF02464046314638E055F8043B70
:10D1D0002BA0002B314608BF034640462AA2F3F796
:10D1E00099F92FE055F8043B4046314629A2F3F760
:10D1F00091F927E055F8043B4046314624A2F3F765
:10D2000089F91FE0B84208F1010188F800B003D1A4
:10D2100000200026884615E09AF8000008F1020870
:10D22000023E087000200DE055F8043B40463146B0
:10D2300012A204E055F8043B404631460EA2F3F733
:10D2400069F9A2460028C4BF361A8044444646B154
:10D250001AF8013F5246002B7FF4DFAE01E000BF19
:10D260000C4400202070A4EB090001B0BDE8F08F51
:10D27000256C7800256C5800256C7500256C6400C1
:10D28000286E756C6C29000025730000255800007D
:10D290002578000025750000002070470000000080
:10D2A000AEB0F7F785FFFEF73FF86C46902104F12A
:10D2B0002800F3F718FD002001904FF400210091A1
:10D2C0000221029110220990CDE90321CDE9051137
:10D2D000C0212890CDE907102046F9F7C1FA28B1FE
:10D2E000EFF3108072B600BFFEE700BFFDF77CF9D8
:10D2F000FDF772F8FDF754F8FCF7A2FFFDF7F0FA1E
:10D30000FDF786FAFDF7B8FAFDF7FAFBFDF714FD15
:10D31000FDF752FDFDF794FDFDF78EFCFDF7CCFC0B
:10D32000FDF79EF8FDF7D0F8FDF706F9FDF720FBB5
:10D33000FDF792FBFDF730FAFDF736FCFCF7E8FF4E
:10D34000FDF7C2FD00F040F8FDF72EF900F06CF893
:10D35000FEE7000000000000EFF3058100291CBF7C
:10D360006FF00500704728B180B501F075FA002014
:10D3700080BD00BF0020704710B582B0EFF305817B
:10D3800021B16FF0050002B010BD00BF044602F0ED
:10D39000BFFC211A0190012906DB01A801F09CFACB
:10D3A000002002B010BD00BF6FF0030002B010BD3E
:10D3B000EFF3058010B102F0B3BC00BF02F0A8BCCF
:10D3C0004FF47A7070470000EFF3058000281CBF0F
:10D3D0006FF00500704740F67470C2F200400168BB
:10D3E00000291CBF4FF0FF30704701210160002071
:10D3F000704700000000000080B5EFF305800028B2
:10D400001CBF6FF0050080BD02F072FC30B1022835
:10D4100006D101F09DFC002080BD00BF012080BD31
:10D420004FF0FF3080BD000010B5EFF3058018B15C
:10D430006FF00504204610BD40F67470C2F2004043
:10D44000016801290CD14EF61F510024CEF20001D3
:10D450000C700221016001F0FFFB204610BD00BFEF
:10D460004FF0FF34204610BD10B5EFF3058018B122
:10D470006FF00504204610BD02F03AFC02280FD0E0
:10D4800090B902F015FE01284FF001040ED002F011
:10D490002FFC002808BF4FF0FF34204610BD00BF0E
:10D4A0000024204610BD00BF4FF0FF34204610BDC1
:10D4B00070B582B0154600240029EFF3058218BF2D
:10D4C000002803D1204602B070BD00BF002AF9D168
:10D4D000B5B1AB68EA681BB3502A26D32A6922B3D8
:10D4E00001FB00F66C69B4424FF00004EAD30094EB
:10D4F00001F0BAFD06460028E4D02C6807E000BF22
:10D500000022002401F068FD0028DBD006463046EA
:10D51000214601F015F93446204602B070BD00BF27
:10D520001AB92A690AB96A6922B10024204602B0F0
:10D5300070BD00BF0022002401F04EFD0646002809
:10D54000DBD1BFE700000000B0B582B0B0FA80F2D6
:10D55000EFF30585B1FA81F452096409002D1D46E7
:10D5600042EA04020AD0002D18BF01252A430BD03D
:10D570006FF00304204602B0B0BD00BFF2B16FF0FF
:10D580000304204602B0B0BD0022019201AA00238C
:10D5900001F042FF012821D1019828B34EF6045032
:10D5A0004FF08051CEF2000000240160BFF34F8F96
:10D5B000BFF36F8F204602B0B0BD00BF00232A46E4
:10D5C000002401F009FE0128D4D06FF00104002DE1
:10D5D00008BF6FF00204204602B0B0BD6FF0020435
:10D5E000204602B0B0BD00BF0024204602B0B0BD4E
:10D5F00010B5EFF3058119B16FF00504204610BD99
:10D6000030B10021002401F09FFD204610BD00BF75
:10D610006FF00304204610BDB0B584B050B3B1F133
:10D62000FF3F27DD04464FF0FF300390EFF3058006
:10D6300030B30122002302A8009020460025029565
:10D6400002F0B2FA03AB002100222046009502F05E
:10D65000ABFA029850B14EF604504FF08051CEF222
:10D6600000000160BFF34F8FBFF36F8F039804B0CA
:10D67000B0BD00BF6FF003000390039804B0B0BDCD
:10D6800001220023204602F0FFF903AB0021002213
:10D69000204602F0F9F9039804B0B0BD0000000084
:10D6A0002DE9F04F81B0EFF305832BB16FF0050743
:10D6B000384601B0BDE8F08F8246002836D4554682
:10D6C00016460C46880748BF002502F021FB6FF084
:10D6D000010B002E08BF6FF0020BE10780462BD133
:10D6E000002E51D0E946002703E000BF5F46002C22
:10D6F000DED0002029464A46334602F0A1FB04460C
:10D700000128F3D107EA0A00009941EA000717EA65
:10D710000A0FCDD102F0FCFAA0EB0800361A4FF048
:10D72000000038BF0646002CE3D1C1E76FF00307C5
:10D73000384601B0BDE8F08F002E41D0E946002701
:10D7400003E000BF5F46002CB2D0002029464A46C5
:10D75000334602F075FB04460128F3D107EA0A00BC
:10D76000009941EA000707EA0A005045A0D002F0FC
:10D77000CFFAA0EB0800361A4FF0000038BF06467B
:10D78000002CE2D194E700BF00206C460646002042
:10D7900000232946224602F053FB68B3012858466D
:10D7A000F4D106EA0A00009941EA000717EA0A0FD5
:10D7B00008BF6FF00207384601B0BDE8F08F00BF28
:10D7C00000206C460646002000232946224602F02F
:10D7D00037FB88B101285846F4D106EA0A000099BF
:10D7E00041EA000707EA0A00504518BF6FF0020738
:10D7F000384601B0BDE8F08F5F46384601B0BDE85D
:10D80000F08F00000000000002F06ABA0000000083
:10D81000F0B585B08C4600230493EFF3058140B149
:10D8200039B94AB19469002C08BF1824382C13D98F
:10D830000023184605B0F0BD0021802318249AB2B9
:10D8400004AB01936346009402F0AEF8012829D19D
:10D85000049B184605B0F0BD1179C90722D156695D
:10D8600095684FEA960E002E734608BF8023116814
:10D87000D7689DB1602F15D3002E4FF00003D8D08C
:10D880001269002AD5D0CDE900427246634602955E
:10D8900002F0BAF80346184605B0F0BD17B9126990
:10D8A000002ACCD00023184605B0F0BD00000000CF
:10D8B00010B5EFF3058100291CBF6FF0050010BD06
:10D8C000044638B12046FFF743FB042806D16FF029
:10D8D000020010BD6FF0030010BD00BF204601F034
:10D8E00063F8002010BD00002DE9F04F93B090F8D0
:10D8F00000C090ED090A90ED0A1AB7EEC00A90ED4B
:10D900000B2A90ED0C3A90ED0D4A90F8394090F8C2
:10D910003850B0F93C70B0F93A60B0F93E8090F8F8
:10D9200040900FF2500E90F841A014A3B0F842B00E
:10D9300008460AA9BCF1000F944640F2F432B7EE53
:10D94000C44AC0F6010208BF734681E8F007614689
:10D95000B7EEC11AB7EEC22ACDF844B0B7EEC33A5B
:10D960008DEC080B8DED084BFCF75AFC13B0BDE8AD
:10D97000F08F00BF4F66666C696E65004F6E6C6914
:10D980006E650000000000002DE9F041044600F043
:10D99000DFFD40F6885642F27C25C2F20046C2F214
:10D9A0000045F0680130F060306858B130690028F7
:10D9B00040F007813068E16AC06A884298BF3460ED
:10D9C000FFE000BF3460F068012840F0FA8028468C
:10D9D00000F05EFD05F1140000F05AFD05F128008D
:10D9E00000F056FD05F13C0000F052FD05F150003D
:10D9F00000F04EFD05F1640000F04AFD05F17800ED
:10DA000000F046FD05F18C0000F042FD05F1A0009C
:10DA100000F03EFD05F1B40000F03AFD05F1C8004C
:10DA200000F036FD05F1DC0000F032FD05F1F000FC
:10DA300000F02EFD05F5827000F02AFD05F58C70D2
:10DA400000F026FD05F5967000F022FD05F5A070AA
:10DA500000F01EFD05F5AA7000F01AFD05F5B47082
:10DA600000F016FD05F5BE7000F012FD05F5C8705A
:10DA700000F00EFD05F5D27000F00AFD05F5DC7032
:10DA800000F006FD05F5E67000F002FD05F5F0700A
:10DA900000F0FEFC05F5FA7000F0FAFC05F50270E6
:10DAA00000F0F6FC05F5077000F0F2FC05F50C70CF
:10DAB00000F0EEFC05F5117000F0EAFC05F51670BB
:10DAC00000F0E6FC05F51B7000F0E2FC05F52070A7
:10DAD00000F0DEFC05F5257000F0DAFC05F52A7093
:10DAE00000F0D6FC05F52F7000F0D2FC05F534707F
:10DAF00000F0CEFC05F5397000F0CAFC05F53E706B
:10DB000000F0C6FC05F5437000F0C2FC05F5487056
:10DB100000F0BEFC05F54D7000F0BAFC05F5527042
:10DB200000F0B6FC05F5577000F0B2FC05F55C702E
:10DB300000F0AEFC05F5617000F0AAFC05F566701A
:10DB400000F0A6FC05F56B7000F0A2FC05F5707006
:10DB500000F09EFC05F5757000F09AFC05F57A70F2
:10DB600000F096FC05F57F7000F092FC05F58260F0
:10DB700000F08EFC05F2244000F08AFC05F5876079
:10DB800000F086FC05F24C4000F082FC40F608787C
:10DB9000C2F20048404600F07BFC08F1140738460A
:10DBA00000F076FC06F1680000F072FC06F140001F
:10DBB00000F06EFC06F1540000F06AFCC6F81C8010
:10DBC00037627068716A421CE06A726088426264FF
:10DBD00088BF706200EB8000211D05EB800000F023
:10DBE0009BFC00F0DDFC306988B13068E16AC06AF6
:10DBF000884228BFBDE8F0814EF604504FF08051B6
:10DC0000CEF200000160BFF34F8FBFF36F8FBDE80E
:10DC1000F08100000000000040F6885542F27C26AA
:10DC20004EF60458C2F20045C2F20046CEF2000899
:10DC30004FF0805703E000BF204600F0C9FCA86801
:10DC4000D0B100F085FCE86CC468201D00F0E8FB52
:10DC5000E8680138E860A8680138A86000F0A0FC16
:10DC600094F85D000228EAD00128E5D070B9206B55
:10DC700000F0AEFCE0E700BF30680228DFD3C8F850
:10DC80000070BFF34F8FBFF36F8FD8E74FF0500096
:10DC900080F31188BFF36F8FBFF34F8FFEE7000053
:10DCA0002DE9F0470A9C16460F468246206B9100EC
:10DCB000A5229846DDE90859F2F7EBFF206B002F0B
:10DCC00000EB8600A0F1040020F0070654D038785D
:10DCD00084F83400387800284AD0787884F8350001
:10DCE0007878002844D0B87884F83600B8780028CE
:10DCF0003ED0F87884F83700F878C8B3387984F8DB
:10DD000038003879A0B3787984F83900787978B315
:10DD1000B87984F83A00B87950B3F87984F83B00C0
:10DD2000F87928B3387A84F83C00387A00B3787AE6
:10DD300084F83D00787AD8B1B87A84F83E00B87A91
:10DD4000B0B1F87A84F83F00F87A88B1387B84F86B
:10DD50004000387B60B1787B84F84100787B38B133
:10DD6000B87B84F84200B87B10B1F87B84F843009C
:10DD7000002084F8430002E0002084F83400372DAE
:10DD800004F1040028BF37250027E562C4E91357D2
:10DD900000F08AFB04F1180000F086FBC5F13800A2
:10DDA000A061304651464246246164626765A765BA
:10DDB00084F85C7000F01CFBB9F1000F206018BF04
:10DDC000C9F80040BDE8F08708480068006880F3A3
:10DDD00008884FF0000080F3148862B661B6BFF384
:10DDE0004F8FBFF36F8F00DF00BF00BF08ED00E073
:10DDF0002DE9F04F85B0814601F08AFF40F60464BA
:10DE00008346C2F20044216988423DD2A06801687D
:10DE100000293BD04FF0000A0DF1040809E000BFD3
:10DE200078603146A0683F6100F042FBA06801685D
:10DE300061B3C068C76805683E1D304600F0F0FA5F
:10DE4000396A3846884797F828004007EED5B86900
:10DE50002844A842E4D8206860B1CDE901A5039721
:10DE600001F046FF206800220023414601F0B4F98A
:10DE70000028DBD14FF0500080F31188BFF36F8F83
:10DE8000BFF34F8FFEE700BF002003E0E168C4E965
:10DE900002100120C9F800005846C4F810B005B0BF
:10DEA000BDE8F08F0000000081B00020009040F637
:10DEB0002050C2F2004000684FF0500181F31188F9
:10DEC000BFF36F8FBFF34F8F013003D0FEE700BF6A
:10DED000009838B9009828B90098002804BF009825
:10DEE0000028F5D001B070478AB040F6046602AC55
:10DEF000C2F200464FF000090DF118080DF1040AB6
:10DF0000B068076827B1C068D0F800B002E000BF71
:10DF10004FF0000B00F01CFF2046FFF769FF02994D
:10DF200011B102F0C5F853E00546AFB15D4513D31A
:10DF300002F0BEF8B068C068C76807F10409484637
:10DF400000F06EFA97F82800410709D400F0FE00AF
:10DF500087F8280031E000BF67B100220FE000BF62
:10DF6000B8693F6100EB0B017960A9421CD9B06828
:10DF700020E000BFF0680068B0FA80F04209306825
:10DF8000ABEB050100F034FC02F092F800BB4EF65A
:10DF900004504FF08051CEF200000160BFF34F8F6C
:10DFA000BFF36F8F14E000BFA5EB0B01814280F03F
:10DFB0009180F068494600F07BFA4FF00009396A19
:10DFC0003846884704E000BFF06800F071FA00BFEF
:10DFD00030680022214601F0CBFA00283FF490AFD0
:10DFE0000298B0F1FF3F06DCDDE903200599904778
:10DFF00002980028ECD4049F786910B1381D00F015
:10E000000FFA5046FFF7F4FE02990929E0D8DFE83D
:10E0100001F0050505393D530505393D97F82810F0
:10E02000039ABD693F6141F0010187F82810AB18E0
:10E030003946834241F8043F04D9904238D2934292
:10E0400003D235E0801AA842BED3396A38468847E1
:10E0500097F828004007BBD53068002856D00398B1
:10E06000B969CDF818900844CDE9070701F040FEE2
:10E07000306800220023414601F0AEF80028A7D105
:10E0800044E000BF97F828001EE000BF97F8281072
:10E0900041F001020399002987F82820B9613FD097
:10E0A0000A18394682423F6141F8042F7FF68CAF4F
:10E0B000B06800F0FDF98BE797F82800810703D4DA
:10E0C000384600F085FA83E700F0FE0087F8280064
:10E0D0007EE700BF306878B14FF000090897CDE9BE
:10E0E000069B01F005FE306800220023414601F046
:10E0F00073F800287FF463AF4FF0500080F311886D
:10E10000BFF36F8FBFF34F8FFEE700BF4FF050009C
:10E1100080F31188BFF36F8FBFF34F8FFEE700BF0F
:10E120004FF0500080F31188BFF36F8FBFF34F8F14
:10E13000FEE7000000000000F0B581B0044600F0EA
:10E1400007FA94F94560012E10DB04F1240503E081
:10E1500070B2013E012809DD286838B1284601F077
:10E160006BFF0028F4D000F09FFCF1E7FF2684F855
:10E17000456000F015FA00F0EBF994F94470012FB6
:10E1800010DB04F1100503E078B2013F012809DD3E
:10E19000286838B1284601F04FFF0028F4D000F07D
:10E1A00083FCF1E784F8446001B0BDE8F04000F082
:10E1B000F7B9000000000000F0B581B0044600F09F
:10E1C000C7FD40F64061C2F20041486840B108789E
:10E1D00001282AD000204FF0000564BB9DE000BF5D
:10E1E00042F2B870C2F20040C21D10F0070322F0E4
:10E1F0000702A0EB020718BF10464FF48032002B35
:10E2000018BF07F58032002388610244CB61083AC9
:10E2100022F007024A60C2E90033121A42604B68DA
:10E220000360C1E90222012008704FF00040002C79
:10E230004FF0000571D020406FD114F0070004F1B9
:10E2400008031EBF181A00F108035FEA43702DD1BE
:10E2500088685A1E824223D2084650F8187FBE466C
:10E260005EF8045F9D423FD23A684AB33C46556827
:10E270009D4229D216683EB375689D422AD2306805
:10E2800040B345689D422BD204684CB365689D42FB
:10E2900002D22268002AEAD104F1040E274623E0C4
:10E2A000002501F005FF68073BD192E04FF05000D8
:10E2B00080F31188BFF36F8FBFF34F8FFEE700BF6E
:10E2C00001F1180010E000BF02F1040E17462046CD
:10E2D0000AE000BF06F1040E3746104604E000BF16
:10E2E00000F1040E074630464A68974214D0EA1AF5
:10E2F000D0F800C0112A3C6804604CD3F8184407D9
:10E300001AD04FF0500080F31188BFF36F8FBFF326
:10E310004F8F00BFFEE700BF002501F0C9FE680770
:10E3200057D04FF0500080F31188BFF36F8FBFF3C9
:10E330004F8F00BFFEE700BF4260CEF8003001F112
:10E3400018031A6882420BD2136883420CD21A68EF
:10E35000824205D2136815468342F2D305E000BF1E
:10E360001D46134601E000BF15466C682A1982421B
:10E37000426802D1224428466A6084189C4206D131
:10E380004C68A3421EBFD3E9003422444260854258
:10E39000036018BF2860DEF800000CF10805D1E921
:10E3A0000223101A8860984238BFC8600878DEF8E7
:10E3B000002000284FF0000018BF42F000423860F3
:10E3C000CEF8002008690130086101F071FE68078D
:10E3D000A7D1284601B0F0BD40F68850C2F20040F7
:10E3E000016819B101680A6D01320A650068704759
:10E3F0004DF6A96321F00101C0F6000340F80C3C82
:10E400004FF0807340F8202C40E902136FF00201B6
:10E4100040F8241CA0F144010846704700000000A9
:10E42000D0E9013201699A60D0F808C04A68824296
:10E430004FF00002CCF8043008BFC1F804C00261FC
:10E440000868013808600868704700000000000094
:10E4500042F6BC13C2F20143036042F2BC70C2F246
:10E46000014008608020106070470000000000003C
:10E4700042F61C63C2F20143036042F61C20C2F262
:10E48000014008604FF48070106070470000000089
:10E4900002464FF0FF3142F8081F00214260C0E9F8
:10E4A00003220160704700000021016170470000F5
:10E4B00010B5D1F800C01CF1010213D000F108041E
:10E4C00062681368634511D853681C68644511D8A5
:10E4D0005A68146864450FD85468A6462368634593
:10E4E000EED90BE00269D2F804E007E09646224636
:10E4F00004E000BF9E4601E096461A46C1F804E0DB
:10E50000CEF808108A60516008610168013101602D
:10E5100010BD000000000000D0F800C043684B6050
:10E520009A688A609A689960086151600CF10101EB
:10E530000160704700000000DFF80C00016841F442
:10E5400070010160704700BF88ED00E0000000002E
:10E550004FF0500080F31188BFF36F8FBFF34F8FE0
:10E5600040F62050C2F200400168002901F101018B
:10E57000016001D0704700BF4EF60450CEF200009B
:10E580000068000608BF70474FF0500080F3118804
:10E59000BFF36F8FBFF34F8FFEE700000000000056
:10E5A00040F62050C2F20040016839B101390160E3
:10E5B00018BF7047002080F3118870474FF050005B
:10E5C00080F31188BFF36F8FBFF34F8FFEE700001A
:10E5D00070B5002808BF70BD40F640650446C2F221
:10E5E00000452878002818BF4FF0004054F8041C5C
:10E5F00008420DD0A4F1080632689AB14FF05000DD
:10E6000080F31188BFF36F8FBFF34F8FFEE700BF1A
:10E610004FF0500080F31188BFF36F8FBFF34F8F1F
:10E62000FEE700BF21EA000044F8040C00F090FB74
:10E6300054F8041CA8680844A86005F1180000BF3D
:10E640000368B3420AD21868B04225D20368B342C5
:10E6500004D218681A46B042F2D301E002461846C6
:10E660005368D418B44202D1194416465160731845
:10E67000834206D16B6898421EBFD0E9000319445B
:10E680007160B242306018BF16606869013068611D
:10E69000BDE8704001F00CBD1A465368D418B4426E
:10E6A000E5D1E1E7000000004EF210000021CEF2BB
:10E6B000000044F6D352C1F262020160816040F270
:10E6C0000801C2F200410968A1FB02124FF0FF31BC
:10E6D00001EB9211416007210160704700000000CA
:10E6E00040F66060EFF305811029C2F2004011D3BB
:10E6F0004EF2F032CEF20002895C0278914209D2E9
:10E700004FF0500080F31188BFF36F8FBFF34F8F2E
:10E71000FEE700BF4EF60C51CEF2000109684068DA
:10E7200001F4E061814298BF70474FF0500080F3E0
:10E730001188BFF36F8FBFF34F8F00BFFEE700005C
:10E7400042F67C6CC2F2014CDCF8002022B3634636
:10E7500053F8082F42B3634653F8102F52B3634661
:10E7600053F8182F62B3634653F8202F72B36346F1
:10E7700053F8282F82B3634653F8302F92B3634681
:10E7800053F8382F002A18BF704707220CEBC2023B
:10E7900019605060704700BF002263460CEBC20254
:10E7A00019605060704700BF01220CEBC202196073
:10E7B0005060704702220CEBC20219605060704733
:10E7C00003220CEBC20219605060704704220CEB6C
:10E7D000C20219605060704705220CEBC20219603A
:10E7E0005060704706220CEBC202196050607047FF
:10E7F00070B515460E460446FFF7AAFE94F844008D
:10E80000FF280DD094F84500FF2810D0FFF7C8FE70
:10E81000A06BA0B12046BDE87040FFF78DBC00BFE3
:10E82000002084F8440094F84500FF28EED1002031
:10E8300084F84500FFF7B4FEA06B0028EAD104F18C
:10E84000240031462A4600F073F92046BDE87040A6
:10E85000FFF772BC0000000070B588B340F6885521
:10E860000446C2F20045686950B14FF0500080F391
:10E870001188BFF36F8FBFF34F8F00BFFEE700BF5C
:10E88000686901306861AE6928680430FFF7C8FD27
:10E890002868A419446005D3286A29680431FFF761
:10E8A00007FE08E0E86929680431FFF701FEE86A1D
:10E8B000844238BFEC6201F0FBFB002818BF70BD3A
:10E8C0004EF604504FF08051CEF200000160BFF3CD
:10E8D0004F8FBFF36F8F70BD70B588B1D1B140F667
:10E8E0008854C2F200446269F2B14FF0500080F3E4
:10E8F0001188BFF36F8FBFF34F8F00BFFEE700BFDC
:10E900004FF0500080F31188BFF36F8FBFF34F8F2C
:10E91000FEE700BF4FF0500080F31188BFF36F8F08
:10E92000BFF34F8FFEE700BF626901326261A269E7
:10E9300003689A42194403D2994203D316E000BFF8
:10E94000994201D3914211D901608E1AA5692068BC
:10E950000430FFF765FD2068AD19456008D3206AD3
:10E9600021680431FFF7A4FD0BE000BF016008E05F
:10E97000E06921680431FFF79BFDE06A854238BFFA
:10E98000E56201F095FB002818BF70BD4EF60450FB
:10E990004FF08051CEF200000160BFF34F8FBFF304
:10E9A0006F8F70BD0000000070B50446FFF7D0FD0A
:10E9B00040F68856002CC2F2004608BF3468251D78
:10E9C0002846FFF72DFDA06A18B104F11800FFF7E3
:10E9D00027FD30687168844201F10100706019D030
:10E9E000F0680138F06094F85D00022809D0012831
:10E9F00004D0002840D1206BFFF7EAFD2046FFF746
:10EA0000E7FDF069006898B1F069C068C0684068C7
:10EA100010E000BF06F140002946FFF77DFDB06819
:10EA20000130B060FFF7BCFD306948B970BD00BF70
:10EA30004FF0FF30F062FFF7B3FD30690028F5D0EA
:10EA40003068844218BF70BD706948B14FF0500003
:10EA500080F31188BFF36F8FBFF34F8FFEE700BFC6
:10EA60004EF604504FF08051CEF200000160BFF32B
:10EA70004F8FBFF36F8F70BD4FF0500080F3118840
:10EA8000BFF36F8FBFF34F8FFEE700000000000061
:10EA900040F68851C2F200418A6B02608969416088
:10EAA000704700000000000040F688500121C2F2CB
:10EAB000004001637047000070B5D8B140F688543B
:10EAC0000D46C2F2004421681831FFF7F1FCA66937
:10EAD00020680430FFF7A4FC681C15D02068AD192D
:10EAE000456019D3206A21680431BDE87040FFF702
:10EAF000DFBC00BF4FF0500080F31188BFF36F8F71
:10EB0000BFF34F8FFEE700BF54F8540B011D2046A2
:10EB1000BDE87040FFF700BDE06921680431FFF7F0
:10EB2000C7FCE06A854238BFE56270BD00000000A6
:10EB3000F0B581B0C0B140F688540D46C2F2004431
:10EB4000164621681831FFF7E7FCA76920680430F2
:10EB5000FFF766FC96B154F8540B011D204601B036
:10EB6000BDE8F040FFF7D8BC4FF0500080F31188AB
:10EB7000BFF36F8FBFF34F8FFEE700BF2068ED1923
:10EB8000456007D3206A2168043101B0BDE8F04038
:10EB9000FFF78EBCE06921680431FFF789FCE06A69
:10EBA000854238BFE56201B0F0BD00000000000002
:10EBB000F0B581B020B3026D04461AB3E06C884210
:10EBC00038BF0846012A1BD1E16A814218D040F6BD
:10EBD0008856C2F200463268A2421DD0A269E062A5
:10EBE000002A42F27C275CBFC0F13800A06101EB33
:10EBF0008100C2F20047616907EB8000814215D0B5
:10EC000001B0F0BD4FF0500080F31188BFF36F8F5B
:10EC1000BFF34F8FFEE700BF4FF0500080F3118825
:10EC2000BFF36F8FBFF34F8FFEE700BF251D284650
:10EC3000FFF7F6FBE06A716A8842294688BF706276
:10EC400000EB800007EB800001B0BDE8F040FFF76B
:10EC500063BC00000000000010B588B0002005A9CA
:10EC6000CDE9050006A804AAFFF7F2FB05980028E5
:10EC700040D0069C002C47D0049A60210791079948
:10EC800060294BD107992063022084F85D0007A812
:10EC90000021CDE900104DF619402AA1C0F6000070
:10ECA00000230294FEF7FCFF2046FEF76DFE40F6BF
:10ECB00088540798C2F20044A062C0B101F070FA13
:10ECC000411C35D0012812D14FF0500080F311883B
:10ECD000BFF36F8FBFF34F8F4FF0FF30E062012023
:10ECE00020610020A061FEF72FF900F099F808B02C
:10ECF00010BD00BF4FF0500080F31188BFF36F8F3D
:10ED0000BFF34F8FFEE700BF4FF0500080F3118834
:10ED1000BFF36F8FBFF34F8FFEE700BF4FF0500080
:10ED200080F31188BFF36F8FBFF34F8FFEE700BFF3
:10ED30004FF0500080F31188BFF36F8FBFF34F8FF8
:10ED4000FEE700BF49444C45000000000000000001
:10ED500040F68850C2F2004041690131416170477C
:10ED600010B540F68854C2F20044606910B1012029
:10ED7000206310BD00202063FEF78EFAE16B88420D
:10ED800004D92268411A536D19445165E06342F277
:10ED90007C21606AC2F2004100EB800251F822300F
:10EDA00073B100EB800201EB820252F8041F131DC5
:10EDB0004968116099421DD0C9682160606210BD28
:10EDC00001EB8202283AD8B153691BBB012817D046
:10EDD00013680BBB022813D052F8143CF3B9032874
:10EDE0000ED052F8283C0438002BA2F15002EAD091
:10EDF000D7E700BF49681160C9682160606210BD33
:10EE00004FF0500080F31188BFF36F8FBFF34F8F27
:10EE1000FEE700BF0138C4E70238C2E70338C0E7A5
:10EE2000B0B584B04EF200404CF27021CEF200003A
:10EE3000C4F20F114B1CD0F800299A420AD14FF0AE
:10EE4000500080F31188BFF36F8FBFF34F8F00BF67
:10EE5000FEE700BFD0F800298A4209D14FF05000E8
:10EE600080F31188BFF36F8FBFF34F8FFEE700BFB2
:10EE700001780291FF21017001788DF8071040F6AA
:10EE800060619DF80720C2F2004102F050020A7052
:10EE900007224A609DF90720B2F1FF3F6CDC072290
:10EEA0009DF807305B008DF807309DF90730002B87
:10EEB0001ED59DF807305B008DF807309DF90730AF
:10EEC000B3F1FF3F1ADC9DF807305B008DF8073087
:10EED0009DF90730B3F1FF3F4ADC9DF80730043A53
:10EEE0005B008DF807309DF90730002BD8D406E081
:10EEF000013A032A4A6005D03EE000BF023A032AE5
:10EF00004A6039D14FF440724A6002990170D0F8DA
:10EF1000201941F47001C0F82019D0F8201941F0EF
:10EF20007041C0F82019FFF7BFFB40F620540025C0
:10EF3000C2F200442560FFF7FFFA4EF63470CEF2BD
:10EF40000000016841F040410160FEF73DFFFFF71E
:10EF500007FF039520684FF0500181F31188BFF33C
:10EF60006F8FBFF34F8F013012D000BFFEE700BF9D
:10EF7000033A032A4A60C5D04FF0500080F311884D
:10EF8000BFF36F8FBFF34F8FFEE700BF039838B911
:10EF9000039828B90398002804BF03980028F5D0E7
:10EFA000002004B0B0BD000080B54FF0500080F3E9
:10EFB0001188BFF36F8FBFF34F8F00F0BDFE30B1EC
:10EFC0004EF604504FF08051CEF200000160002058
:10EFD00080F3118880BD0000F0B581B090B1064685
:10EFE000484314460F465030FFF7E6F80546B0B3E5
:10EFF0004FF0000085F8460077B105F15000286019
:10F000000BE000BF4FF0500080F31188BFF36F8F0B
:10F01000BFF34F8FFEE700BF2D60C5E90F67FFF715
:10F0200097FAD5E90F012A68002701FB0023013870
:10F0300000FB0120AF636A60C5E90230FF2085F85C
:10F04000440085F8450005F11000FFF721FA05F1AD
:10F050002400FFF71DFAFFF7A3FA85F84C40284675
:10F0600001B0F0BD0000000070B582B070B11C4668
:10F07000B3B1F9B9F2B14FF0500080F31188BFF38A
:10F080006F8FBFF34F8F00BFFEE700BF4FF0500000
:10F0900080F31188BFF36F8FBFF34F8FFEE700BF80
:10F0A0004FF0500080F31188BFF36F8FBFF34F8F85
:10F0B000FEE700BF51B14AB94FF0500080F311880C
:10F0C000BFF36F8FBFF34F8FFEE700BF5023019355
:10F0D000019B502B08D1069E019B4FF0010384F841
:10F0E000463059B122600AE04FF0500080F3118899
:10F0F000BFF36F8FBFF34F8FFEE700BF2460C4E9FB
:10F100000F01FFF725FAD4E90F012268002501FB62
:10F110000023013800FB0120A5636260C4E90230CE
:10F12000FF2084F8440084F8450004F11000FFF744
:10F13000AFF904F12400FFF7ABF9FFF731FA84F8D7
:10F140004C60204602B070BD70B518B304460E4640
:10F15000FFF7FEF9D4E90F012268002501FB002327
:10F16000013800FB0120A5636260C4E902304FF062
:10F17000FF0084F8440084F8450004F110009EB1BB
:10F18000FFF786F904F12400FFF782F9FFF708FA88
:10F19000012070BD4FF0500080F31188BFF36F8FD6
:10F1A000BFF34F8FFEE700BF01680029EED000F0EB
:10F1B00043FF0028EAD04EF604504FF08051CEF2C3
:10F1C00000000160BFF34F8FBFF36F8FFFF7E8F9C7
:10F1D000012070BD000000002DE9F04F83B00292C5
:10F1E000C0B104461D4617460E46E9B1022D03D1B3
:10F1F000E06B012840F0908000F07AFD10BB0FB367
:10F200004FF0500080F31188BFF36F8FBFF34F8F23
:10F21000FEE700BF4FF0500080F31188BFF36F8FFF
:10F22000BFF34F8FFEE700BF206C0028DED04FF009
:10F23000500080F31188BFF36F8FBFF34F8F00BF73
:10F24000FEE700BFFFF784F9022DA06B6ED0E16BE3
:10F2500088426BD304F1100801206F460DF10809B4
:10F260000DE000BF2046FEF767FF00F021FFFFF72B
:10F270006FF9A06BE16B88424FF0000056D3029902
:10F28000002900F07B80C00702D03846FFF700FC61
:10F29000FFF786F9FFF75CFDFFF75AF994F8440091
:10F2A000FF282DD094F84500FF2830D0FFF778F9DB
:10F2B0003846494600F028FB002865D1FFF748F999
:10F2C000D4F838A0D4F83CB0FFF76AF9DA45C9D1D0
:10F2D00002994046FFF7F0FB2046FEF72DFF00F0B5
:10F2E000E7FE0028C3D14EF604504FF08051CEF215
:10F2F00000000160BFF34F8FBFF36F8FB7E700BF10
:10F30000002084F8440094F84500FF28CED1002066
:10F3100084F84500CAE700BF4FF0500080F3118821
:10F32000BFF36F8FBFF34F8FFEE700BFA76B226C59
:10F33000D2B19DB3E0683146F1F734FCE168206C4E
:10F340002268091A9142E16003D24042A168084450
:10F35000E060A81E3946B0FA80F0002F18BF0121E6
:10F36000400908403F1A26E02068002520BBA0681D
:10F3700000F0CEFDA56005461EE000BFFFF710F9C6
:10F38000002003B0BDE8F08F2046FEF7D5FE00F068
:10F390008FFE002003B0BDE8F08F00BF60683146EB
:10F3A000F1F700FC216CD4E901020844606090424E
:10F3B00001D3206860600025781CA06354F8240FF6
:10F3C000A0B1204600F038FE50B14EF604504FF088
:10F3D0008051CEF200000160BFF34F8FBFF36F8FFB
:10F3E000FFF7DEF8012003B0BDE8F08F002DF7D065
:10F3F0004EF604504FF08051CEF200000160BFF392
:10F400004F8FBFF36F8FFFF7CBF8012003B0BDE83C
:10F41000F08F0000000000002DE9F04700B3054622
:10F420001E4614460F4629B3022E02D1E86B01286E
:10F4300052D1FFF755F9EFF311884FF0500080F3E8
:10F440001188BFF36F8FBFF34F8F022EA86B1FD0B1
:10F45000E96B88421CD3002088F31188BDE8F0874F
:10F460004FF0500080F31188BFF36F8FBFF34F8FC1
:10F47000FEE700BF286C0028D6D04FF0500080F384
:10F480001188BFF36F8FBFF34F8F00BFFEE700BF40
:10F4900095F84590A86BD5F838A02A6C32B36EB3B6
:10F4A000E8683946F1F77EFBE968286C2A68091A92
:10F4B0009142E96003D24042A9680844E860B01E66
:10F4C0005146B0FA80F0BAF1000F18BF012140098F
:10F4D0000840AAEB000A1EE04FF0500080F31188AC
:10F4E000BFF36F8FBFF34F8FFEE700BF286890B95F
:10F4F000A86800F00DFD0020A8600CE0686839469F
:10F50000F1F750FB296CD5E901020844686090428C
:10F5100001D328686860B9F1FF0F0AF10100A86300
:10F5200010D155F8240FB8B1284600F085FD0146EA
:10F530000120002C18BF002914D188F31188BDE8E0
:10F54000F08700BF09F1010085F84500012088F32C
:10F550001188BDE8F08700BF012088F31188BDE85D
:10F56000F08700BF0120206088F31188BDE8F08794
:10F570002DE9F04F83B0029290B1044616460D4635
:10F5800000294BD000F0B4FBA0B99EB14FF0500061
:10F5900080F31188BFF36F8FBFF34F8FFEE700BF7B
:10F5A0004FF0500080F31188BFF36F8FBFF34F8F80
:10F5B000FEE700BFFEF7CCFFD4F838A0BAF1000F89
:10F5C0003AD0226C52B1D4E902308118E1609942FC
:10F5D00001D32168E1602846F1F7E4FAAAF10100BD
:10F5E000A06354F8100F002800F08C80204600F033
:10F5F00023FD002800F08E804EF604504FF080511D
:10F60000CEF2000001260160BFF34F8FBFF36F8F72
:10F61000FEF7C6FF304603B0BDE8F08F206C00282F
:10F62000B0D04FF0500080F31188BFF36F8FBFF35D
:10F630004F8F00BFFEE700BF002E4FF000066AD0DC
:10F64000EB4604F124085846FFF722FA0DF10809A9
:10F65000FEF7A6FFFFF77CFBFEF77AFF94F8440065
:10F66000FF2808BF84F8446094F84500FF2808BFCD
:10F6700084F84560FEF794FF5846494600F044F987
:10F6800060B12046FEF758FD00F012FDFEF760FF66
:10F69000A76BFEF785FF1FBB44E000BFFEF758FFD6
:10F6A000A76BFEF77DFF2FB12046FEF745FD00F06A
:10F6B000FFFC15E002994046FFF7FEF92046FEF7F1
:10F6C0003BFD00F0F5FC58B94EF604504FF0805168
:10F6D000CEF200000160BFF34F8FBFF36F8F00BF0A
:10F6E000FEF736FFD4F838A0BAF1000F7FF469AF07
:10F6F00002980028ACD10026FEF752FF304603B036
:10F70000BDE8F08F0126FEF74BFF304603B0BDE8A1
:10F71000F08F00BF0126FEF743FF304603B0BDE87F
:10F72000F08F00BF0026304603B0BDE8F08F000028
:10F730002DE9F04F83B0029160B10446006C98B19E
:10F740004FF0500080F31188BFF36F8FBFF34F8FDE
:10F75000FEE700BF4FF0500080F31188BFF36F8FBA
:10F76000BFF34F8FFEE700BF0D4600F0C1FA58B956
:10F7700055B14FF0500080F31188BFF36F8FBFF386
:10F780004F8F00BFFEE700BFFEF7E2FEA16BF9B1AD
:10F79000481EA063206810B9FEF71EFEA06054F852
:10F7A000100F70B1204600F047FC50B14EF60450E7
:10F7B0004FF08051CEF200000160BFF34F8FBFF3D6
:10F7C0006F8F0124FEF7ECFE204603B0BDE8F08FFA
:10F7D00004F124094FF0000B01206E4602AF4FF0F8
:10F7E00000082AE0FEF7DCFEFFF7B2FAFEF7B0FEF3
:10F7F00094F84400FF2808BF84F844B094F845000A
:10F80000FF2808BF84F845B0FEF7CAFE30463946E7
:10F8100000F07AF8D0B12046FEF78EFC00F048FCEC
:10F82000FEF796FEA56BFEF7BBFE002D4ED0FEF751
:10F830008FFEA16B00200029AAD10299C1B3C00795
:10F84000D0D03046FFF724F9CCE700BFFEF780FEAA
:10F85000D4F838A0FEF7A4FEBAF1000F06D0204677
:10F86000FEF76AFC00F024FCE1E700BF206838B92D
:10F87000FEF76EFEA06800F093FB8046FEF790FE58
:10F8800002994846FFF718F92046FEF755FC00F0AC
:10F890000FFC0028CBD14EF604504FF08051CEF231
:10F8A00000000160BFF34F8FBFF36F8FBFE700BF52
:10F8B000B8F1000F20D04FF0500080F31188BFF353
:10F8C0006F8FBFF34F8F00BFFEE700BFB8F1000F8F
:10F8D00008D0FEF73DFE606A50B1206B0068C0F1B1
:10F8E000380106E00024204603B0BDE8F08F00BFD9
:10F8F0000021A068FFF75CF90024FEF751FE2046C6
:10F9000003B0BDE8F08F0000B0B5D8B10D4619B313
:10F910000446FEF71DFE40F6885CC2F2004CDCF89F
:10F9200018202968481C21D06368DCF838E09A4226
:10F9300022D3206886451FD00124FEF731FE2046E1
:10F94000B0BD00BF4FF0500080F31188BFF36F8F40
:10F95000BFF34F8FFEE700BF4FF0500080F31188D8
:10F96000BFF36F8FBFF34F8FFEE700BF0024FEF79A
:10F9700017FE2046B0BD00BFD21A91420CD9881A9A
:10F980002860DCF838002060DCF818006060002493
:10F99000FEF706FE2046B0BD012400202860FEF7D9
:10F9A000FFFD2046B0BD00002DE9F04383B00746BF
:10F9B0009000984615468946FEF7FEFBF8B10646CC
:10F9C0006020FEF7F9FBB8B104460022DDE90A1019
:10F9D0002663434684F85D202A46CDE90010384668
:10F9E00049460294FEF75CF92046FDF7CDFF012061
:10F9F00003B0BDE8F08300BF3046FEF7E9FD4FF0ED
:10FA0000FF3003B0BDE8F08370B586B00B9CDCB16D
:10FA10000C9E1EB360250495049D602D28D1DDF851
:10FA200028C0049D3463022586F85D50CDF800C0DF
:10FA300005ADCDE90156FEF733F93046FDF7A4FFD9
:10FA4000059806B070BD00BF4FF0500080F31188DC
:10FA5000BFF36F8FBFF34F8FFEE700BF4FF0500033
:10FA600080F31188BFF36F8FBFF34F8FFEE700BFA6
:10FA70004FF0500080F31188BFF36F8FBFF34F8FAB
:10FA8000FEE7000000000000F0B581B0E0B10446E0
:10FA90001F4616460D46FEF75BFD002F4FF0020194
:10FAA0001CBFA06D386094F85C00042E84F85C10D4
:10FAB00014D8DFE806F0280321274F00A16D294361
:10FAC000A165012867D120E04FF0500080F3118834
:10FAD000BFF36F8FBFF34F8FFEE700BFA16D013102
:10FAE00011D04FF0500080F31188BFF36F8FBFF338
:10FAF0004F8F00BFFEE700BFA16D0131A165012856
:10FB000049D102E0A565012845D1251D2846FEF70B
:10FB100087FC40F68856E06AC2F20046716A884265
:10FB200042F27C2188BF706200EB8000C2F200418B
:10FB300001EB80002946FEF7EFFCA06A90B14FF080
:10FB4000500080F31188BFF36F8FBFF34F8F00BF5A
:10FB5000FEE700BF02281BD10024FEF721FD20464E
:10FB600001B0F0BDE06A3168C96A884213D94EF627
:10FB700004504FF08051CEF2000001240160BFF329
:10FB80004F8FBFF36F8FFEF70BFD204601B0F0BD26
:10FB9000A5650128B9D00124FEF702FD204601B079
:10FBA000F0BD0000000000002DE9F04120B3044644
:10FBB0001F4616460D46FEF793FDEFF311884FF0F2
:10FBC000500080F31188BFF36F8FBFF34F8F002F6A
:10FBD0001CBFA06D386094F85C00042E4FF0020149
:10FBE00084F85C1012D8DFE806F026031F253500E4
:10FBF000A16D29431AE000BF4FF0500080F3118837
:10FC0000BFF36F8FBFF34F8FFEE700BFA16D0131D0
:10FC100011D04FF0500080F31188BFF36F8FBFF306
:10FC20004F8F00BFFEE700BFA16D0131A165012824
:10FC300027D102E0A565012823D1A06A90B14FF039
:10FC4000500080F31188BFF36F8FBFF34F8F00BF59
:10FC5000FEE700BF022811D1002088F31188BDE81B
:10FC6000F08100BF40F68856C2F20046706968B164
:10FC700004F1180106F168001AE000BFA56501282B
:10FC8000DBD0012088F31188BDE8F081251D2846CE
:10FC9000FEF7C6FBE06A716A884242F27C2188BFA7
:10FCA000706200EB8000C2F2004101EB8000294647
:10FCB000FEF732FCE06A3168C96A88420AD90698C0
:10FCC00000281CBF012101600120306388F31188E6
:10FCD000BDE8F081012088F31188BDE8F0810000C3
:10FCE00040F68850C2F200400068704700000000F3
:10FCF00040F68850C2F20040016929B14069B0FA6B
:10FD000080F040094000704701207047000000006B
:10FD100040F68850C2F20040806970470000000041
:10FD200080B5FEF7DDFC40F68850C2F200408069E5
:10FD300080BD0000000000002DE9F04381B040F6D6
:10FD40008856C2F20046706940B1706B00240130E1
:10FD50007063204601B0BDE8F08300BFB06910F1C8
:10FD60000109C6F8189020D3F069006850B14FF02F
:10FD7000500080F31188BFF36F8FBFF34F8F00BF28
:10FD8000FEE700BFF069316AF1613062B06B0130AB
:10FD9000B063F069006828B1F069C068C068406865
:10FDA00002E000BF4FF0FF30F062F06A42F27C28C0
:10FDB0008145C2F2004801D200242EE0F0690024FF
:10FDC000006813E0F86A716A8842294688BF706249
:10FDD00000EB800008EB8000FEF79EFBF86A3168BC
:10FDE000C96AF269884228BF0124106890B1F0699D
:10FDF000C068C7683D4655F8040F81450CD32846B6
:10FE0000FEF70EFBB86A0028DCD007F11800FEF7F9
:10FE100007FBD7E74FF0FF30F0623068C06A00EBB5
:10FE2000800058F82000012888BF0124306B00288A
:10FE300018BF0124204601B0BDE8F0830000000097
:10FE40002DE9F0411E46154688460746FEF780FB21
:10FE500040F68854C2F20044206890F85C00022802
:10FE600038D02068816D21EA0701816520684FF054
:10FE7000010180F85C106EB3A76920680430FEF7BA
:10FE8000CFFA701C0AD02068F61946600ED3206A9B
:10FE900021680431FEF70CFB11E000BF204650F84A
:10FEA000541B0431FEF738FB09E000BFE06921680C
:10FEB0000431FEF7FDFAE06A864238BFE6624EF68C
:10FEC00004504FF08051CEF200000160BFF34F8F1D
:10FED000BFF36F8FFEF764FBFEF73AFB15B12068A6
:10FEE000806D28602068002590F85C0002284FF0A3
:10FEF000000005D1216801258A6D22EA08028A6581
:10FF0000216881F85C00FEF74BFB2846BDE8F081D4
:10FF100070B588B140F688560446C2F20046306893
:10FF2000A0420BD04FF0500080F31188BFF36F8FC9
:10FF3000BFF34F8FFEE700BF002070BD206D18B3E8
:10FF4000013820654FF000001DD1E16AE26C91425A
:10FF500008BF70BD251D2846FEF762FAE06CE0621E
:10FF6000C0F13801A161716A884242F27C2188BFE8
:10FF7000706200EB8000C2F2004101EB8000294674
:10FF8000FEF7CAFA012070BD4FF0500080F31188CF
:10FF9000BFF36F8FBFF34F8FFEE70000000000003C
:10FFA000F0B581B010B340F688560446C2F2004660
:10FFB000C06A3168C96A88421CD2A169002904D488
:10FFC0003168C96AC1F13801A16100EB800042F2D9
:10FFD0007C27C2F20047616907EB8000814213D0A1
:10FFE0003068C06AE062012001B0F0BD002001B0BD
:10FFF000F0BD00BFE16C3068C26A0020914238BF9A
:020000040801F1
:10000000012001B0F0BD00BF251D2846FEF708FA0B
:100010003068C06AE062716A8842294688BF7062AF
:1000200000EB800007EB8000FEF776FA012001B0BC
:10003000F0BD00000000000070B5C068C5686DB17B
:1000400005F118042046FEF7EBF940F68856C2F297
:100050000046706960B106F168001AE04FF0500088
:1000600080F31188BFF36F8FBFF34F8FFEE700BFA0
:100070002C1D2046FEF7D4F9E86A716A884242F2E4
:100080007C2188BF706200EB8000C2F2004101EB6E
:1000900080002146FEF740FAE86A3168C96A884262
:1000A00002D90120306370BD002070BD0000000047
:1000B0002DE9F04140F68855C2F20045686968B103
:1000C000FEF746FA686901386861686980B1002402
:1000D000FEF766FA2046BDE8F08100BF4FF0500001
:1000E00080F31188BFF36F8FBFF34F8FFEE700BF20
:1000F000E8680028EBD0A86E88B342F27C264FF067
:100100000108C2F2004600BF686FC76807F1180017
:10011000FEF786F93C1D2046FEF782F9F86A696A07
:100120008842214688BF686200EB800006EB8000B1
:10013000FEF7F2F9F86A2968C96A884228BFC5F84B
:100140003080A86E0028DFD1E869006820B1E86936
:10015000C068C068406801E04FF0FF30E8626C6B37
:100160004CB10126FFF7E8FD002818BF2E63013CC3
:10017000F8D100206863286B0028A8D04EF6045000
:100180004FF08051CEF2000001240160BFF34F8F89
:10019000BFF36F8FFEF704FA2046BDE8F081000040
:1001A00070B586B0FEF7D4F940F60466C2F2004698
:1001B000306808BB06F114042046FEF769F906F121
:1001C00028052846FEF764F942F28C1242F22C23ED
:1001D000C2F20042C2F200430A201021C6E90245E1
:1001E00000250095FEF740FF306028B140F2EC3169
:1001F000C0F60101FEF7A4FAFEF7D2F93068D8B1D3
:10020000002004A9CDE9040005A803AAFEF730F9EF
:10021000DDE9032002210023CDE900104DF6E9605D
:100220000AA1C0F60000059D0295FFF7EDFB706086
:1002300010B1012006B070BD4FF0500080F311885E
:10024000BFF36F8FBFF34F8FFEE700BF546D722077
:100250005376630030380A2801D20120704700200D
:100260007047000010B500290AD00878002807D090
:1002700005487844F0F78CFD002801D0002010BD1F
:100280000248784410BD0000620200005A020000DB
:10029000F1EE100A4FF6FF71C0F2C03120EA010002
:1002A00040F04070E1EE100A7047000000000000CE
:1002B00000000000303132333435363738394142AE
:1002C00043444546403058003031323334353637B8
:1002D0003839616263646566403078000400000864
:1002E00000000000000000020001000010000000FB
:1002F00000000000000000000000000000000000FE
:1003000000000000010000000200000003000000E7
:1003100004000000000000000500000000000000D4
:1003200000000000000000000600000000000000C7
:1003300000000000000000000700000000000000B6
:100340000102030401020304060708090100020078
:100350000400060008000A000C0010002000400005
:1003600080000001AA040108000000000000000055
:10037000000000000000000000100000300000003D
:100380000000000000000000A704010800000000B9
:100390000000000000000000000000000004000059
:1003A000180000000000000000000000010101032F
:1003B000070100000804020408010101E00301082C
:1003C000000000000000000000000000000000002D
:1003D0000002000018000000000000000000000003
:1003E00064656661756C745461736B00546D725111
:1003F000002564002020537461747573203A202511
:10040000730D0A202043684C582020203A20252EC6
:100410003366202043684C59203A20252E33660D40
:100420000A2020436852582020203A20252E336687
:10043000202043685259203A20252E33660D0A2089
:1004400020436852657320203A20252E33660D0A1A
:10045000202053774C202020203A20256420202083
:100460002053775220203A2025640D0A20204D6F1A
:1004700075736520203A20583D256420593D256438
:10048000205A3D256420284C3A256420523A2564A0
:10049000290D0A20204B6579732020203A203078DE
:1004A000253034580D0A007263005461736B5F4944
:1004B0006E697400E805010800000024280D0000A2
:1004C0000803000818060108280D002498510100AF
:1004D000440300081001000043000000F8FFFFFF84
:1004E0000040404040404040404041414141414047
:1004F00040404040404040404040404040404040FC
:10050000400502020202020202020202020202028A
:10051000022020202020202020202002020202028F
:1005200002029090909090901010101010101010E7
:1005300010101010101010101010101002020202F3
:100540000202888888888888080808080808080837
:100550000808080808080808080808080202020233
:10056000400000000000000000000000000000004B
:10057000000000000000000000000000000000007B
:10058000000000000000000000000000000000006B
:10059000000000000000000000000000000000005B
:1005A000000000000000000000000000000000004B
:1005B000000000000000000000000000000000003B
:1005C000000000000000000000000000000000002B
:1005D000000000000000000000000000000000001B
:1005E00000000000000000004201521008FF90D0FF
:1005F000030090D00301FF01FF01FF01FF01FF0194
:10060000FF01FF01FF01FF015B02C32F02FF010198
:08061000FFB155AAAAAAAA0035
:04000005080002CD20
:00000001FF
